:100000000C94E9300C941A310C941A310C941A3176
:100010000C941A310C94F2D30C941A310C941A31BA
:100020000C9483D70C941A310C942D880C941A31AB
:100030000C941A310D9461440C941A310C941A31B9
:100040000C941A310C9491A80C941A310C941A3116
:100050000C941A310C941A310D949B1D0D94074683
:100060000C941A310D9475760C941A310C941A3143
:100070000C941A310C941A310C941A310C941A31D4
:100080000C941A310C941A310C941A310C941A31C4
:100090000D9431760C941A310C941A310C941A3157
:1000A0000C941A310C941A310C941A310C941A31A4
:1000B0000C941A310C941A310C941A310C941A3194
:1000C0000C941A310C941A310C941A310D94127A42
:1000D0000C941A310C941A310C941A310C941A3174
:1000E0000C941A31E086E486EA86F3860C87298729
:1000F00066879D87799B809B329B009BD09AB89D99
:10010000A69B869C099D6B9D22A738A74BA758A745
:1001100062A790A7B1A7B7A7C5A7C8A7CAA7D4A722
:10012000E5A7F6A79C014A013201680196017E010C
:100130003C01AA01880190016E0162012801800141
:100140007E017201AE01BE018C016601780186015B
:1001500074014E014C01B4016C01600182019401F3
:100160004201BC014E01AC012A01840170017C01F5
:100170003601A6013A016A018A01A801A2019E0185
:10018000B601084AD73B3BCE016E84BCBFFDC12FF0
:100190003D6C74319ABD56833DDA3D00C77F11BE78
:1001A000D9E4BB4C3E916BAAAABE000000803F057B
:1001B000A84CCDB2D44EB93836A9020C50B99186AC
:1001C00088083CA6AAAA2ABE000000803F07634216
:1001D00036B79BD8A71A39685618AEBAAB558C1DDE
:1001E0003CB7CC5763BD6DEDFD753EF6177231BF60
:1001F000000000803F08000000BE922449123EAB80
:10020000AAAA2ABECDCCCC4C3E00000080BEABAA30
:10021000AAAA3E00000000BF000000803F000000CE
:100220000000084178D3BB4387D1133D190E3CC36E
:10023000BD4282AD2B3E68EC8276BED98FE1A93EED
:100240004C80EFFFBE01C4FF7F3F000000000000B4
:100250000D94AA420D94A6450D941F8F0D942F174F
:100260000D94A88E0D9479420D9488170D94454DE8
:100270000D946E8E0D94734D0D948E420D94718D70
:100280000D945A8C0D9488450D94F1420D947D4344
:100290000D94379C0D948A420D944B450D94BA45AC
:1002A0000D94B68C0D946F430D94E28E0D940C76E4
:1002B0000D94518E0D948B8E0D94F3750D94F06406
:1002C0000D9465450D94A6420D94F98C0D94284526
:1002D0000D947D420D94794D0D945B450D94A04293
:1002E0000D94314D0D94B4420D9441450D940E8FF3
:1002F0000D942D450D94274A0D943F4D0D94C14208
:100300000D94AE420D946F450D94B0450D94374554
:100310000D9498420D947F4D0D9423450D9473A731
:100320000D949C420D94E7420D9479450D948342BF
:100330000D94F6420D94268D0D9487420D94A94D8F
:100340000D94C58E0D949B4D0D94AB8D0D94574D12
:100350000D948D4D0D9492420D949C450D94B84290
:100360000D94888C0D94FF8E0D9453450D94C04DC3
:100370000D94EB420D94338E0D9492450D94BC4236
:100380004E414E494E495459494E46CDCCCC3D0A7A
:10039000D7233C17B7D13877CC2B329595E6241F5D
:1003A000B14F0A000020410000C84200401C462016
:1003B000BCBE4CCA1B0E5AAEC59D746364696E6F99
:1003C00070737578585B0000407A10F35A00A07281
:1003D0004E18090010A5D4E80000E8764817000080
:1003E000E40B54020000CA9A3B000000E1F505004E
:1003F0000080969800000040420F000000A0860197
:10040000000000102700000000E803000000006466
:1004100000000000000A00000000000100000000D1
:10042000002C76D888DC674F0823DFC1DFAE59E1A6
:10043000B1B796E5E3E453C63AE651997696E8E615
:10044000C28426EB898C9B62ED407C6FFCEFBC9CE8
:100450009F40F2BAA56FA5F490055A2AF75C936BFA
:100460006CF9676DC11BFCE0E40D47FEF520E6B5B5
:1004700000D0ED902E0300943577050080841E088F
:100480000000204E0A000000C80C333333330F98AD
:100490006E12831141EF8D2114893BE65516CFFE74
:1004A000E6DB18D1844B381BF77C1D901DA4BBE400
:1004B00024203284725E228100C9F124ECA1E53D42
:1004C0002725642062797465732077726974746576
:1004D0006E20746F20454550524F4D20617420614D
:1004E0006464726573732030782530347800443347
:1004F000202D20526561642F57726974652045452F
:1005000050524F4D0A0020436F756E7420583A20A8
:10051000005344207072696E74696E67206279744A
:100520006520004E6F7420696E206661726D206DCB
:100530006F64652E00416374697665204578747236
:10054000756465723A2000496E76616C6964206555
:1005500078747275646572005A204F6666736574AC
:1005600000556E6B6E6F776E20636F6D6D616E649C
:100570003A2022004D32303020496E76616C696439
:1005800020657874727564657220007A5F6D617899
:100590003A20007A5F6D696E3A2000795F6D61786C
:1005A0003A2000795F6D696E3A2000785F6D61785E
:1005B0003A20006F70656E005452494747455245D6
:1005C0004400785F6D696E3A20005265706F7274F6
:1005D000696E6720656E6473746F702073746174E4
:1005E0007573000053494C454E54004E4F524D41D7
:1005F0004C002553204D4F44453A205065726365A9
:100600006E7420646F6E653A2025643B20707269B9
:100610006E742074696D652072656D61696E696EB6
:100620006720696E206D696E733A2025640A004563
:100630006E642066696C65206C697374004265673E
:10064000696E2066696C65206C6973740025643A74
:100650002025640A000A50494E44412074656D709B
:10066000657261747572653A20252E3166205A20B4
:10067000736869667420286D6D293A20252E3366CB
:10068000000A537465703A2025642F360A000A5315
:100690007465703A2025642F362028736B6970705A
:1006A0006564290A50494E44412074656D70657235
:1006B00061747572653A202564205A2073686966F2
:1006C0007420286D6D293A300A000A5A45524F3A73
:1006D00020252E33660A0073746172742074656D70
:1006E00070657261747572653A20252E31660A0054
:1006F00025642020252E326600255320583A2025D7
:100700002E356620593A20252E3566205A3A202566
:100710002E35660A00536C6565702E2E2E004E6FC6
:100720007420696E206661726D206D6F64652E00A5
:1007300025640045303A25642052504D0A50524EEF
:10074000303A25642052504D0A00256400417574EA
:100750006F0020452F443D00416476616E63652043
:100760004B3D004D323230205325690025534669F8
:100770006C616D656E742073657474696E67733A2D
:100780002044697361626C65640A00255346696C94
:10079000616D656E742073657474696E67733A0A6F
:1007A00025532020204D3230302044252E32660A39
:1007B000002553526574726163743A20533D4C6551
:1007C0006E67746820286D6D2920463A5370656500
:1007D0006420286D6D2F6D29205A3A205A4C696685
:1007E0007420286D6D290A25532020204D32303782
:1007F0002053252E32662046252E3266205A252E7D
:1008000032660A25535265636F7665723A20533D0E
:100810004578747261206C656E67746820286D6D10
:100820002920463A537065656420286D6D2F6D2927
:100830000A25532020204D3230382053252E326691
:100840002046252E32660A25534175746F2D526558
:1008500074726163743A20533D3020746F20646970
:100860007361626C652C203120746F20696E746531
:10087000727072657420657874727564652D6F6E20
:100880006C79206D6F766573206173207265747268
:1008900061637473206F72207265636F766572692D
:1008A00065730A25532020204D32303920532564AA
:1008B0000A002553504944206865617462656420CC
:1008C00073657474696E67733A0A25532020204D4E
:1008D0003330342050252E32662049252E326620B2
:1008E00044252E32660A002553504944207365740E
:1008F00074696E67733A0A25532020204D333031D6
:100900002050252E32662049252E32662044252E81
:1009100032660A0025535374657073207065722027
:10092000756E69743A0A255320204D3932205825B6
:100930002E32662059252E3266205A252E32662008
:1009400045252E32660A25534D6178696D756D20F7
:10095000666565647261746573202D206E6F726DBB
:10096000616C20286D6D2F73293A0A255320204D84
:100970003230332058252E32662059252E326620FB
:100980005A252E32662045252E32660A25534D61A2
:1009900078696D756D206665656472617465732034
:1009A0002D20737465616C746820286D6D2F732918
:1009B0003A0A255320204D3230332058252E3266F6
:1009C0002059252E3266205A252E32662045252EA6
:1009D00032660A25534D6178696D756D20616363D8
:1009E000656C65726174696F6E202D206E6F726D1B
:1009F000616C20286D6D2F7332293A0A255320200F
:100A00004D3230312058256C752059256C75205A8F
:100A1000256C752045256C750A25534D6178696DE7
:100A2000756D20616363656C65726174696F6E20BA
:100A30002D20737465616C746820286D6D2F73327E
:100A4000293A0A255320204D3230312058256C7523
:100A50002059256C75205A256C752045256C750A22
:100A60002553416363656C65726174696F6E3A20EA
:100A7000533D616363656C65726174696F6E2C20B0
:100A8000543D7265747261637420616363656C6563
:100A9000726174696F6E0A255320204D3230342004
:100AA00053252E32662054252E32660A2553416482
:100AB00076616E636564207661726961626C6573EC
:100AC0003A20533D4D696E206665656472617465B8
:100AD00020286D6D2F73292C20543D4D696E207494
:100AE000726176656C206665656472617465202844
:100AF0006D6D2F73292C20423D6D696E696D756D8A
:100B0000207365676D656E742074696D6520286D4E
:100B100073292C20583D6D6178696D756D20585989
:100B2000206A65726B20286D6D2F73292C20205A46
:100B30003D6D6178696D756D205A206A65726B2014
:100B4000286D6D2F73292C2020453D6D6178696DCE
:100B5000756D2045206A65726B20286D6D2F732995
:100B60000A255320204D3230352053252E32662061
:100B700054252E32662042252E32662058252E32EC
:100B8000662059252E3266205A252E3266204525AC
:100B90002E32660A2553486F6D65206F6666736551
:100BA0007420286D6D293A0A255320204D323036A5
:100BB0002058252E32662059252E3266205A252EA1
:100BC00032660A004625642025640A004D4D5520F2
:100BD0003C3D2027462564202564270A00504944CF
:100BE000204175746F74756E652066696E697368EF
:100BF0006564212050757420746865206C6173747D
:100C0000204B702C204B6920616E64204B64206364
:100C10006F6E7374616E74732066726F6D206162A3
:100C20006F766520696E746F20436F6E66696775B5
:100C3000726174696F6E2E6800504944204175746A
:100C40006F74756E65206661696C656421207469D6
:100C50006D656F75740020403A00543A00423A00C6
:100C6000504944204175746F74756E6520666169E2
:100C70006C6564212054656D706572617475726570
:100C800020746F6F206869676800204B643A200009
:100C9000204B693A2000204B703A200020436C61C1
:100CA000737369632050494420002054753A200032
:100CB000204B753A2000206D61783A2000206D6944
:100CC0006E3A200020643A200020626961733A2065
:100CD0000020453A00205A3A0020593A0020453A6F
:100CE00000205A3A0020593A00583A00005A300081
:100CF0005A31005930005931005830005831004500
:100D00006E642073746F70732064696167002E00D5
:100D100044656C6574696F6E206661696C65642CEE
:100D20002046696C653A200046696C652064656CF4
:100D3000657465643A004E6F742053442070726984
:100D40006E74696E67005072696E742073617665A7
:100D500064005344207072696E742070617573650D
:100D600064000A002F000A002F2F20616374696F4E
:100D70006E3A63616E63656C0043524153485F4352
:100D8000414E43454C0043524153485F5245434F07
:100D90005645520043524153485F5245434F5645D2
:100DA0005200222832290054004475706C6963692E
:100DB0007420542D636F64652069676E6F7265647B
:100DC0002E0A004475706C6963697420542D636F3A
:100DD00064652069676E6F7265642E0A00496E76DD
:100DE000616C6964205420636F64652E00556E6BDE
:100DF0006E6F776E204D20636F64653A20257320F7
:100E00000A006E6F2076616C696420636F6D6D619E
:100E10006E64002C20002C20002C20006E2F61001E
:100E20002C20002C20002C20006E2F61002F005061
:100E30003A005761697420666F722050494E4441F0
:100E4000207461726765742074656D706572617479
:100E50007572653A004C414E472053454C20464F31
:100E600052434544002228312900303030303030A0
:100E700030302D303030302D303030302D3030307B
:100E8000302D3030303030303030303030300020A5
:100E9000555549443A00310020455854525544456F
:100EA000525F434F554E543A00507275736120693A
:100EB00033204D4B3300204D414348494E455F544C
:100EC0005950453A00312E3000206261736564202C
:100ED0006F6E204D61726C696E204649524D5741CC
:100EE00052455F55524C3A68747470733A2F2F67AD
:100EF00069746875622E636F6D2F707275736133DC
:100F0000642F50727573612D4669726D77617265D9
:100F10002050524F544F434F4C5F56455253494F08
:100F20004E3A004649524D574152455F4E414D455C
:100F30003A50727573612D4669726D7761726520E2
:100F4000004D31313320530020423A0020453A0011
:100F5000543A0020413A0020503A002042403A00E2
:100F600020403A00202F003A00205400202F00207B
:100F7000423A00202F006F6B20543A002569206D03
:100F8000696E2C2025692073656300496E76616C5B
:100F90006964204D20636F64653A202573200A0040
:100FA000556E6B6E6F776E204720636F64653A20D5
:100FB0002573200A004D65736820626564206C65A6
:100FC00076656C696E67206E6F74206163746976F4
:100FD000652E000A002020000A4D65617375726558
:100FE0006420706F696E74733A000A5A20736561E9
:100FF000726368206865696768743A20002C004E47
:10100000756D20582C593A2000206D6963726F6EFF
:101010007300457863657373697665206265642043
:101020006C6576656C696E6720636F727265637458
:10103000696F6E3A20004732382057300050494ED1
:1010400044412070726F62652063616C69627261F5
:1010500074696F6E20737461727400473238205760
:1010600030004D3234005345545F43484F505F00C9
:101070005345545F535445505F005345545F5741A7
:1010800056455F00544D435F0043524153485F0053
:101090005072657373206B6E6F6220746F20707274
:1010A0006568656174206E6F7A7A6C6520616E6424
:1010B00020636F6E74696E75652E00506C65617388
:1010C0006520707265737320746865206B6E6F6243
:1010D00020746F20756E6C6F61642066696C616D41
:1010E000656E740052656D6F7665206F6C64206666
:1010F000696C616D656E7420616E642070726573D9
:101100007320746865206B6E6F6220746F20737437
:10111000617274206C6F6164696E67206E65772000
:1011200066696C616D656E742E00616E642070720C
:1011300065737320746865206B6E6F6200496E730F
:101140006572742066696C616D656E7400436F6CC6
:101150006F72206E6F7420636F72726563740046E5
:10116000696C616D656E74206E6F74206C6F616464
:101170006564004368616E67656420636F727265C1
:1011800063746C793F004C6F6164696E6720636FB4
:101190006C6F72004368616E676520737563636589
:1011A00073732100506C65617365206F70656E20EC
:1011B00069646C657220616E642072656D6F76651E
:1011C0002066696C616D656E74206D616E75616C11
:1011D0006C792E005761732066696C616D656E7461
:1011E00020756E6C6F6164207375636365737366DD
:1011F000756C3F00506C6561736520757067726136
:1012000064652E004E6577206669726D7761726540
:101210002076657273696F6E20617661696C6162B8
:101220006C653A0057616974696E6720666F722059
:1012300050494E44412070726F626520636F6F6C3D
:10124000696E6700437261736820646574656374D6
:1012500065642E20526573756D65207072696E74B9
:101260003F004372617368206465746563746564EC
:101270002E0045787472756465720043686F6F73F1
:10128000652065787472756465723A0043686F6FA3
:1012900073652066696C616D656E743A004E6F20EF
:1012A0006D6F76652E005761697420666F722075C8
:1012B0007365722E2E2E00536F6D652070726F62F3
:1012C0006C656D20656E636F756E74657265642CF8
:1012D000205A2D6C6576656C696E6720656E666F49
:1012E00072636564202E2E2E00537461626C65203B
:1012F000616D6269656E742074656D70657261748C
:101300007572652032312D323643206973206E6547
:101310006564656420612072696769642073746123
:101320006E642069732072657175697265642E0040
:10133000506C656173652072756E2058595A206330
:10134000616C6962726174696F6E20666972737430
:101350002E0073746172740A006164635F696E6960
:10136000740A001B5B324A1B5B313B31484F726988
:1013700067696E616C2050727573612069331B5B05
:10138000323B3348507275736120526573656172E8
:10139000636800466163746F727920524553455407
:1013A000004A616E203137203230313900436F6D91
:1013B00070696C65643A2000286E6F6E652C20643D
:1013C000656661756C7420636F6E66696729004A93
:1013D000616E20313720323031392032333A3433A4
:1013E0003A33360020332E352E312D313737380A37
:1013F000002055706C6F616420696E2070726F6799
:101400007265737300205A3A0020593A0020583A06
:101410000043524153485F44455445435445445862
:10142000590043524153485F444554454354454451
:10143000590043524153485F444554454354454441
:1014400058004D3239005072757361206933204D58
:101450004B332072656164792E00426C61636B6F5F
:101460007574206F636375727265642E20526563B4
:101470006F766572207072696E743F0053656C669A
:10148000746573742077696C6C2062652072756E68
:1014900020746F2063616C6962726174652061639E
:1014A0006375726174652073656E736F726C6573BA
:1014B00073207265686F6D696E672E00546865727F
:1014C00065206973207374696C6C2061206E65659A
:1014D0006420746F206D616B65205A2063616C69B4
:1014E00062726174696F6E2E20506C656173652045
:1014F000666F6C6C6F7720746865206D616E7561C6
:101500006C2C206368617074657220466972737414
:101510002073746570732C2073656374696F6E201B
:1015200043616C6962726174696F6E20666C6F777B
:101530002E005072696E74657220686173206E6F40
:1015400074206265656E2063616C696272617465A6
:1015500064207965742E20506C6561736520666F18
:101560006C6C6F7720746865206D616E75616C2C92
:1015700020636861707465722046697273742073A9
:10158000746570732C2073656374696F6E2043619A
:101590006C6962726174696F6E20666C6F772E0081
:1015A0004F6C642073657474696E677320666F7521
:1015B0006E642E2044656661756C74205049442C1D
:1015C00020457374657073206574632E2077696C91
:1015D0006C206265207365742E005761726E696EAF
:1015E000673A20626F7468207072696E7465722049
:1015F0007479706520616E64206D6F7468657262C5
:101600006F6172642074797065206368616E6765CC
:10161000642E005761726E696E673A207072696E4F
:101620007465722074797065206368616E676564A3
:101630002E005761726E696E673A206D6F7468652F
:1016400072626F6172642074797065206368616E84
:101650006765642E0045787465726E616C20535026
:101660004920666C61736820573235583230434CDC
:10167000206E6F7420726573706F6E64696E672E72
:101680000043726173684465746563742044495310
:1016900041424C454400437261736844657465631C
:1016A0007420454E41424C454421002020506C613D
:1016B0006E6E657242756666657242797465733ADC
:1016C00020002046726565204D656D6F72793A2065
:1016D00000207C20417574686F723A2000204C61B4
:1016E000737420557064617465643A200020536FF0
:1016F0006674776172652052657365740020576166
:10170000746368646F672052657365740020427269
:101710006F776E206F757420526573657400204575
:10172000787465726E616C20526573657400506FD9
:101730007765725570006572726F72207772697486
:10174000696E6720746F2066696C6500656E6473EE
:10175000746F7073206869743A2000446F6E65205E
:10176000736176696E672066696C652E006F6B0029
:1017700058595A2063616C6962726174696F6E2096
:10178000616C6C2072696768742E20536B657720DA
:1017900077696C6C20626520636F72726563746533
:1017A00064206175746F6D61746963616C6C792E0E
:1017B0000058595A2063616C6962726174696F6E76
:1017C00020616C6C2072696768742E20582F592034
:1017D000617865732061726520736C696768746CE9
:1017E0007920736B657765642E20476F6F64206A7C
:1017F0006F62210058595A2063616C69627261748A
:10180000696F6E206F6B2E20582F59206178657399
:10181000206172652070657270656E646963756CB5
:1018200061722E20436F6E67726174756C617469AA
:101830006F6E73210058595A2063616C696272613E
:1018400074696F6E206661696C65642E20526967E9
:1018500068742066726F6E742063616C6962726175
:1018600074696F6E20706F696E74206E6F74207271
:101870006561636861626C652E0058595A20636126
:101880006C6962726174696F6E206661696C65640F
:101890002E2046726F6E742063616C69627261748F
:1018A000696F6E20706F696E7473206E6F74207232
:1018B0006561636861626C652E0058595A206361E6
:1018C0006C6962726174696F6E206661696C6564CF
:1018D0002E20506C6561736520636F6E73756C7438
:1018E00020746865206D616E75616C2E0058595AC0
:1018F0002063616C6962726174696F6E20636F6DE1
:1019000070726F6D697365642E2052696768742008
:1019100066726F6E742063616C6962726174696F64
:101920006E20706F696E74206E6F742072656163D3
:101930006861626C652E0058595A2063616C696257
:10194000726174696F6E20636F6D70726F6D697311
:1019500065642E2046726F6E742063616C696272DA
:101960006174696F6E20706F696E7473206E6F742E
:1019700020726561636861626C652E0058595A2057
:1019800063616C6962726174696F6E206661696C13
:1019900065642E204265642063616C6962726174C3
:1019A000696F6E20706F696E7420776173206E6F3F
:1019B0007420666F756E642E00506C6561736520CF
:1019C000706C61636520737465656C207368656510
:1019D00074206F6E20686561746265642E004469CE
:1019E0007374616E6365206265747765656E2074DB
:1019F0006970206F6620746865206E6F7A7A6C65F6
:101A000020616E642074686520626564207375725D
:101A10006661636520686173206E6F74206265651E
:101A20006E20736574207965742E20506C65617327
:101A30006520666F6C6C6F7720746865206D616ED1
:101A400075616C2C206368617074657220466972E0
:101A500073742073746570732C2073656374696F7D
:101A60006E204669727374206C61796572206361BF
:101A70006C6962726174696F6E2E00506C6163658F
:101A80002061207368656574206F662070617065E1
:101A90007220756E64657220746865206E6F7A7A44
:101AA0006C6520647572696E672074686520636177
:101AB0006C6962726174696F6E206F66206669720C
:101AC0007374203420706F696E74732E2049662001
:101AD000746865206E6F7A7A6C65206361746368E0
:101AE0006573207468652070617065722C20706F5A
:101AF000776572206F666620746865207072696E03
:101B000074657220696D6D6564696174656C792EA8
:101B100000506C656173652072656D6F766520732A
:101B20007465656C2073686565742066726F6D20DE
:101B3000686561746265642E00497320737465651D
:101B40006C207368656574206F6E206865617462CF
:101B500065643F00206F66203400536561726368DE
:101B6000696E67206265642063616C69627261748A
:101B7000696F6E20706F696E7400206F6620390087
:101B80004D6561737572696E672072656665726511
:101B90006E636520686569676874206F662063619D
:101BA0006C6962726174696F6E20706F696E740027
:101BB000506C6561736520636C65616E2074686547
:101BC000206E6F7A7A6C6520666F722063616C6933
:101BD00062726174696F6E2E20436C69636B20774B
:101BE00068656E20646F6E652E004175746F2068A5
:101BF0006F6D650078797A63616C5F6D6561737391
:101C00007572655F656E7465720A0078797A6361D2
:101C10006C5F73706972616C382063783D25642055
:101C200063793D2564207A303D256420647A3D2522
:101C300064207261646975733D25642061643D258B
:101C4000640A0078797A63616C5F736561726368B6
:101C50005A206E6F207369676E616C0A20783D258B
:101C60006C6420793D256C64207A3D256C640A0003
:101C7000204F4E2D5349474E414C20617420783DF2
:101C8000256420793D2564207A3D25642061643DEA
:101C900025640A0078797A63616C5F7365617263A9
:101CA000685A20783D256C6420793D256C64207A43
:101CB0003D256C640A000A00253032780078797A74
:101CC00063616C5F7363616E5F706978656C735F8D
:101CD00033327833322063783D25642063793D25A3
:101CE00064206D696E5F7A3D2564206D61785F7A4E
:101CF0003D25640A00202532642025640A000A007C
:101D00002530327800206D696E3D2564206D617844
:101D10003D2564206469663D25640A006D61785F35
:101D2000633D253264206D61785F6C3D25640A0057
:101D30006D61785F633D2564206D61785F723D253C
:101D400064206D61785F6D617463683D25640A008D
:101D500020783D256420793D2564207A3D25640A5C
:101D600000207061747465726E20666F756E6420F9
:101D700061742025642025640A000000F000F80149
:101D8000FC03FE07FE07FE07FE07FC03F801F00058
:101D9000000073697A656F6628746F74616C293D01
:101DA00025640A0073697A656F6628626C6F636BDD
:101DB0005F627566666572293D25640A0078797AE6
:101DC00063616C5F6D656173737572655F6C65618E
:101DD00076650A00706F696E743D256420783D2534
:101DE0006420793D2564207A3D25640A0058025814
:101DF00002584D584DB004F055F055B00478797A3A
:101E000063616C5F66696E645F6265645F696E647E
:101E1000756374696F6E5F73656E736F725F706FF9
:101E2000696E745F787920783D256C6420793D2552
:101E30006C64207A3D256C640A00203C20005741E8
:101E4000524E494E473A2046726F6E7420706F6949
:101E50006E74206E6F7420726561636861626C6578
:101E60002E205920636F6F7264696E6174653A0049
:101E700000000040410000C04000005C430000C082
:101E80004000005C43000046430000404100004623
:101E900043497465726174696F6E3A200043616CE6
:101EA0006962726174696F6E206661696C65642134
:101EB00020436865636B20746865206178657320D2
:101EC000616E642072756E20616761696E2E0025F7
:101ED0006920686F757273202569206D696E75744D
:101EE00065730054494D454F55543A004D313130DA
:101EF0000046756C6C20525820427566666572000B
:101F00006673656E736F725F73746F705F616E641A
:101F10005F736176655F7072696E740A00667365DF
:101F20006E736F725F726573746F72655F707269E2
:101F30006E745F616E645F636F6E74696E75650A5F
:101F40000044495341424C45440A00454E41424CED
:101F50004544004653656E736F722025530A005046
:101F60004154393132355F696E69743A2568687554
:101F70000A00504154393132355F696E69743A252F
:101F80006868750A0050415439313235206E6F74DB
:101F900020726573706F6E64696E672028256429EE
:101FA000210A00446F6E65207072696E74696E67F5
:101FB0002066696C65005072696E74657220737476
:101FC0006F707065642064756520746F206572722F
:101FD0006F72732E2046697820746865206572726E
:101FE0006F7220616E6420757365204D3939392018
:101FF000746F20726573746172742E202854656D3D
:10200000706572617475726520697320726573659D
:10201000742E205365742069742061667465722083
:1020200072657374617274696E6729004E6F204C1B
:10203000696E65204E756D626572207769746820DF
:10204000636865636B73756D2C204C617374204CF1
:10205000696E653A20004E6F20436865636B737547
:102060006D2077697468206C696E65206E756D628D
:1020700065722C204C617374204C696E653A2000A7
:10208000636865636B73756D206D69736D617463EF
:10209000682C204C617374204C696E653A20004CAA
:1020A000696E65204E756D626572206973206E6F72
:1020B00074204C617374204C696E65204E756D629E
:1020C00065722B312C204C617374204C696E653A1B
:1020D00020006673656E736F725F6175746F6C6FED
:1020E00061645F636865636B5F7374617274202DF4
:1020F000206175746F6C6F616420454E41424C45A0
:10210000440A006673656E736F725F6175746F6CFD
:102110006F61645F636865636B5F73746F70202DBC
:10212000206175746F6C6F61642044495341424C67
:1021300045440A0053544F505045442E20006F6BC5
:102140000A0073746172740A004D4D55322066693D
:10215000726D776172652076657273696F6E206942
:102160006E76616C69642E20526571756972656462
:102170002076657273696F6E3A206275696C6420AF
:102180006E756D626572202564206F7220686967C4
:102190006865722E004D4D55203D3E20276F6B2700
:1021A0000A002564004D4D552072657472792061D6
:1021B0007474656D7074206E722E2025640A004D53
:1021C0004D55203D3E20276F6B270A00410A004DE8
:1021D0004D55203C3D202741270A004D3630300028
:1021E0004D363030204155544F004653454E534FE5
:1021F000525F5245434F564552002568687500505E
:10220000300A0053330A004D4D55203C3D202753E2
:1022100033270A0052300A004D4D55203C3D2027FF
:102220005230270A004525640A004D4D55203C3D9B
:102230002027452564270A0055300A004D4D5520BA
:102240003C3D20275530270A0043300A004D4D55AC
:10225000203C3D20274330270A004C25640A004DCE
:102260004D55203C3D20274C2564270A0054256409
:102270000A004D4D55203C3D2027542564270A0077
:102280004D4D55202D20454E41424C45440025687A
:1022900068750050300A0050300A004D4D552076C8
:1022A000657273696F6E2076616C6964004D4D557F
:1022B000203D3E202725646F6B270A0025750053BB
:1022C000320A004D4D55203C3D2027533227004D0A
:1022D0004D55203D3E202725646F6B270A0025754C
:1022E000004D4D55206E6F7420726573706F6E6473
:1022F000696E67202D2044495341424C45440053A8
:10230000310A004D4D55203C3D2027533127004DCB
:102310004D55203D3E2027737461727427006D6D0A
:10232000755F6765745F726573706F6E736528297A
:102330002072657475726E696E673A2025640A00B2
:10234000556E6C6F6164696E672066696E6973684B
:10235000656420320A00556E6C6F616420320A0099
:10236000556E6C6F6164696E672066696E6973682B
:10237000656420310A00556E6C6F616420310A007B
:102380006D6D755F6765745F726573706F6E736591
:10239000202D20626567696E206D6F76653A256431
:1023A0000A004D4D55207374617274732072657309
:1023B000706F6E64696E670A004D4D55206E6F74C4
:1023C00020726573706F6E64696E670A000000802A
:1023D0003F555585410000803F0000C84100000086
:1023E00040555505420000C03F0000484200002013
:1023F0004055558542000070C1ABAAA6420000605E
:10240000C10000A0410000C0C00000204100002029
:1024100041ABAA3A41000020C15555D540000048C3
:10242000C2555505424D373031204530004D3730CB
:1024300031204531004D373031204532004D3730A5
:1024400031204533004D373031204534004D373091
:1024500031204534004D373031204533004D373081
:1024600031204532004D373031204531004D373075
:10247000312045300046696C616D656E74206E7266
:10248000206F7574206F662072616E676521004150
:1024900064646974696F6E616C206C6F6164206143
:1024A0007474656D7074206E722E2025640A00505D
:1024B0006C6561736520757064617465206669720E
:1024C0006D7761726520696E20796F7572204D4D50
:1024D00055322E2057616974696E6720666F7220CD
:1024E00072657365742E004D4D55204F4B2E205252
:1024F0006573756D696E672E2E2E004D4D55204FFC
:102500004B2E20526573756D696E6720706F73690D
:1025100074696F6E2E2E2E004D4D55204F4B2E2080
:10252000526573756D696E672074656D7065726153
:10253000747572652E2E2E004669782074686520A9
:10254000697373756520616E64207468656E2070B0
:102550007265737320627574746F6E206F6E204D98
:102560004D5520756E69742E00507265737320741A
:102570006865206B6E6F6220746F20726573756D75
:1025800065206E6F7A7A6C652074656D7065726116
:10259000747572652E004D4D55206E65656473200F
:1025A0007573657220617474656E74696F6E2E0048
:1025B000506C656173652072656D6F766520666924
:1025C0006C616D656E7420616E64207468656E2048
:1025D000707265737320746865206B6E6F622E0075
:1025E000456A656374696E672066696C616D656EC6
:1025F00074004D4D55206C6F6164206661696C6597
:102600006420202020200025632533642F256425A5
:102610006300473830004D3435004D3435205A00C2
:102620004737360057697A61726420737461746544
:102630003A2025640044697361626C6520666172AA
:102640006D206D6F6465004661726D206E756D6200
:102650006572004D3834004D34340047323820570D
:10266000004739390044697361626C6520666172A4
:102670006D206D6F64653F0043616C6962726174C7
:102680006500506C65617365206C6F616420504C0F
:10269000412066696C616D656E7420666972737441
:1026A0002E00497320504C412066696C616D656E47
:1026B00074206C6F616465643F0043616E63656C98
:1026C0000046696C616D656E740053656C6563747A
:1026D00020504C412066696C616D656E743A005201
:1026E000756E6E696E672057697A617264207769CA
:1026F0006C6C2064656C6574652063757272656EC0
:10270000742063616C6962726174696F6E207265B6
:1027100073756C747320616E6420737461727420BD
:1027200066726F6D2074686520626567696E6E6998
:102730006E672E20436F6E74696E75653F00507230
:102740006568656174696E67206E6F7A7A6C652E54
:1027500020506C6561736520776169742E00456A4D
:1027600065637400556E6C6F616400557365207508
:102770006E6C6F616420746F2072656D6F7665207A
:1027800066696C616D656E742031206966206974BC
:102790002070726F747275646573206F75747369DD
:1027A0006465206F66207468652072656172204DD3
:1027B0004D5520747562652E2055736520656A65D8
:1027C0006374206966206974206973206869646491
:1027D000656E20696E20747562652E004C6F6164B1
:1027E000696E672066696C616D656E7400506C651A
:1027F00061736520696E7365727420504C41206668
:10280000696C616D656E7420746F207468652065F5
:10281000787472756465722C207468656E207072AD
:10282000657373206B6E6F6220746F206C6F6164D0
:102830002069742E00506C6561736520696E736544
:10284000727420504C412066696C616D656E742015
:10285000746F207468652066697273742074756281
:1028600065206F66204D4D552C207468656E207074
:102870007265737320746865206B6E6F6220746F6D
:10288000206C6F61642069742E00596F752063613C
:102890006E20616C7761797320726573756D652048
:1028A0007468652057697A6172642066726F6D2062
:1028B00043616C6962726174696F6E202D3E2057AE
:1028C000697A6172642E00506C656173652063687B
:1028D00065636B206F75722068616E64626F6F6BE9
:1028E00020616E6420666978207468652070726F5C
:1028F000626C656D2E205468656E20726573756D0F
:1029000065207468652057697A6172642062792055
:102910007265626F6F74696E67207468652070728B
:10292000696E7465722E00416C6C20697320646F4F
:102930006E652E204861707079207072696E7469BE
:102940006E672100506C6561736520636C65616E14
:10295000206865617462656420616E6420746865D6
:102960006E20707265737320746865206B6E6F6281
:102970002E00446F20796F752077616E7420746F1C
:1029800020726570656174206C6173742073746566
:102990007020746F20726561646A75737420646955
:1029A0007374616E6365206265747765656E206E11
:1029B0006F7A7A6C6520616E642068656174626507
:1029C000643F00492077696C6C20737461727420D5
:1029D000746F207072696E74206C696E6520616E10
:1029E0006420796F752077696C6C206772616475FB
:1029F000616C6C79206C6F77657220746865206EED
:102A00006F7A7A6C6520627920726F746174696E76
:102A10006720746865206B6E6F622C20756E746918
:102A20006C20796F75207265616368206F707469BE
:102A30006D616C206865696768742E204368656302
:102A40006B207468652070696374757265732069A2
:102A50006E206F75722068616E64626F6F6B2069A3
:102A60006E20636861707465722043616C69627284
:102A70006174696F6E2E004E6F7720492077696C04
:102A80006C2063616C69627261746520646973743F
:102A9000616E6365206265747765656E2074697028
:102AA000206F6620746865206E6F7A7A6C6520618D
:102AB0006E64206865617462656420737572666116
:102AC00063652E00497320697420504C412066696B
:102AD0006C616D656E743F0053656C656374206E48
:102AE0006F7A7A6C652070726568656174207465B0
:102AF0006D706572617475726520776869636820AE
:102B00006D61746368657320796F7572206D61748F
:102B1000657269616C2E004E6F7720492077696C71
:102B20006C2070726568656174206E6F7A7A6C656E
:102B300020666F7220504C412E0049732066696CEC
:102B4000616D656E74206C6F616465643F004973EC
:102B50002066696C616D656E742031206C6F6164F4
:102B600065643F004E6F7720492077696C6C207058
:102B7000726568656174206E6F7A7A6C6520666F25
:102B80007220504C412E00492077696C6C20727580
:102B90006E207A2063616C6962726174696F6E2065
:102BA0006E6F772E004E6F772072656D6F766520A1
:102BB0007468652074657374207072696E74206621
:102BC000726F6D20737465656C2073686565742E13
:102BD00000506C656173652072656D6F766520735A
:102BE00068697070696E672068656C7065727320C3
:102BF00066697273742E00492077696C6C20727557
:102C00006E2078797A2063616C6962726174696F91
:102C10006E206E6F772E2049742077696C6C20745B
:102C2000616B6520617070726F782E203132206D7B
:102C3000696E732E0046697273742C20492077697F
:102C40006C6C2072756E207468652073656C667498
:102C500065737420746F20636865636B206D6F7398
:102C60007420636F6D6D6F6E20617373656D626C40
:102C7000792070726F626C656D732E0048692C202C
:102C80004920616D20796F7572204F726967696E96
:102C9000616C205072757361206933207072696EA7
:102CA0007465722E20576F756C6420796F75206C77
:102CB000696B65206D6520746F2067756964652098
:102CC000796F75207468726F756768207468652005
:102CD00073657475702070726F636573733F004520
:102CE0002D636F7272656374005A2D636F72726523
:102CF000637400592D636F727265637400582D639D
:102D00006F72726563740053706F6F6C4A6F696E97
:102D10002020205B4E2F415D0053706F6F6C4A6F17
:102D2000696E2020205B6F66665D0053706F6F6C6C
:102D30004A6F696E202020205B6F6E5D00536F75B7
:102D40006E642020202020205B6C6F75645D005332
:102D50006F756E642020202020205B6D7574655D8A
:102D600000536F756E64202020205B73696C656E64
:102D7000745D00536F756E642020202020205B6FEF
:102D80006E63655D00536F756E64202020202020E7
:102D90005B6C6F75645D00536F72743A2020202065
:102DA00020205B6E6F6E655D00536F72743A202059
:102DB0005B616C7068616265745D00536F72743A38
:102DC0002020202020205B74696D655D0053442025
:102DD0006361726420205B6E6F726D616C5D005385
:102DE000442063617264205B666C73684169725D44
:102DF0000052506920706F727420202020205B6F79
:102E00006E5D0052506920706F7274202020205B2C
:102E10006F66665D0054656D702E2063616C2E20B8
:102E200020205B6F6E5D0054656D702E2063616CB9
:102E30002E20205B6F66665D004C696E2E20636FEE
:102E40007272656374696F6E0046616E73206368A9
:102E500065636B20205B6F66665D0046616E732064
:102E6000636865636B2020205B6F6E5D00462E20DB
:102E70006175746F6C6F6164205B6F66665D0046A0
:102E80002E206175746F6C6F616420205B6F6E5DC6
:102E900000462E206175746F6C6F6164205B4E2F4D
:102EA000415D0046696C2E2073656E736F72205B06
:102EB0004E2F415D0044697361626C6520737465D7
:102EC0007070657273004D6F76652061786973006C
:102ED00054656D70657261747572650054656D70CE
:102EE0002E2063616C6962726174696F6E00526555
:102EF0007365742058595A2063616C6962722E00A0
:102F00005049442063616C6962726174696F6E003C
:102F1000426564206C6576656C20636F72726563D0
:102F200074004D65736820426564204C6576656C5D
:102F3000696E670043616C696272617465205A0052
:102F400043616C6962726174652058595A00536517
:102F50006C667465737420202020202020202000BF
:102F60004669727374206C617965722063616C2E9E
:102F70000057697A617264004C6F61642066696C05
:102F8000616D656E742035004C6F61642066696CFC
:102F9000616D656E742034004C6F61642066696CED
:102FA000616D656E742033004C6F61642066696CDE
:102FB000616D656E742032004C6F61642066696CCF
:102FC000616D656E742031004C6F616420616C6CC2
:102FD000004C6F61642066696C616D656E742035AC
:102FE000004C6F61642066696C616D656E7420349D
:102FF000004C6F61642066696C616D656E7420338E
:10300000004C6F61642066696C616D656E7420327E
:10301000004C6F61642066696C616D656E7420316F
:1030200000456A6563742066696C616D656E742025
:103030003500456A6563742066696C616D656E7400
:10304000203400456A6563742066696C616D656E45
:1030500074203300456A6563742066696C616D6530
:103060006E74203200456A6563742066696C616D18
:10307000656E74203100506C656173652070756CED
:103080006C206F75742066696C616D656E74206963
:103090006D6D6564696174656C7900556E6C6F6106
:1030A00064696E672066696C616D656E740057694E
:1030B0007A61726420656E642073746174653A206D
:1030C00025640A0024F4D43050C38E20C2A24017D5
:1030D000828B7011127A910D816CD90AA861E10876
:1030E000C7586607615143061E4B5D05C145A704DD
:1030F0001A411104093D9803713931034036DB024E
:1031000065339102D4305402802E1D02632CEE01EF
:10311000752AC501B028A001102781018F256401FF
:103120002B244B01E0223401AC211F018D200D0125
:10313000801FFC00841EED00971DDF00B81CD2002C
:10314000E61BC600201BBC00641AB200B219A8001E
:103150000A19A0006A189900D117910040178B0036
:10316000B516840031167E00B31579003A15730048
:10317000C7146F0058146A00EE13660088136300CA
:1031800025135E00C7125B006C1257001512540025
:10319000C111510070114F0021114B00D610490090
:1031A0008D1047004610440002104200C00F40003E
:1031B000800F3E00420F3C00060F3B00CB0E380054
:1031C000930E37005C0E3500270E3400F30D3200ED
:1031D000C10D3100900D3000600D2E00320D2D001C
:1031E000050D2C00D90C2B00AE0C2900850C2900F4
:1031F0005C0C2700350C27000E0C2600E80B240081
:10320000C40B2400A00B23007D0B23005A0B2100CC
:10321000390B2100180B2000F80A1F00D90A1E00E4
:10322000BB0A1E009D0A1D00800A1D00630A1C00C7
:10323000470A1B002C0A1B00110A1A00F7091A0082
:10324000DD091900C4091900AB091900920917001A
:103250007B091800630917004C091600360916008F
:10326000200916000A091500F5081500E0081400E9
:10327000CC081400B8081400A40814009008130027
:103280007D0812006B08130058081200460812004F
:103290003408110023081100120811000108110060
:1032A000F0071000E0071000D0071000C007100062
:1032B000B0070F00A107100091070E0083070F0051
:1032C00074070F0065070E0057070E0049070E0030
:1032D0003B070D002E070E0020070D0013070D0001
:1032E00006070D00F9060C00ED060D00E0060C00C7
:1032F000D4060C00C8060C00BC060C00B0060C007E
:10330000A4060B0099060C008D060B0082060B002C
:1033100077060B006C060B0061060A0057060B00CF
:103320004C060A0042060A0038060A002E060A0069
:1033300024060A001A060A001006090007060A00F9
:10334000FD050900F4050900EB050900E205090087
:10335000D9050900D0050900C7050900BE05090007
:10336000B5050800AD050800A50509009C05080085
:10337000940508008C050800840508007C050800F9
:10338000740508006C050700650508005D05070069
:10339000560508004E0507004705070040050800D0
:1033A00038050700310507002A0507002305070037
:1033B0001C050600160507000F0507000805060096
:1033C00002050700FB040600F5040700EE040600F2
:1033D000E8040600E2040700DB040600D50406004A
:1033E000CF040600C9040600C3040600BD0406009D
:1033F000B7040600B1040500AC040600A6040600EC
:10340000A00405009B040600950405009004060036
:103410008A04050085040500800406007A0405007E
:1034200075040500700405006B04050066040500C2
:10343000610405005C040500570405005204050002
:103440004D04050048040500430405003E04040043
:103450003A04050035040500300404002C0405007E
:1034600027040400230405001E0404001A040400B9
:1034700016040500110404000D04040009040500ED
:103480000404040000040400FC030400F803040026
:10349000F4030400F0030400EC030400E803040058
:1034A000E4030400E0030400DC030400D803040088
:1034B000D4030400D0030400CC030400C8030300B9
:1034C000C503030024F404D9201BC40C5C0E98042B
:1034D000C4095F0265077101F405F900FB04B3003C
:1034E00048048700C10369005803550003034500E1
:1034F000BE023A008402310053022A00290225004C
:1035000004022000E4011C00C8011900AF011700EB
:103510009801140084011300710110006101100072
:1035200051010E0043010D0036010B002B010B0071
:1035300020010B00150109000C010900030108001E
:10354000FB000800F3000800EB000700E4000600A1
:10355000DE000600D8000600D2000600CC00050000
:10356000C7000500C2000500BD000400B90004004A
:10357000B5000400B1000400AD000400A90004007F
:10358000A5000300A20003009F0004009B000300AD
:1035900098000300950002009300030090000300D0
:1035A0008D0002008B0003008800020086000200EC
:1035B00084000300810002007F0002007D00020001
:1035C0007B00020079000200770001007600020013
:1035D0007400020072000100710002006F0002001E
:1035E0006D0001006C0002006A0001006900020029
:1035F0006700010066000100650001006400020030
:103600006200010061000100600001005F00020033
:103610005D0001005C0001005B0001005A00010038
:103620005900010058000100570001005600010038
:103630005500010054000100530000005300010038
:103640005200010051000100500001004F00010034
:103650004E0000004E0001004D0001004C00010032
:103660004B0000004B0001004A000100490001002E
:10367000480000004800010047000100460000002B
:103680004600010045000000450001004400010023
:10369000430000004300010042000000420001001E
:1036A0004100000041000100400001003F00000017
:1036B0003F0001003E0000003E0001003D00000010
:1036C0003D0001003C0000003C0000003C00010007
:1036D0003B0000003B0001003A0000003A000100FE
:1036E00039000000390001003800000038000000F7
:1036F00038000100370000003700010036000000EC
:1037000036000000360001003500000035000000E2
:1037100035000100340000003400000034000100D6
:1037200033000000330000003300010032000000CD
:1037300032000000320001003100000031000000C2
:1037400031000100300000003000000030000100B6
:103750002F0000002F0000002F0000002F000100AC
:103760002E0000002E0000002E0001002D000000A1
:103770002D0000002D0000002D0001002C00000095
:103780002C0000002C0000002C0001002B00000089
:103790002B0000002B0000002B0001002A0000007D
:1037A0002A0000002A0000002A0001002900000071
:1037B0002900000029000000290000002900010064
:1037C0002800000028000000280000002800000059
:1037D000280001002700000027000000270000004B
:1037E000270000002700010026000000260000003E
:1037F0002600000026000000260001002500000031
:103800002500000025000000250000002500000024
:103810002500010024000000240000002400000016
:103820002400000024000100230000002300000009
:1038300023000000230000002300000023000000FC
:1038400023000100220000002200000022000000EE
:1038500022000000220000002200010021000000E0
:1038600021000000210000002100000021000000D4
:1038700021000000210001002000000020000000C5
:1038800020000000200000002000000020000000B8
:1038900020000000200001001F0000001F000000A9
:1038A0001F0000001F0000001F0000001F0000009C
:1038B0001F0001001E0000001E0000001E0000008E
:1038C0001E00000043686F6F736520636F6C6F723A
:1038D0003A004D3730322043004661726D206E75DC
:1038E0006D626572004D363030004D3234004D321D
:1038F0003320257300052E2E00526573756D696E99
:1039000067207072696E7400537570706F72740006
:103910004661696C207374617473204D4D55004687
:1039200061696C207374617473005374617469739A
:103930007469637320200043616C69627261746909
:103940006F6E004175746F4C6F61642066696C61C5
:103950006D656E7400556E6C6F61642066696C6194
:103960006D656E7400456A6563742066696C616D8F
:10397000656E74004C6F616420746F206E6F7A7A8C
:103980006C65004C6F61642066696C616D656E7476
:10399000004E6F2053442063617264005072696E60
:1039A000742066726F6D20534400526573756D65A7
:1039B000207072696E740050617573652070726951
:1039C0006E7400507265686561740054756E6500B0
:1039D0004C6976652061646A757374205A00496E7B
:1039E000666F2073637265656E0046696E69736801
:1039F000696E67206D6F76656D656E747300536FC9
:103A0000756E642020202020205B6C6F75645D0043
:103A1000536F756E642020202020205B6D757465C7
:103A20005D00536F756E64202020205B73696C65A8
:103A30006E745D00536F756E642020202020205B23
:103A40006F6E63655D00536F756E642020202020CB
:103A5000205B6C6F75645D00437261736820646500
:103A6000742E20205B4E2F415D00437261736820ED
:103A70006465742E2020205B6F6E5D00437261735D
:103A800068206465742E20205B6F66665D004D6F54
:103A90006465202020205B537465616C74685D0050
:103AA0004D6F646520202020205B4E6F726D616C2D
:103AB0005D0046696C2E2073656E736F7220205B0B
:103AC0006F6E5D0046696C2E2073656E736F722099
:103AD0005B6F66665D004368616E67652066696C52
:103AE000616D656E7400466C6F7700537065656438
:103AF0000046616E20737065656400426564004E27
:103B00006F7A7A6C650053657474696E67730050E0
:103B100072696E742061626F7274656400596573B6
:103B2000004E6F0053746F70207072696E7400469F
:103B3000696C6520696E636F6D706C6574652E20AD
:103B4000436F6E74696E756520616E797761793F38
:103B5000004D61696E00416D6269656E7400426579
:103B600064004E6F7A7A6C650042656C74207374E1
:103B70006174757300436F6F6C646F776E00566F7E
:103B80006C74616765730054656D706572617475FE
:103B90007265730042656C74207374617475730090
:103BA00053686F772073656E736F72730045787416
:103BB000727564657220696E666F0058595A206389
:103BC000616C2E2064657461696C7300756E6B6E38
:103BD0006F776E004D4D553220636F6E6E65637466
:103BE000656400446174653A00686F77746F2E7085
:103BF0007275736133642E636F6D00666F72756DDD
:103C00002E707275736133642E636F6D0070727500
:103C1000736133642E636F6D0046696C616D656E10
:103C20007420657874727564696E672026207769E0
:103C3000746820636F727265637420636F6C6F7257
:103C40003F005072656865617420746865206E6F0E
:103C50007A7A6C6521004552524F523A0041757490
:103C60006F6C6F6164696E672066696C616D656E0B
:103C700074206973206163746976652C206A75739A
:103C80007420707265737320746865206B6E6F6248
:103C900020616E6420696E736572742066696C6160
:103CA0006D656E742E2E2E00546F74616C207072D0
:103CB000696E742074696D6500546F74616C206660
:103CC000696C616D656E74005072696E7420746900
:103CD0006D650046696C616D656E74207573656411
:103CE000005269676874004C656674005920646905
:103CF0007374616E63652066726F6D206D696E000E
:103D000053657665726520736B657700536C6967E0
:103D1000687420736B6577004D65617375726564B7
:103D200020736B6577005B303B305D20706F696E90
:103D300074206F66667365740041646A7573746994
:103D40006E67205A00526573657400526561722077
:103D500073696465205B756D5D0046726F6E7420DB
:103D6000736964655B756D5D005269676874207383
:103D70006964655B756D5D004C656674207369648C
:103D800065205B756D5D005365742074656D7065AD
:103D90007261747572653A001B5B323B3148255382
:103DA0003A2020256425631B5B333B314850494E44
:103DB00044413A2020202025642563001B5B303BD2
:103DC000314825533A202020256425631B5B313B75
:103DD000314825533A2020202020202564256300E7
:103DE0001B5B313B31485057523A20202020202085
:103DF00025642E25303164561B5B323B31484245E9
:103E0000443A20202020202025642E25303164567D
:103E1000001B5B303B314825531B5B313B3248581C
:103E20002025641B5B323B32485920256400464CF8
:103E30004558202D20203234302F3530005050206E
:103E400020202D20203235342F3130300048495089
:103E500053202D20203232302F3130300041425358
:103E600020202D20203235352F3130300050455460
:103E700020202D20203233302F383500504C412067
:103E8000202D20203231352F363000414253202062
:103E900020202D20203235352F313030006E6F7AC2
:103EA0007A6C65202D20203235302F30006661720B
:103EB0006D2020202D20203235302F363000466CEA
:103EC00061736841697220495020416464723A000C
:103ED0004D4D5532202020202020204E2F410025FE
:103EE000642E25642E25642D2564002046573A0053
:103EF0004A616E2031372032303139004533447603
:103F00003666756C6C0045494E53795F31306100FF
:103F1000315F37356D6D5F4D4B33002D2D2D2D2DC0
:103F20002D2D2D2D2D2D2D00207265706F20556E9D
:103F30006B6E6F776E0020332E352E312D31373773
:103F400038004669726D776172653A0025642E25E6
:103F5000642E25642E2564004D373032004D3730F5
:103F600031004578747275646572006D6D0000599A
:103F7000005800580059005A002563252E3132534D
:103F80003A2573252B30362E3366001B5B324A25CB
:103F900053203A1B5B313B394825382E3266206D61
:103FA0000A2553203A0A25376C6464203A25326882
:103FB000686468203A253032686864206D001B5BB5
:103FC000324A25533A1B5B313B364825382E326640
:103FD0006D200A2553203A1B5B333B384825326459
:103FE0006820253032646D20253032647300253618
:103FF0002E32666D6D004E2F41001B5B303B30480A
:1040000025533A0A25530A25533A0A25533A001BE9
:104010005B303B3135484E2F41001B5B303B313527
:104020004825342E326601001B5B303B3048255357
:104030003A0A25530A25533A202025352E326601A7
:104040000A25533A202025352E3266010020423AB7
:104050000020453A00543A00494E543400726563DA
:104060006F7665725F6D616368696E655F737461B9
:1040700074655F61667465725F706F7765725F709B
:10408000616E69632C20696E697469616C200072CD
:1040900065636F7665725F6D616368696E655F7396
:1040A000746174655F61667465725F706F77657265
:1040B0005F70616E69632C20696E697469616C2040
:1040C0000047393220450050525553412075766CD7
:1040D0006F004734205330004D32362053256C7525
:1040E000004D3130362053004D38320047312046E4
:1040F00025640047312045322A64656661756C7419
:104100005F72657472616374696F6E204634383013
:10411000004731205A00204632303030002059000C
:1041200047312058004D383300506F736974696F00
:104130006E20726561642066726F6D2065657072B5
:104140006F6D3A004D3233202573002E67636F0088
:1041500046656564726174653A00473120452D6497
:10416000656661756C745F72657472616374696FA2
:104170006E204634383000473120453520463132F4
:1041800030004D3833004D31393020532564004D17
:1041900031303920532564004732382058205900E7
:1041A0004731205A3235204638303000204600470B
:1041B00031205A0020460047312045004D38330059
:1041C000627573793A2070617573656420666F72E9
:1041D00020696E70757400627573793A207061752C
:1041E00073656420666F7220757365720062757303
:1041F000793A2070726F63657373696E67006F6BD5
:104200000A0055564C4F202D20656E642025640A07
:10421000007374707325640A00776F726C64206396
:104220006F6F7264696E617465733A2028252E334E
:10423000662C20252E33662C20252E3366290A0075
:10424000706879736963616C20636F6F7264696E03
:10425000617465733A2028252E33662C20252E3371
:10426000662C20252E3366290A0043757272656E0E
:104270007420706F73205A5F415849533A252E338A
:10428000660A43757272656E7420706F7320455FA5
:10429000415849533A252E33660A004166746572C7
:1042A0002077616974696E6720666F722074656D2E
:1042B000703A0A43757272656E7420706F7320587D
:1042C0005F415849533A252E33660A437572726529
:1042D0006E7420706F7320595F415849533A252EF0
:1042E00033660A005265636F766572696E67207087
:1042F00072696E74202020200020003E003E0020C5
:10430000003E003E0054656D7065726174757265A3
:104310002063616C6962726174696F6E20666169A5
:104320006C65642E20436F6E74696E7565207769C5
:104330007468207072657373696E67207468652095
:104340006B6E6F622E0054656D706572617475726C
:10435000652063616C6962726174696F6E20646F5D
:104360006E652E20436F6E74696E75652077697473
:1043700068207072657373696E6720746865206B5E
:104380006E6F622E0054656D706572617475726532
:104390002063616C6962726174696F6E2066616925
:1043A0006C65640054656D7065726174757265202A
:1043B00063616C6962726174696F6E2069732066F3
:1043C000696E697368656420616E642061637469F5
:1043D00076652E2054656D702E2063616C69627263
:1043E0006174696F6E2063616E2062652064697319
:1043F00061626C656420696E206D656E7520536521
:104400007474696E67732D3E54656D702E20636100
:104410006C2E004E2F41004F6666004F6E20004903
:10442000523A0046494E44413A0050494E44413ABE
:104430000053656E736F7220737461746500457804
:10444000747275646572004D6F7665205A004D6F09
:1044500076652059004D6F76652058001B5B324A07
:10446000437261736820646574656374696F6E205C
:1044700063616E1B5B313B30486265207475726E00
:104480006564206F6E206F6E6C7920696E1B5B32E5
:104490003B30484E6F726D616C206D6F6465001B20
:1044A0005B324A5741524E494E473A1B5B313B30D3
:1044B00048437261736820646574656374696F6EE4
:1044C0001B5B323B304864697361626C65642069D0
:1044D0006E1B5B333B3048537465616C7468206DB0
:1044E0006F6465004175746F6C6F6164696E6720FD
:1044F00066696C616D656E7420617661696C61627C
:104500006C65206F6E6C79207768656E2066696CCB
:10451000616D656E742073656E736F7220697320B0
:104520007475726E6564206F6E2E2E2E0045525289
:104530004F523A2046696C616D656E742073656EEA
:10454000736F72206973206E6F7420726573706F61
:104550006E64696E672C20706C656173652063689A
:1045600065636B20636F6E6E656374696F6E2E009A
:1045700000002110422063308440A550C660E770DF
:10458000088129914AA16BB18CC1ADD1CEE1EFF187
:104590003112100273325222B5529442F772D6622F
:1045A000399318837BB35AA3BDD39CC3FFF3DEE3D7
:1045B0006224433420040114E664C774A44485547F
:1045C0006AA54BB528850995EEE5CFF5ACC58DD527
:1045D0005336722611163006D776F6669556B446CF
:1045E0005BB77AA719973887DFF7FEE79DD7BCC777
:1045F000C448E5588668A77840086118022823381F
:10460000CCC9EDD98EE9AFF9488969990AA92BB9C6
:10461000F55AD44AB77A966A711A500A333A122A6E
:10462000FDDBDCCBBFFB9EEB799B588B3BBB1AAB16
:10463000A66C877CE44CC55C222C033C600C411CBE
:10464000AEED8FFDECCDCDDD2AAD0BBD688D499D66
:10465000977EB66ED55EF44E133E322E511E700E0E
:104660009FFFBEEFDDDFFCCF1BBF3AAF599F788FB6
:104670008891A981CAB1EBA10CD12DC14EF16FE196
:104680008010A100C230E3200450254046706760CE
:10469000B9839893FBA3DAB33DC31CD37FE35EF3E6
:1046A000B1029012F322D23235421452776256721E
:1046B000EAB5CBA5A89589856EF54FE52CD50DC536
:1046C000E234C324A014810466744764245405446E
:1046D000DBA7FAB79987B8975FE77EF71DC73CD786
:1046E000D326F2369106B0165766767615463456BE
:1046F0004CD96DC90EF92FE9C899E9898AB9ABA9D6
:104700004458654806782768C018E1088238A3280D
:104710007DCB5CDB3FEB1EFBF98BD89BBBAB9ABB25
:10472000754A545A376A167AF10AD01AB32A923A5D
:104730002EFD0FED6CDD4DCDAABD8BADE89DC98D75
:10474000267C076C645C454CA23C832CE01CC10CAD
:104750001FEF3EFF5DCF7CDF9BAFBABFD98FF89FC5
:10476000176E367E554E745E932EB23ED10EF01EFD
:104770007C3C3E5E2B3D3F2F5B5D3B2C2A225C0048
:1047800022206661696C65643A20427566666572CE
:104790002066756C6C21002200656E717565696E0E
:1047A00067202200544D4320445249564552204F21
:1047B00056455254454D50002533642E25303175F1
:1047C000256325642563005A2533642E2530327510
:1047D000005A2D2D2D2E2D2D0025632533642525E2
:1047E000002D2D2D002533686864002533532533B3
:1047F00073252500205344002020200055534200FB
:104800002025753E257500203F3E25750020462554
:10481000750020463F0020463020200025632D2DC6
:104820003A2D2D202000256325337568202563252A
:1048300063002563253032753A25303275256325AE
:104840006300726573756C742076616C75653A20CF
:1048500025640A0020693D25326420636E743D257D
:1048600032642076616C3D2532640A00636C757396
:10487000746572733A0A0020693D253264207374AE
:1048800065703D2532640A00736F7274656420732D
:10489000616D706C65733A0A003A20002020202078
:1048A0002020202020202020202020202020200028
:1048B000203A2000202020202020202020202020FE
:1048C0002020202020202020002020202020202008
:1048D0002020202020200025730050494E444120F4
:1048E00048656174696E670054656D702E20636160
:1048F0006C2E202020202020202020200043616CCE
:104900006962726174696F6E20646F6E65004361E5
:104910006C6962726174696E67205A004265642036
:10492000646F6E65004265642048656174696E67F6
:104930000048656174696E6720646F6E652E00487B
:10494000656174696E670043757272656E740055B7
:1049500073656420647572696E67207072696E7425
:10496000005049442063616C2E2066696E6973684B
:104970006564005049442063616C2E202020202073
:1049800020202020202000506C6561736520776115
:104990006974004D313137204669727374206C613F
:1049A0007965722063616C2E005072696E7420709C
:1049B000617573656400496E76616C696420504965
:1049C000442063616C2E20726573756C74732E20A5
:1049D0004E6F742073746F72656420746F20454548
:1049E00050524F4D2E004D353030004731205A3156
:1049F00035204631353030004739310047312058B5
:104A0000353020593139302045302046373030306C
:104A100000473930004D373032004D3730322043B7
:104A2000004D3730322055004D373032004D373091
:104A3000322043004731205A31352046313530305D
:104A4000004739310047312058353020593139304D
:104A5000204530204637303030004D38330047395C
:104A600030004D3834004D313034205330004D3853
:104A700034004D3730322043004731205831302048
:104A800059313830204634303030004731205A31E7
:104A9000302046313330302E303030004D3134301C
:104AA000205330004D313034205330004731204501
:104AB0002D302E30373530302046323130302E30E8
:104AC00030303030004D31303700473120583530EC
:104AD000205935352045332E3632373733004731AC
:104AE0002058323030205935352045302E34393376
:104AF000383600473120583230302059373520457C
:104B0000332E36323737330047312058353020596D
:104B100037352045302E3439333836004731205868
:104B20003530205939352045332E3632373733006A
:104B300047312058323030205939352045302E3415
:104B4000393338360047312058323030205931312E
:104B5000352045332E36323737330047312058352C
:104B60003020593131352045302E34393338360034
:104B700047312058353020593133352045332E36D2
:104B800032373733004731205832303020593133F3
:104B9000352045302E3636313734004731205832F3
:104BA000303020593135352045322E3632373733C3
:104BB00000473120583130302059313535204532C9
:104BC0000047312058373520593135352045322EB0
:104BD00035004731204631303830004731205A30D7
:104BE0002E3135302046373230302E3030300047CD
:104BF0003120583530205931353500473120463481
:104C0000303030004D3230342053313030300047B6
:104C100031205A352046373230302E303030004780
:104C20003120452D312E3530303030204632313074
:104C3000302E3030303030004D38330047393000BE
:104C4000473231004739322045302E30004731207D
:104C5000583130302E30204531322E35204631301B
:104C600030302E30004731205836302E3020453934
:104C70002E302046313030302E300047312058352C
:104C80002E302045342E302046313030302E30004A
:104C90004731205A302E32302046313030302E30DD
:104CA000004731205835352E3020453235204631E9
:104CB0003430302E3000473120592D322E302046EE
:104CC000313030302E3000473120583234302E30E1
:104CD000204532352E30202046323230302E300002
:104CE0004739322045302E30004731205A302E339C
:104CF0002046313030302E30004731205835352EA7
:104D0000302045382E302046323030302E300047AB
:104D1000312058352E30204533322E302046313860
:104D200030302E30004731205835352E3020453375
:104D3000322E302046313037332E30004731205A62
:104D4000302E342046313030302E3000473120595B
:104D50002D332E302046313030302E30004D383358
:104D6000004739322045302E3000473238004D316F
:104D700030392053323135004D31393020533630FF
:104D8000004D31343020533630004D313034205313
:104D9000323135004D31303700526573656E640035
:104DA00025533A20256C640A25530A002079645F54
:104DB0006D696E3D25752079645F6D61783D25755F
:104DC0002079645F6176673D25752073685F617641
:104DD000673D25750A002073745F73756D3D2575F9
:104DE0002079645F73756D3D25752065725F7375FD
:104DF0006D3D25752065725F6D61783D256868752C
:104E00000A00004B494C4C45442E20005072696EFC
:104E10007465722068616C7465642E206B696C6CBB
:104E200028292063616C6C656421004B494C4C3A25
:104E30002025640A004D31303420496E76616C695A
:104E40006420657874727564657220004D31303568
:104E500020496E76616C696420657874727564654A
:104E60007220004D31303920496E76616C696420C2
:104E7000657874727564657220004D32313820494E
:104E80006E76616C696420657874727564657220F1
:104E9000004D32323120496E76616C69642065784C
:104EA00074727564657220006673656E736F725FED
:104EB0006F715F6D656173737572655F73746F7029
:104EC0002C20256868752073616D706C65730A000D
:104ED0006673656E736F725F6F715F6D656173731B
:104EE0007572655F73746172740A004D36303000FC
:104EF0004653454E534F525F5245434F564552001D
:104F00006673656E736F725F757064617465202D72
:104F1000204D3630300A006673656E736F725F65C0
:104F200072725F636E74203D20300A004731204565
:104F300033204632303000473120452D3320463271
:104F40003030004D3730310020573A0020453A00CC
:104F5000543A005A206C6976652061646A757374EE
:104F6000206F7574206F662072616E67652E205306
:104F7000657474696E6720746F20302E20436C69ED
:104F8000636B20746F20636F6E74696E75652E009D
:104F90005A206C6976652061646A757374206F7538
:104FA00074206F662072616E67652E20536574747D
:104FB000696E6720746F20300048656174696E67A0
:104FC0002064697361626C65642062792073616634
:104FD0006574792074696D65722E00000E131511C9
:104FE0000E00000004120912040000001C1F111121
:104FF0001F00000006191803130C00040E1F041CE8
:10500000000000040A0A0A0A11110E001F151115EA
:105010001F0000000103161C0800000000110A0414
:10502000110A040C12120C000000002563252D311A
:1050300038532563002563252E3135533A257325D2
:105040003364002563252E3132533A2573250045FC
:105050007872656D65207370616E206F662074686C
:1050600065205A2076616C7565732100000040410F
:10507000000000400000E4420000004000005743F0
:1050800000000040000057430000C4420000E4421A
:105090000000C442000040410000C4420000404102
:1050A000000042430000E442000042430000574336
:1050B00000004243205B6F66665D00426564206CC1
:1050C0006576656C696E67206661696C65642E2023
:1050D00053656E736F72206469646E7420747269B4
:1050E000676765722E20446562726973206F6E2057
:1050F0006E6F7A7A6C653F2057616974696E6720BC
:10510000666F722072657365742E001000C90210FC
:10511000012C014001220170011801B0010E01F0C3
:105120000104015002FA00B002F0003003E600D0A2
:1051300003DC009004D2007005C800A006BE000089
:1051400008B400B009AA00D00BA000600E96006061
:10515000118C000015820020197800C01D6E00A07F
:10516000226400B0275A00902C500000314600E025
:10517000343C0010383200903A2800603C1E00A0F9
:105180003D1400803E0A00203F000070012C019079
:10519000012701B0012201C0011D01F00118011019
:1051A00002130130020E016002090190020401C0E5
:1051B00002FF000003FA004003F5008003F000D076
:1051C00003EB002004E6007004E100E004DC004092
:1051D00005D700C005D2004006CD00D006C800802B
:1051E00007C3003008BE00F008B900C009B400B021
:1051F0000AAF00B00BAA00D00CA500000EA0005012
:105200000F9B00C01096005012910000148C00C03B
:10521000158700B0178200B0197D00D01B78000000
:105220001E730040206E0090226900F0246400404C
:10523000275F0090295A00E02B5500102E500020C7
:10524000304B0010324600E033410090353C0010F6
:1052500037370070383200A0392D00B03A2800A04E
:105260003B2300603C1E00103D1900903D140010CF
:105270003E0F00703E0A00C03E0500003F00009057
:10528000137D00B0157800F0177300601A6E00F0FF
:105290001C6900A01F640050225F0020255A00E016
:1052A000275500902A5000202D4B00A02F4600F0DB
:1052B00031410010343C00F0353700A03732002077
:1052C000392D00603A2800703B2300603C1E00200E
:1052D0003D1900C03D1400403E0F00A03E0A00F002
:1052E0003E0500403F0000703FFBFF903FF6FFB0DF
:1052F0003FF1FFC03FECFFD03FE7FFE03FE2FFF0B0
:105300003FDDFFF03FD8FF20484F54454E44205426
:105310004845524D414C2052554E4157415900206D
:105320004845415442454420544845524D414C2043
:1053300052554E4157415900544845524D414C2019
:1053400052554E4157415900424544205448455218
:105350004D414C2052554E4157415900205448452B
:10536000524D414C2052554E415741592028205012
:1053700052454845415420484F54454E4429002049
:10538000544845524D414C2052554E4157415920A9
:1053900028205052454845415420484541544245F3
:1053A00044290050524548454154204552524F52DD
:1053B00000424544205052454845415420455252F0
:1053C0004F52004572723A204D415854454D50009D
:1053D0003A204578747275646572207377697463D6
:1053E000686564206F66662E204D415854454D50C7
:1053F0002074726967676572656420210045727266
:105400003A204D415854454D502042454400546582
:105410006D7065726174757265206865617465642C
:1054200020626564207377697463686564206F66C1
:10543000662E204D415854454D502074726967675F
:10544000657265642021004572723A204D494E54C0
:10545000454D50204245440054656D70657261743D
:105460007572652068656174656420626564207387
:1054700077697463686564206F66662E204D494EB7
:1054800054454D50207472696767657265642021C8
:10549000004572723A204D494E54454D50003A2015
:1054A0004578747275646572207377697463686592
:1054B00064206F66662E204D494E54454D50207431
:1054C0007269676765726564202100746D633231AB
:1054D00033305F686F6D655F656E746572286178E3
:1054E00065735F6D61736B3D307825303278290AC2
:1054F00000746D63323133305F686F6D655F65785E
:10550000697420746D63323133305F73675F686F25
:105510006D696E675F617865735F6D61736B3D3058
:1055200078253032780A0043616E6E6F7420656EA4
:10553000746572207375626469723A200053442066
:1055400063617264206F6B006F70656E526F6F7471
:10555000206661696C656400766F6C756D652E6997
:105560006E6974206661696C656400534420696EDD
:105570006974206661696C0057726974696E67208E
:10558000746F2066696C653A200046696C6520730B
:10559000656C6563746564002053697A653A200020
:1055A00046696C65206F70656E65643A20001F1F48
:1055B0001F1F1F1F1F1F2E002E004E6F77206672A9
:1055C0006573682066696C653A20004E6F772064C9
:1055D0006F696E672066696C653A20002220706FE3
:1055E00073002220706172656E743A220053554236
:1055F000524F5554494E452043414C4C20746172E2
:105600006765743A2200747279696E6720746F203E
:1056100063616C6C207375622D67636F64652066CF
:10562000696C6573207769746820746F6F206D6191
:105630006E79206C6576656C732E204D4158206C18
:105640006576656C2069733A00536F7274696E6792
:105650002066696C657300536F6D652066696C65C3
:10566000732077696C6C206E6F7420626520736F95
:10567000727465642E204D61782E204E6F2E206F3F
:10568000662066696C657320696E203120666F6CD8
:1056900064657220666F7220736F7274696E672022
:1056A0006973203130302E00773235783230636CB8
:1056B0005F63666D0A00773235783230636C5F6500
:1056C0006E7465720A0020746F6F206C6F6E6720B5
:1056D000657874727573696F6E2070726576656E29
:1056E0007465640020636F6C6420657874727573F0
:1056F000696F6E2070726576656E746564004669C8
:105700006C616D656E742073656E736F723A0050D4
:1057100072696E742066616E3A00457874727564C1
:1057200065722066616E3A0053656C6674657374C9
:10573000206661696C6564202000416C6C20636F99
:105740007272656374202020202020004368656306
:105750006B696E672073656E736F727320004368A8
:1057600065636B696E6720626564202020202000DD
:10577000436865636B696E67205A2061786973209E
:105780002000436865636B696E6720592061786902
:1057900073202000436865636B696E672058206141
:1057A000786973202000436865636B696E672068C1
:1057B0006F74656E64202000436865636B696E6773
:1057C00020656E6473746F7073004572726F72201F
:1057D0002D20737461746963206D656D6F7279201B
:1057E000686173206265656E206F76657277726995
:1057F0007474656E00436172642072656D6F7665C6
:1058000064004361726420696E736572746564003C
:105810002D2D2D2D2D2D2D2D2D2D2D2D2D2D2D2DB8
:105820002D2D2D2D0043616C6962726174696E6764
:1058300020686F6D65000000000000110A045052DE
:1058400055534133444657002079303D25640A00C2
:105850002078303D25640A004F4B0A004552524FD4
:10586000522061643D25640A002020207A303D25C5
:10587000640A00207A303D25640A002079303D25F5
:10588000640A002078303D25640A0078797A6361E3
:105890006C5F66696E645F706F696E745F63656E7E
:1058A000746572320A0000002100240027002A00DB
:1058B0002D003000330001010000040107010A013E
:1058C000000020002300260029002C002F003200B9
:1058D0000001000003010601090100000A0B020992
:1058E0000C0D0E080703040100000000000000007A
:1058F00000000000000000000000000000000000A8
:105900000000000000001211100000000000000064
:105910000000000000000000000000000000000087
:105920000000000000000000000000000000000077
:1059300057616974696E6720666F72206E6F7A7A3C
:105940006C6520616E642062656420636F6F6C69B2
:105950006E670053656C662074657374204F4B004E
:1059600053656C662074657374207374617274205F
:10597000200046696C616D656E742073656E736F8F
:105980007200537761707065640046726F6E742F99
:105990006C6566742066616E7300417869730041BE
:1059A000786973206C656E677468004C6F6F7365FF
:1059B0002070756C6C657900456E6473746F70202F
:1059C0006E6F742068697400456E6473746F700044
:1059D0004D6F746F7200456E6473746F707300570F
:1059E0006972696E67206572726F72004265642029
:1059F0002F20486561746572004E6F7420636F6E6E
:105A00006E6563746564004865617465722F5468DF
:105A100065726D6973746F7200506C656173652097
:105A2000636865636B203A0053656C6674657374D4
:105A3000206572726F722021006C63645F73656C05
:105A400066636865636B5F617869732025642C20E9
:105A500025640A004D3834004731205A313520463C
:105A6000313030300047323820570025632041580C
:105A70004953205347313D25640A0041786973201A
:105A80006C656E67746820646966666572656E63CE
:105A9000653A252E33660A004D656173757265643B
:105AA0002061786973206C656E6774683A252E33BF
:105AB000660A00332E352E31007263006265746110
:105AC00000616C706861006465760078797A636162
:105AD0006C5F73706972616C322063783D2564205D
:105AE00063793D2564207A303D256420647A3D2524
:105AF00064207261646975733D25642061643D258D
:105B0000640A0001021020200808102040102040E4
:105B10008002010201080402010102040810204071
:105B2000808040201008040201800402018040208F
:105B300010080402010804020101020408102040B8
:105B40008001020408102040801008040880102002
:105B500040044080102040048000002200250028DE
:105B6000002B002E00310034000201000005010866
:105B7000010B0105050505070508080808020202D2
:105B8000020A0A08080404040401010101010101D8
:105B9000010303030303030303040707070C0C0CAF
:105BA0000C0C0C0C0C020202020606060606060687
:105BB000060B0B0B0B0B0B0B0B07070A0A0A0A0A47
:105BC0000A050505040404080802746D63323133C4
:105BD000305F676F746F5F73746570202564202574
:105BE00064202564202564200A002E006F70656EF5
:105BF000206661696C65642C2046696C653A2000FA
:105C0000436F6E74696E7565207769746820616E84
:105C10006F7468657220626F7764656E3F0025005F
:105C2000202020202020002020202020200045525D
:105C30004153494E4720616C6C2064617461004699
:105C40006163746F72792052455345540000007FA0
:105C500043008054430000524300000000000080D5
:105C6000C09A99193E00000000000080C09A99195E
:105C70003E0000A0400000A040000000402533642A
:105C800020737465703D253264206D73636E743DBE
:105C90002534640A0000007F43008058439AD9519C
:105CA00043FFFFFF46696C616D656E74206F75740C
:105CB000206F662072616E6765202564200A006788
:105CC000636F64655F4D37303120626567696E0AC6
:105CD00000504154393132355F5245535F593D25AB
:105CE0006868750A00504154393132355F52455366
:105CF0005F583D256868750A00555341525432205B
:105D000072782046756C6C2121210A0053657474E9
:105D1000696E67732053746F7265640053746F7299
:105D200065642073657474696E677320726574723C
:105D300069657665640048617264636F64656420B8
:105D400044656661756C742053657474696E67731D
:105D5000204C6F6164656400563200000000C84248
:105D60000000C8420000C84300008C4300004843C4
:105D700000004843000040410000F042E8030000FA
:105D8000E8030000C80000008813000000409C44A5
:105D900000409C440000000000000000204E000075
:105DA0000000204100002041CDCCCC3E000020402E
:105DB000000000000000000000000000CDCCCC3E40
:105DC0003D0A8141FF08433EB099AB438F42FC42FC
:105DD000E65A343F4C62B0450000000000404000ED
:105DE00000344200000000000000000000004100FC
:105DF0000000E03F0000C8420000C84200004041EF
:105E00000000F042C0030000C0030000C800000012
:105E100088130000454550524F4D204572726F72F5
:105E2000004D3234004D3233202573006175746F9C
:105E300025692E670022206661696C65643A2042FC
:105E400075666665722066756C6C2100456E7175AD
:105E500065696E6720746F207468652066726F6E66
:105E6000743A2022004572726F723A002200456E29
:105E7000717565696E6720746F207468652066723D
:105E80006F6E743A2022006563686F3A0045727243
:105E90003A205052494E542046414E204552524FCE
:105EA00052005072696E742066616E207370656571
:105EB00064206973206C6F776572207468656E204A
:105EC0006578706563746564004572723A20455860
:105ED00054522E2046414E204552524F5200457892
:105EE0007472756465722066616E20737065656496
:105EF000206973206C6F776572207468656E206509
:105F000078706563746564002F2F20616374696F16
:105F10006E3A7061757365002563252E3132533AF0
:105F20002573252B30362E3166002020202020209E
:105F30002020202020202020202020202020003E63
:105F4000003E0020003E003E0020004E6F74207393
:105F500070696E6E696E67005370696E6E696E6708
:105F6000004C65667420686F74656E642066616EAF
:105F70003F0046726F6E74207072696E74206661A5
:105F80006E3F0046616E20746573740046696C2E26
:105F90002058643A2533642059643A2533640A4909
:105FA0006E743A202533642020536875743A202596
:105FB00033640046696C616D656E742073656E7341
:105FC0006F720A69732064697361626C65642E0084
:105FD0001B5B303B304825533A2025346420525017
:105FE0004D0A25533A20202534642052504D0A0092
:105FF0005072696E742046414E004E6F7A7A6C651D
:106000002046414E00546F74616C004C61737420E3
:106010007072696E74004D4D55206C6F616420661E
:1060200061696C73004D4D55206661696C73004C5D
:10603000617374207072696E74206661696C757228
:106040006573004D4D5520706F77657220666169EC
:106050006C73004D4D55206C6F6164206661696CF6
:1060600073004D4D55206661696C7300546F746107
:106070006C206661696C7572657300437261736848
:106080000046696C616D2E2072756E6F75747300B9
:10609000506F776572206661696C75726573005424
:1060A0006F74616C206661696C7572657300437210
:1060B0006173680046696C616D2E2072756E6F7534
:1060C000747300506F776572206661696C757265D4
:1060D00073004C617374207072696E74206661691C
:1060E0006C7572657300546F74616C004C617374ED
:1060F000207072696E74001B5B303B304825531B67
:106100005B313B314825532020252D33641B5B3206
:106110003B314825532020252D33641B5B333B3115
:1061200048001B5B303B304825531B5B313B3148FB
:1061300025532020252D33641B5B323B31482553EA
:106140002020252D33641B5B333B3148255320250C
:106150002D3364001B5B303B304825531B5B313BC8
:10616000314825532020252D33641B5B323B3148B9
:1061700025532020252D33641B5B333B31482553A9
:1061800020205820252D336420205920252D3364CC
:10619000001B5B303B304825531B5B313B314825AE
:1061A000532020252D33641B5B323B31482553207F
:1061B00020252D33641B5B333B3148255320205869
:1061C00020252D336420205920252D3364008E0195
:1061D000480111241FBECFEFD1E2DEBFCDBF00E0EA
:1061E0000CBF16E0A0E0B2E0EAE0F8E703E00BBF86
:1061F00002C007900D92A03BB107D9F729E1A0EBAF
:10620000B6E001C01D92A53DB207E1F710E3C8EE6C
:10621000D0E300E006C021970109802FFE010F9412
:1062200010BBC73ED10780E00807A9F70F944B8F3A
:106230000D94F4BB0C9400002F923F924F925F920A
:106240006F927F928F929F92AF92BF92CF92DF9286
:10625000EF92FF920F931F93CF93DF93CDB7DEB7EB
:10626000C757D1090FB6F894DEBF0FBECDBF8091DE
:106270009D1390919E13892B11F40C94877082E0EA
:1062800090E090932602809325028AE393E00F9496
:1062900000678823B1F08091100D9091110D6AE292
:1062A00070E005960F9473BB009711F0DC011C920F
:1062B0008091100D9091110D05960F94844B0C94C4
:1062C000A56BC0908C15D0908D1586010E551C4E77
:1062D00046E050E069E870E1C8010F94D4AB892B27
:1062E00009F0EFC08FE393E00F940067882309F46F
:1062F0009BC088E50F9448A7182F89E50F9448A7FD
:10630000811112600F94F9888091B10601E0080FA5
:106310000093B106811105C089E696E10E9411E360
:106320000EC048EC5FEA60E070E089E696E10E940A
:10633000CCE2882331F0109269161092B10601E088
:1063400007C0033049F7109269161092B10600E0B9
:1063500081E00F94AB190F94A11982E00F941712EA
:1063600010FF15C086E69FE00F94A2B561E0680FAC
:1063700086E69FE00F94B4B585E09FE00F94AFB53B
:10638000BC016F5F7F4F85E09FE00F94CEB511FF9A
:1063900015C088E69FE00F94A2B561E0680F88E61B
:1063A0009FE00F94B4B583E09FE00F94AFB5BC01BC
:1063B0006F5F7F4F83E09FE00F94CEB581E00F9435
:1063C000AB1982E00F94171282E692E10F94184AFB
:1063D00040E061E081E00F94CF750F94F9880023CD
:1063E00021F061E084E99DE01BC0E091060DF0E042
:1063F000EE0FFF1FE257FA4E1182108240E060E07C
:1064000084E492E10E948FDF182F81E00F94AB1992
:1064100061E0112319F086E89DE002C089E79DE064
:106420000E9459E10C94A56B8EE493E00F940067F1
:10643000882379F08091390E882331F060E070E094
:1064400080E89FE30E9402CC81E080930F020C94CD
:10645000A56B8CE593E00F940067882311F40C94EE
:10646000A56B1092390E81E080930F0280916B0E24
:10647000811104C00E943BBC0C94A56B813011F0CB
:106480000C94A56BE8E6FDE084918F01882339F038
:106490000F94B9760F5F1F4FF8018491F7CF8AE010
:1064A0000F94B976EDE6F7E184918F01882311F41A
:1064B0000C94326A0F94B9760F5F1F4FF8018491E4
:1064C000F5CF44E050E064E870E1C8010F94D4AB2C
:1064D000892B09F00EC186010A551C4E49E050E097
:1064E0006AE770E1C8010F94D4AB892BD9F4F601A7
:1064F000E155FC4E1081153431F01855143010F070
:106500000C94A56B01C013E04AE050E060E070E03D
:10651000C60180559C4E0F9462AA812F0F94FE5A9B
:106520000C94A56B49E050E060E770E1C8010F945E
:10653000D4AB892B61F5F601E155FC4E1081153481
:1065400031F01855143010F00C94A56B01C013E015
:106550004AE050E060E070E0C60180559C4E0F9428
:1065600062AAE12FF0E0E85EF84F40E051E00080E1
:1065700002C0569547950A94E2F7842F880F880F3A
:1065800081506823812F0F94AC5C0C94A56B49E07B
:1065900050E066E670E1C8010F94D4AB892B11F08E
:1065A0000C94A56BF601E155FC4E8081853449F0D1
:1065B00008EA902E980EF3E0F91510F40C94A56BF0
:1065C00002C013E0912EE92CF12C5701AA0CBB1C40
:1065D000F501E65BFD4F1081012F0F70712E729453
:1065E000BFE07B22272D2770722E111F1127111F4C
:1065F00061816770660F162BF501E55BFD4F8081A9
:10660000882E869486948694382D3370832E1A8231
:106610001982C60180559C4EDC012C912223E1F1A8
:106620004AE050E0BE016F5F7F4F0F9462AA062FD1
:106630000F7089819A81009779F1FC0120812223D2
:1066400059F14AE050E0BE016F5F7F4F0F9462AA9C
:106650006770762E89819A810097F1F0DC012C9188
:106660002223D1F04AE050E0BE016F5F7F4F0F94CC
:1066700062AA162F1F7089819A81009769F0FC0128
:106680002081222349F04AE050E0BE016F5F7F4F36
:106690000F9462AA6370862EF501E65BFD4F972D7D
:1066A00097709295907F612F679566276795902BDD
:1066B000962B9083612F66951181107E882D8370B3
:1066C000880F880F880F162B182B1183C701845E43
:1066D0009D4FD701A05EBD4FB701685E784FFC01AA
:1066E00020814C91DB016C91892D0E94CFF40C9498
:1066F000A56B89E693E00F940067882321F00E9440
:10670000D08A0C94A56B89E793E00F9400678823E7
:1067100009F4B5C18FE793E00F940067882391F0E7
:106720008091A90F882311F40C94A56B0F94FB455D
:1067300060937F16709380168093811690938216D3
:106740000C94A56B84E893E00F940067882349F0CC
:106750008091C30E8F938091C20E8F938AE497E04D
:106760003DC088E893E00F940067882329F14091A9
:106770001510509116102CE3249FC001259F900DF9
:1067800011249F938F934091131050911410249FC4
:10679000C001259F900D11249F938F9383E397E071
:1067A0009F938F930F94AEAC0F900F900F900F901C
:1067B0000F900F900C94A56B8CE893E00F940067FA
:1067C0008823C9F08091A90F882391F08091320726
:1067D0008F93809131078F9380E397E09F938F93FE
:1067E0000F94AEAC0F900F900F900F900C94A56B80
:1067F0008EE197E0F0C08FE893E00F940067882364
:1068000021F0109230070C94A56B83E993E00F946C
:106810000067882349F060E085EA9FE00F94B4B5F3
:1068200061E082E690E1FCCD88E993E00F94006797
:10683000882321F00E94669A0C94A56B8FE993E05F
:106840000F940067882319F18091A90F8823C9F05C
:106850008AEA95E5DC018093FC1F9093FD1FA093CD
:10686000FE1FB093FF1F88E08093FB1F98E10FB6D7
:10687000F894A895909360000FBE80936000F89400
:10688000FFCF85EA93E00F94BB770C94A56B87EB61
:1068900093E00F940067882339F18091100D909157
:1068A000110D41E061E003960F948E268091B3189C
:1068B0009091B418A091B518B091B6188093601952
:1068C00090936119A0936219B09363198BEA98E1D0
:1068D0000E9408E98C010F94B9760A30110531F74E
:1068E0000F94CA560C94A56B8AEB93E00F94006743
:1068F000882381F00F94D36D81E0809343078091CA
:10690000100D9091110D41E060E004960F948E26D9
:106910000C94A56B8EEB93E00F940067882309F429
:106920005EC08091A90F882309F453C0109290157E
:106930006091CF197091D0198BE390E00F94DFB480
:106940006091CF197091D01983E590E00F94DFB476
:1069500019821B821A82CE0101960E94C0E200E0D9
:1069600010E0FF24F3948091E20D9091E30D2091CB
:10697000E40D3091E50D821B930B8F779927892BBE
:1069800081F00F941576F09290156091CF19709167
:10699000D01990E00F94DFB40F5F1F4F1092901545
:1069A000E2CF64E670E0CE0101960E9497E2811189
:1069B00003C003311105BCF281E080939015609112
:1069C000CF197091D0198AE090E00F94DFB40C9445
:1069D000A56B83E295E00F94D5AC0C94A56B81EC8C
:1069E00093E00F940067882361F005EC13E0F80151
:1069F00081918F01882311F40C94326A0F94B97637
:106A0000F6CF80ED93E00F940067882361F004EDEA
:106A100013E0D8018D918D01882311F40C94326A12
:106A20000F94B976F6CF83EF93E00F94006781114E
:106A30000C94A56B88EF93E00F940067882341F0D6
:106A400060E070E088EF9FE00E94D9C80C94A56BCD
:106A50008BEF93E00F940067882321F00F94FB45A0
:106A60000C94A56B80E094E00F940067882311F4E8
:106A70000C94A56B80E00F94F6680C94A56B8EE5E2
:106A80000F9448A78AAF81110C94A56B87E40F94EB
:106A900048A7F82E882311F40C9420430F9440A7A4
:106AA0000F948DB76C34710509F404C27CF5643021
:106AB000710509F4FCC054F46230710509F4E2C0B8
:106AC0000CF0E9C077FF6DC00C9414436C31710574
:106AD00009F43FC15CF46A30710509F435C16B30CB
:106AE000710511F00C94144380E02FC16E317105D3
:106AF00009F471C16B34710511F00C94144308E270
:106B000010E0F0EFEF2EF6E0FF2EB5C1683571050D
:106B100011F40C94A56BECF46135710511F40C942F
:106B2000DB4154F46F34710509F431C760357105E8
:106B300009F459C70C9414436635710511F40C948B
:106B400084426735710511F00C94144381E00C9474
:106B500085426C35710511F40C948D427CF46A35D4
:106B6000710511F40C9489426B35710511F00C9488
:106B7000144381E08093FE0E0C94A56B6236710580
:106B800011F40C94ED426336710511F00C9414432A
:106B90001092A90F60E084EC9FE00F94B4B50C94C0
:106BA0000F4380913F0F81110C94A56B0F9416A495
:106BB0006091260E7091270E8091280E9091290EDB
:106BC0000F9446AD6B017C014090481050904910E5
:106BD00060904A1070904B108090B60F9090B70F55
:106BE000A090B80FB090B90FA5019401C301B201F4
:106BF0000F942DB620E030E048EC52E40F943AA810
:106C00009B01AC01C701B6010F9479B81816D4F4F2
:106C1000A3019201C501B4010F942DB620E030E02C
:106C200048EC52E40F943AA8A70196010F942EB6AF
:106C30000F9493B76093260E7093270E8093280EBF
:106C40009093290E80910211882311F40C94A36B68
:106C500088E50F9448A781110C94A36B89E50F94E4
:106C600048A781110C94A36B8AE50F9448A7811162
:106C70000C94A36B85E40F9448A781110C947A6B54
:106C80000C94A36B80913F0F81110C94A56B0F9412
:106C9000D3A481E008C080913F0F81110C94A56BB3
:106CA0000F94D3A480E00F94D99D0C94A56B80E53C
:106CB0000F9448A7882339F00F9440A70F9493B7F7
:106CC0006B017C0103C0C12CD12C760183E50F94AC
:106CD00048A7882361F00F9440A720E030E04AE7FE
:106CE00054E40F943AA80F9493B76B017C01C1143C
:106CF000D104E104F10421F085E197E00F94184AF2
:106D00000F94F9880F94FB45C60ED71EE81EF91E96
:106D10000F94FB456093030F7093040F8093050F4E
:106D20009093060F0F94FB456C157D058E059F050E
:106D300010F00C94A56B0F94AA8380E00F94730855
:106D400080E00F941712EECF81E00F9401A50C9410
:106D5000A56B88E50F9448A78EAF0F9436A71B014B
:106D60002C0189E50F9448A7682E0F9436A7269624
:106D70006CAF7DAF8EAF9FAF26978AE50F9448A783
:106D8000D82E0F9436A74B015C0187E50F9448A7D6
:106D9000782E83E40F9448A77F928F93CD2C26966C
:106DA000ECACFDAC0EAD1FAD2697262DB201A101B6
:106DB0008EAD0F94ED720F900F90BEADB1110C948B
:106DC000A56B61100C94A56B71100C94A56BD11080
:106DD0000C94A56B08C60F94F98881E00F94166592
:106DE0008C0180E090E0A8E4B4E480937C0290936E
:106DF0007D02A0937E02B0937F0260E070E080E2AB
:106E000091EC0F944625809147108F938091461006
:106E10008F93809145108F93809144108F93809130
:106E200043108F93809142108F93809141108F93E4
:106E3000809140108F9380913F108F9380913E10EE
:106E40008F9380913D108F9380913C108F938BEFA7
:106E50009AE39F938F9389EF96E09F938F930F947C
:106E6000AEACC8010F94F5640FB6F894DEBF0FBE48
:106E7000CDBF0C94A56BB801012E000C880B990BAB
:106E80000F9448AD0F94B1029F938F937F936F93AC
:106E90001F930F93FF92EF920F94AEAC0F5F1F4FB3
:106EA0000FB6F894DEBF0FBECDBF0F36110519F730
:106EB0000C94A56B0F94506C8A3F30F080E393E103
:106EC0000E9433E00C94A56B8091070D882341F05C
:106ED0008091080D882321F08091090D811106C051
:106EE00081E080939C138BE590E197C589EE92E158
:106EF0000E9433E040E060E089E39BE10E948FDF85
:106F0000882309F493C080E090E0A0EAB0E4809385
:106F1000441090934510A0934610B09347102091D1
:106F200040103091411040914210509143106091B7
:106F30003C1070913D1080913E1090913F10F6E012
:106F40006F2EFDE07F2E7F926F92812C912CA8E412
:106F5000AA2EA2E4BA2EB8E4CB2EB0E1DB2EE12CAF
:106F6000F12C00EA10E40F94C83080924410909203
:106F70004510A0924610B092471080E090E0A4E344
:106F8000B3E48093401090934110A0934210B093CB
:106F9000431060913C1070913D1080913E10909193
:106FA0003F107F926F928501740120E030E044E34E
:106FB00053E40F94C8300F94F98881E19BE10E945B
:106FC00033E0E5E7FEE12591359145915491209319
:106FD0004010309341104093421050934310E1E72A
:106FE000FEE1659175918591949160933C10709349
:106FF0003D1080933E1090933F10E0904410F0902D
:10700000451000914610109147107F926F920F9497
:10701000C8300F94F98841E060E080E00F94CF75AC
:107020000F900F900F900F900F900F9020E030E096
:107030004CE052E460915D0E70915E0E80915F0EA7
:107040009091600E0F9479B818160CF0A4C080913E
:10705000A90F8111A0C080E090E0A8ECB2E4809379
:10706000441090934510A0934610B0934710209180
:107070004010309141104091421050914310609166
:107080003C1070913D1080913E1090913F10E6E0D1
:10709000FDE0FF93EF93812C912C18E4A12E12E4D4
:1070A000B12E08E4C02E00E1D02EE12CF12C08EC2A
:1070B00012E40F94C83080E090E0ACE0B2E48F8F2F
:1070C00098A3A9A3BAA30F94C61419821A821B828B
:1070D0001C82CE0101960F94A37C10920B0D10928E
:1070E0000A0D19821A821B821C821D82CE01019612
:1070F0000E9411E30F900F902F8D38A149A15AA142
:1071000060915D0E70915E0E80915F0E9091600EA9
:107110000F9479B8181694F584E292E10E9482DF08
:1071200064E080E00F94F21482E00E949A868DE57C
:107130009EE00E94068C0F94941383E094E00F94D9
:107140009413CE014F960E94068C0F94941385E001
:1071500094E00F94941388EE93E00F94B70C0E9480
:10716000F2D740E053E567E070E0CE0101960E945F
:10717000CCE2882309F4C0CF10E001C011E066E33F
:1071800078E581E00F94A71481E00F94AB191111F9
:1071900002C080E0F8C381E00F94AB1981E090E079
:1071A0009093260280932502EDE3F0E184918F0114
:1071B000882339F00F94B9760F5F1F4FF80184913F
:1071C000F7CF8AE00F94B9761A821982C0905D0ECB
:1071D000D0905E0EE0905F0EF090600E20E030E008
:1071E00040EA50E4C701B6010F941CB70F948DB765
:1071F00025E0269FA001279F500D1124BA01550FAD
:10720000880B990B0F9448AD3B01382E292E20E0B6
:1072100030E04CE052E40F9442AD87FF06C0612C91
:10722000712CACE03A2EB2E42B2EC101262D372D65
:10723000492F522DC701B6010F9479B8181674F46E
:1072400020E030E040EA50E4F101662D772D8F2FE9
:10725000922D0F942EB63B01382E292E2F923F925D
:107260007F926F9287ED96E09F938F930F94AEACD1
:1072700020E030E040EF51E4F101662D772D8F2FB3
:10728000922D0F942DB620E030E04CE852E40F949C
:107290002EB60F948DB770930B0D60930A0D84E09A
:1072A00090E090931F0E80931E0E81E090E09093EB
:1072B000F40E8093F30E88EE98E40F94184A80E061
:1072C00090E0A0EAB0E48093441090934510A0931E
:1072D0004610B093471020914010309141104091DA
:1072E00042105091431060913C1070913D1080917C
:1072F0003E1090913F10B6E04B2EBDE05B2E5F92AA
:107300004F92812C912C18E4A12E12E4B12E08E4A6
:10731000C02E00E1D02EE12CF12C00EA10E40F94F5
:10732000C83080E090E0A0EAB1E480933C109093F4
:107330003D10A0933E10B0933F1080E090E0A0E796
:10734000B2E48093401090934110A0934210B09308
:107350004310E0904410F0904510009146101091B9
:1073600047105F924F929C01AD0160E070E080EAAF
:1073700091E40F94C8308AE999E9A9E1BEE38093CA
:10738000441090934510A0934610B093471020915D
:107390004010309141104091421050914310609143
:1073A0003C1070913D1080913E1090913F105F9283
:1073B0004F921AE9E12E19E9F12E09E11EE30F942B
:1073C000C8300F94F9880FB6F894DEBF0FBECDBF5A
:1073D00020915D0E30915E0E40915F0E5091600ED7
:1073E000F101662D772D8F2F922D0F9479B81816F5
:1073F0003CF488EE93E00F94B70C0E94F2D7E8CFEC
:1074000060E086EA9FE00F94B4B580E090E0A0EAE7
:10741000B0E48093441090934510A0934610B0932D
:1074200047102091401030914110409142105091EE
:10743000431060913C1070913D1080913E109091EE
:107440003F1006E0402E0DE0502E5F924F92812CAF
:10745000912CE8E4AE2EE2E4BE2EF8E4CF2EF0E16B
:10746000DF2EE12CF12C00EA10E40F94C830E1E7A4
:10747000FEE1659175918591949160933C107093B4
:107480003D1080933E1090933F10E5E7FEE125917B
:107490003591459154912093401030934110409381
:1074A000421050934310E0904410F090451000912A
:1074B0004610109147105F924F920F94C8300F946E
:1074C000F98860E070E080E89FEB0F9446250F900C
:1074D0000F900F900F90882309F45BCE30914410E9
:1074E00027963FAF2797409145102B964FAF2B978C
:1074F000509146102F965FAF2F976091471063967B
:107500006FAF63976F935F934F933F938AEC96E0CF
:107510009F938F930F94AEAC0F900F900F900F909E
:107520000F900F908EEA9FE09FAF8EAF44244A9455
:10753000542C13E2C12ED12CE12CF12C8201B60186
:107540000D2C000C880B990B0F9448AD4B015C017E
:1075500097012F5F3F4F3BAF2AAFDF92CF923F9310
:107560002F934EE856E05F934F930F94AEAC0F907D
:107570000F900F900F900F900F908FEF48165806B6
:1075800011F40C947870BE016F5F7F4F8EAD9FAD8C
:107590000E94D9C8A5019401F101662D772D8F2F86
:1075A000922D0F9442AD1816A4F495E0E916F1045B
:1075B00071F095E0C90ED11CAFEF4A1A5A0AEEAD30
:1075C000FFAD3296FFAFEEAFEAACFBACB7CF05E054
:1075D00010E0C8018752984FDC01AA0FBB1FBFAF54
:1075E000AEAF3801B3E06B0E711C25E0209FC001E7
:1075F000219F900D11241BAE1AAEFC01BD9666961C
:10760000FFAFEEAF6697A6E04A2EADE05A2EC3015B
:10761000029705970CF0B6C166966EAD7FAD669782
:107620008AAC9BAC680D791D072E000C880B990B5A
:107630000F9448AD26966CAF7DAF8EAF9FAF269767
:107640007F926F92F1E8AF2EF6E0BF2EBF92AF921D
:107650000F94AEAC7092F40E6092F30E20E030E026
:1076600040EF51E426966CAD7DAD8EAD9FAD269773
:107670000F942DB620E030E040E251E40F943AA898
:1076800020E030E040EA50E40F941CB720E030E006
:1076900048E452E40F942EB60F948DB770930B0DFF
:1076A00060930A0D80E090E0A0EAB0E4809344107B
:1076B00090934510A0934610B0934710209140102E
:1076C00030914110409142105091431060913C1014
:1076D00070913D1080913E1090913F105F924F92BB
:1076E000812C912CA8E4AA2EA2E4BA2EB8E4CB2EC9
:1076F000B0E1DB2EE12CF12C00EA10E40F94C8304D
:1077000080E090E0A0EAB1E480933C1090933D10BB
:10771000A0933E10B0933F10812C912CF0E7AF2E38
:10772000F2E4BF2E8092401090924110A09242103D
:10773000B0924310E0904410F09045100091461034
:10774000109147105F924F92812C912C28E4A22E29
:1077500022E4B22E20E030E040E752E4BC01CD014B
:107760000F94C8302AE939E949E15EE320934410D7
:10777000309345104093461050934710209140108D
:1077800030914110409142105091431060913C1053
:1077900070913D1080913E1090913F105F924F92FA
:1077A0001AE9E12E19E9F12E09E11EE30F94C83020
:1077B0000F94F9880FB6F894DEBF0FBECDBF2091AD
:1077C0005D0E30915E0E40915F0E5091600E2696D8
:1077D0006CAD7DAD8EAD9FAD26970F9479B8181620
:1077E0003CF488EE93E00F94B70C0E94F2D7E7CFF9
:1077F00080E090E0A0EAB0E48093441090934510BC
:10780000A0934610B0934710209140103091411042
:10781000409142105091431060913C1070913D1086
:1078200080913E1090913F105F924F92812C912C4D
:10783000B8E4AB2EB2E4BB2E18E4C12E10E1D12E79
:10784000E12CF12C00EA10E40F94C830E1E7FEE1EE
:10785000659175918591949160933C1070933D1062
:1078600080933E1090933F10E5E7FEE1259135911E
:107870004591549120934010309341104093421011
:1078800050934310E0904410F09045100091461042
:10789000109147105F924F920F94C8300F94F9885F
:1078A00060E070E080E89FEB0F944625AAADBBAD89
:1078B0001596BBAFAAAFBFEF6B1A7B0A0F900F9064
:1078C0000F900F90811103C00F941A9D5BC02796F3
:1078D0007FAD27972B966FAD2B972F969FAD2F9748
:1078E00063968FAD6397272F362F492F582F6091BE
:1078F00044107091451080914610909147100F945C
:107900002DB6162F072FF82EE92E20918C103091CE
:107910008D1040918E1050918F10D801F7016B2F70
:107920007A2F8F2F9E2F0F943AA80F948DB77A83BA
:107930006983EF92FF920F931F938091600E8F9354
:1079400080915F0E8F9380915E0E8F9380915D0E7C
:107950008F93E5E5F6E0FF93EF930F94AEACBE0195
:107960006F5F7F4F8EAD9FAD0E94D9C82EAD3FADEA
:107970002E5F3F4F3FAF2EAF0FB6F894DEBF0FBE66
:10798000CDBF45CE81E00F941A9D0C94A56B0FEFEF
:1079900010E0ADE4CA2EA6E0DA2E1093BD190093D4
:1079A000BC19F4E6EF2EF12C84E690E00F94B70CAE
:1079B00051E0E51AF108C1F7809116108F9380917C
:1079C00015108F931F930F93DF92CF920F94AEAC4D
:1079D000055011090F900F900F900F900F900F907E
:1079E000E1F60C94A56B81E08093370E2091070D92
:1079F0008091FF0F90910010222341F02091080DFB
:107A0000222321F05090090D51100FC0029749F028
:107A100081E080939C1386E390E10F94A87C0C9402
:107A2000A56B1092370E0C94A56B0297D1F3809141
:107A30001E0E90911F0E28969FAF8EAF2897A09193
:107A4000F30EB091F40E2C96BFAFAEAF2C9781E041
:107A500090E090931F0E80931E0E83E190E0909330
:107A6000F40E8093F30E81E00F9417120F94886048
:107A70000E94129E80E090E0A0EAB0E4809344105F
:107A800090934510A0934610B0934710209140105A
:107A900030914110409142105091431060913C1040
:107AA00070913D1080913E1090913F10E6E06E2E57
:107AB000EDE07E2E7F926F92F5E58F2E982CA82C0C
:107AC000F1E4BF2EA8E4CA2EA0E1DA2EE12CF12CBD
:107AD00000EA10E40F94C830ECE6F0E5659175918A
:107AE0008591949160933C1070933D1080933E106B
:107AF00090933F10E0E7F0E5259135914591549141
:107B00002093401030934110409342105093431003
:107B1000E0904410F09045100091461010914710ED
:107B20007F926F92812C912CE8ECAE2EE2E4BE2E77
:107B30000F94C8300F94F9880F900F900F900F900A
:107B400005EC1FE0C8010F94AFB5019639F00E5F48
:107B50001F4F053DEFE01E07A9F75AAE80E00F94D6
:107B6000166560969FAF8EAF60978CE6482E80E5D5
:107B7000582E612C712CC30163E070E00F94E1BAC0
:107B800024967FAF6EAF24971C0160FF06C002E011
:107B9000802E912C881A990A14019AAC9920A1F18F
:107BA0006114710489F124968EAD9FAD2497880FDE
:107BB000991F2496AEACBFAC24978A0D9B1D820DF5
:107BC000931D880F991F8D53904F0F94AFB5BC0133
:107BD000990F880B990B0F9448AD2AE037ED43E2DB
:107BE0005CE30F943AA8209192153091931540913F
:107BF0009415509195150F942EB622966CAF7DAFCB
:107C00008EAF9FAF229706C022961CAE1DAE1EAE51
:107C10001FAE229720E030E040EA50E42093441069
:107C200030934510409346105093471020914010D8
:107C300030914110409142105091431060913C109E
:107C400070913D1080913E1090913F10A6E0BDE0F4
:107C5000BF93AF93812C912CB0EAAB2EB1E4BB2E35
:107C600018E4C12E10E1D12EE12CF12C00EA10E431
:107C70000F94C8300F94F988F20185919591A591E0
:107C8000B49180933C1090933D10A0933E10B0931C
:107C90003F10F201349685919591A591B49180930E
:107CA000401090934110A0934210B093431060E4B1
:107CB00070E18CE390E10F94C267E0904410F09083
:107CC00045100091461010914710209140103091BE
:107CD0004110409142105091431060913C107091BE
:107CE0003D1080913E1090913F10F6E08F2EFDE008
:107CF0009F2E9F928F92812C912CA6E1AA2EA3E415
:107D0000BA2E0F94C8300F94F9880F900F900F90EF
:107D10000F90BAACBB2081F06114710469F020E0CF
:107D200030E040E85FE322966CAD7DAD8EAD9FAD57
:107D300022970F942DB604C060E070E080E291ECD1
:107D40000F944625882309F48BC0C0904410D0902E
:107D50004510E0904610F0904710A701960160E0B2
:107D600070E080EA90E40F942DB62DEC3CEC4CECE6
:107D70005DE30F9442AD87FD73C02AAD2223A1F0CD
:107D8000A701960122966CAD7DAD8EAD9FAD229779
:107D90000F942DB69F7720E030E040E85FE30F942A
:107DA00079B818160CF45CC0C0905D0ED0905E0ED1
:107DB000E0905F0EF090600E809117078823A9F085
:107DC0000F94E768882389F0C701B6010F94B102C8
:107DD00020918C1030918D1040918E1050918F1009
:107DE0000F941CB79B01AC0103C020E030E0A90157
:107DF000A7E024968EAD9FAD2497A89F8001A99FF0
:107E0000100D1124020D131D000F111F000F111F63
:107E10000F561A4E60914410709145108091461093
:107E2000909147100F942DB6F8016183728383837C
:107E300094838091F30E9091F40E01979093F40E39
:107E40008093F30EFFEF6F1A7F0A81E00F941712F1
:107E500028E0420E511C39E06316710409F08BCE04
:107E600080E090E0A0EAB0E4809344109093451045
:107E7000A0934610B09347102091401030914110CC
:107E8000409142105091431060913C1070913D1010
:107E900080913E1090913F10E6E0FDE0FF93EF935C
:107EA000812C912C00EAA02E01E4B02EE8E4CE2E25
:107EB000E0E1DE2EE12CF12C00EA10E40F94C83052
:107EC0000F94F9880F900F9049E06416710409F43B
:107ED000B3C08091090790910A078130910531F074
:107EE00018F0029719F005C080E001C081E00E94FF
:107EF00078B4B6E06B2EBDE07B2E212C312C10EA3D
:107F0000412E10E4512E87EB92E10E9482DF8EE138
:107F100090E00F94B59C0F944F655091BC0F5AAFF1
:107F20001092BC0F1092BB0F20E030E040E85FE3FE
:107F300060914410709145108091461090914710C7
:107F40000F942DB67B018C01609344107093451003
:107F5000809346109093471020914010309141102B
:107F6000409142105091431060913C1070913D102F
:107F700080913E1090913F107F926F92812C912CB6
:107F8000E0EAAE2EE1E4BE2EF8E4CF2EF0E1DF2EE3
:107F90000F94C8300F94F98861E06093BC0F109281
:107FA000BB0F84E00F94831A209244103092451046
:107FB000409246105092471020914010309141104D
:107FC000409142105091431060913C1070913D10CF
:107FD00080913E1090913F107F926F92E12CF12C96
:107FE00000EA10E40F94C8300F94F9880F94E81950
:107FF0008AAD8093BC0F1092BB0F82E00F94E6888D
:108000000F900F900F900F90A80197010F9479B8DF
:1080100018160CF478CF10921F0E10921E0E81E0ED
:108020000F94AB1941E061E081E00F94CF7581E0DE
:1080300080939C130C94A56B60968EAD9FAD60975A
:108040000F94F5640E94BF9D6091040D7091050D21
:10805000072E000C880B990B0F9448AD9058209177
:108060008C1030918D1040918E1050918F100F9484
:108070001CB70E94D09D80EC9FE00F94A2B5082F02
:10808000DE0111961D0110E08090890290908A0215
:10809000A0908B02B0908C028AAE9BAEACAEBDAE0F
:1080A00055EE852E55E1952E2AAD3BAD4CAD5DAD1F
:1080B00029833A834B835C83D1018D911D010F94F9
:1080C00048A7882319F00F9436A71BC0013009F088
:1080D00026C1123028F4112341F08EEB9FE00AC034
:1080E000123031F08CEB9FE005C08FEB9FE002C0B7
:1080F0008DEB9FE00F94A2B5682F880F770B880B4C
:10810000990B611571058105910509F408C10F945A
:1081100048AD2FE632E143E85AE30F943AA86B01E9
:108120007C019F7727E139ED4EEC5DE30F9479B840
:1081300018160CF033C0E5E6FEE584915F01882354
:1081400041F00F94B976FFEFAF1ABF0AF5018491A1
:10815000F6CFE2E1F0E184915F01882341F00F94D2
:10816000B976FFEFAF1ABF0AF5018491F6CF42E06E
:10817000C701B6010F943E77E9E0F0E184917F01F9
:10818000882341F00F94B976FFEFEF1AFF0AF70149
:108190008491F6CF8AE00F94B976C1C020E030E038
:1081A00040E05FE3C701B601123009F461C013304B
:1081B00009F48AC0113071F10F943AA82B013C01E7
:1081C00041E9A42E45E1B42EA3019201D5011596F3
:1081D0006D917D918D919C9118970F942EB6F5011C
:1081E0006583768387839087A70196016181728179
:1081F000838194810F942EB6D50111966D937D9352
:108200008D939C931497BCE1AB0EB11C8A149B0414
:10821000D9F685C00F943AA82B013C0131E9A32E71
:1082200035E1B32EA3019201F50165817681878145
:1082300090850F942EB6D50115966D937D938D93F1
:108240009C931897A701960119966D917D918D9138
:108250009C911C970F942EB6F501618772878387D6
:108260009487FCE1AF0EB11C8A149B04D9F657C069
:108270000F943AA82B013C0122E9A22E25E1B22E4F
:10828000A3019201D5015C966D917D918D919C9198
:108290005F970F942EB6F501648F758F868F978F39
:1082A000A701960160817181828193810F942EB61E
:1082B000D5016D937D938D939D935D01BEE9AB16C2
:1082C000B5E1BB06E9F62BC00F943AA82B013C019F
:1082D0009EEAA92E95E1B92EA3019201F5016081D4
:1082E0007181828193810F942EB6D5016D937D9318
:1082F0008D939D935D01A701960158966D917D9197
:108300008D919C915B970F942EB6F501608F718FC4
:10831000828F938FFAEBAF16F5E1BF06E9F61F5F88
:10832000143009F0C1CE0F94A06081E080939115C4
:108330000F94450DE091060D24E0E29FF001112419
:10834000EF5DFF4E20E030E04FE253E46081718149
:10835000828193810F9479B8181684F4809117075D
:10836000882361F00F94E768882341F080910A0D1B
:1083700090910B0DC29714F00C94FB6B81E090E090
:10838000909326028093250286E494E10F94184A84
:1083900028964EAD5FAD289750931F0E40931E0E4A
:1083A0002C968EAD9FAD2C979093F40E8093F30E88
:1083B0001092370E34C180919115882309F495C02D
:1083C000EFEFFFE084918F01882339F00F94B976A5
:1083D0000F5F1F4FF8018491F7CF67E070E080E0F6
:1083E00090E00F94546CEDEFFFE084918F018823AF
:1083F00039F00F94B9760F5F1F4FF8018491F7CFD2
:1084000067E070E080E090E00F94546CEAEEFFE0EB
:1084100084918F01882339F00F94B9760F5F1F4F35
:10842000F8018491F7CF65E070E080E090E00F9470
:10843000546CE8EDFFE084918F01882339F00F94AC
:10844000B9760F5F1F4FF8018491F7CF8AE00F9440
:10845000B97600E010E0B5ED6B2EBFE07B2E83ED2A
:10846000A82E8FE0B82EE12CF12C4801F8EA8F0EEF
:10847000911CF3018491A5EDCA2EAFE0DA2E88237A
:1084800041F00F94B976FFEFCF1ADF0AF60184911D
:10849000F6CFF401EE0DFF1DEF56FA4E61817281A9
:1084A0008381948145E00F943E77F4E0EF0EF11C58
:1084B0002CE1E216F104E9F6F5018491F3EDEF2EDB
:1084C000FFE0FF2E882341F00F94B976FFEFEF1AFB
:1084D000FF0AF7018491F6CF0C5111090C33FFEF1D
:1084E0001F0709F0C0CF0C94A56BE5EBFFE084916A
:1084F0008F01882311F40C94326A0F94B9760F5FC0
:108500001F4FF8018491F5CF86EE0F94F1680C941B
:10851000A56B1092FE0E0C94A56B85E40F9448A7F2
:10852000811102C00F94F98867EF662E62E0762E03
:108530007CE3A72E70E1B72EE8ED8E2EE0E19E2EB3
:10854000D12CD3018D913D010F9448A78823C9F107
:10855000B3E0DB120CC00F9440A7F5016083718378
:108560008283938388E490E10E945FB52AC00F94D0
:1085700040A79B01AC01D4016D917D918D919C919F
:108580000F942EB6F5016083718382839383E0900C
:108590004410F09045100091461010914710209122
:1085A0004010309141104091421050914310609121
:1085B0003C1070913D1080913E1090913F100F94AF
:1085C0004D59D394F4E0AF0EB11C24E0820E911CFF
:1085D00034E0D312B6CF0C94A56B81E08093A90F41
:1085E0000F94FB4560937F167093801680938116DD
:1085F000909382166091A90F84EC9FE00F94B4B51C
:1086000061E377E081EC9FE00E94D9C81092200ED0
:1086100060E08FEF9FE00F94B4B50C94A56B82E0FF
:108620000F9417120C94A56B80918C1590918D1559
:108630008E559C4E9F938F9380EA9FE00C94EE336F
:108640008DE40F9448A7882311F40C94F968E09105
:10865000100DF091110D319681918032E9F389303E
:10866000D9F380538A3060F080918C1590918D15EC
:108670008E559C4E9F938F938BE89FE00C94EE3326
:108680000F9440A70F948DB7AB01BC01CA01509362
:108690003B0D40933A0D4937510511F40C94285184
:1086A0000CF0DDC04F32510509F4B7C60CF061C0C3
:1086B0004931510509F45EC33CF54431510509F4D3
:1086C000C0C294F44131510509F4B1C234F44230CE
:1086D000510508F4F9C10C94E2684231510511F4D6
:1086E0000C941D4E0C94E2684631510509F4EDC21C
:1086F0000CF4E7C24731510509F4EDC24831510588
:1087000009F401C30C94E2684E31510509F468C4C0
:108710008CF44B31510509F448C30CF438C34C3187
:10872000510509F431C44D31510511F40C94F4682C
:108730000C94E2684A32510509F419C654F44F31D9
:10874000510509F4B9C54032510509F41AC50C9414
:10875000E2684C32510509F451C64D32510511F011
:108760000C94E2688AE50F9448A70E94A1700C94CB
:10877000F4684936510509F42AC7A4F54435510572
:1087800011F40C941D4EDCF44135510511F40C9498
:10879000FF4D34F44934510509F487C60C94E2685E
:1087A0004235510511F40C94194E4335510511F021
:1087B0000C94E26881E080933F0D0C94F468463598
:1087C000510511F40C947F4E14F40C94644E4C3506
:1087D000510511F40C949E4E4836510509F4C2C659
:1087E0000C94E2684037510509F4DBC6A4F44B361B
:1087F000510511F40C94F94D14F40C94C94D4D36F7
:10880000510511F40C94064C4E36510511F40C949C
:10881000224F0C94E2684337510511F40C94724FC7
:1088200084F44137510511F40C94354F423751050A
:1088300011F00C94E268E9EEFCE084918F010C9455
:108840004B504737510511F40C942D5148375105C1
:1088500011F00C94E268109224020C94F4688E35A6
:1088600041E0940711F40C9428680CF07FC0803D1F
:10887000910511F40C949E54CCF58B3C910511F4A8
:108880000C94FB52FCF48E3B910511F40C94A04C1B
:1088900034F48C38910509F489C60C94E268883C5C
:1088A000910511F40C944A52893C910511F00C94F5
:1088B000E26847EFE42E42E0F42E00E810E1D12C0C
:1088C0000C94B6528D3C910511F40C94995314F408
:1088D0000C9454538E3C910511F40C9448548F3CE5
:1088E000910511F40C9467540C94E268803F910553
:1088F00011F40C94F468CCF48C3D910511F40C94B3
:108900001B553CF4813D910511F40C94C6540C9414
:10891000E2688D3D910511F40C944655823E910517
:1089200011F40C9467550C94E2688E3261E096075E
:1089300011F40C9456576CF48C32B1E09B0711F48F
:108940000C94CA558D32914011F40C9402560C943B
:10895000E2688F32F1E09F0711F40C946B5780337B
:10896000914011F40C94BE560C94E2688A3532E0C2
:10897000930711F40C94B5630CF049C0853F51E0A6
:10898000950711F40C94795BECF48039A1E09A0717
:1089900011F40C94315B3CF48F35914011F40C943C
:1089A000F4680C94E2688339F1E09F0711F40C94A9
:1089B000355B843F914011F00C94E2680F94AC79E0
:1089C0000C94F4688D3F31E0930711F40C94395EF8
:1089D0006CF4863F51E0950711F40C947D5B873F62
:1089E000914011F40C94815B0C94E2688835A2E00C
:1089F0009A0711F40C94145F8935924011F00C948D
:108A0000E2680E9430E20F941F8F0C94F4688D3559
:108A1000E3E09E0711F40C948964DCF48E3B22E0C1
:108A2000920711F40C94D1683CF48D3B924011F400
:108A30000C94C5680C94E268833553E0950711F4F3
:108A40000C94555E8C35934011F40C94B8630C94DF
:108A5000E2688C38A3E09A0711F40C94F46894F45B
:108A60008438E3E09E0711F40C94A5668B3893409C
:108A700011F00C94E26807EFA02E02E0B02E00E0A7
:108A80000C940868803A23E0920709F4E6C3873E15
:108A9000934011F00C94E26810923F0F1092F30F84
:108AA0008091070F9091080FA091090FB0910A0FC4
:108AB0008093120D9093130DA093140DB093150D88
:108AC0000F94D80C0C94F468E091100DF091110DF6
:108AD0008F010E5F1F4F80E50F9448A7882371F028
:108AE0000F9440A70F9493B76B017C01AA24A39421
:108AF000672B682B692B31F4A12C04C0A12CC12C4D
:108B0000D12C760183E50F9448A7882391F00F9428
:108B100040A720E030E04AE754E40F943AA80F94CD
:108B200093B76B017C01BB24B394672B682B692B33
:108B300009F4B12C6AE270E0C8010F9473BB00978E
:108B400011F0DC011C92F801CF0121912032E1F3F8
:108B5000A11007C0B11005C0222319F00F94844B57
:108B600004C086EA92E10F94184A81E08093250EB2
:108B70001092240E0F94F9880F94FB456093030F15
:108B80007093040F8093050F9093060FC114D104C6
:108B9000E104F10419F10F94FB45C60ED71EE81E3F
:108BA000F91E84E090E090932602809325020F94B2
:108BB000FB456C157D058E059F0510F00C943D6CF2
:108BC0000F94EF1281110C943D6C0F94AA8381E0F5
:108BD0000F94730880E00F941712E9CF84E090E0BF
:108BE00090932602809325020F94EF12811109C001
:108BF0000F94AA8381E00F94730880E00F941712FA
:108C0000F3CF82E090E0909326028093250280913A
:108C10008516882331F089EF98E30F94184A0C9455
:108C2000F46886E494E10F94184A0C94F4688DE992
:108C300092E10F94184A17981698159814980C9466
:108C4000F468EDE3F6E084918F01882339F00F9406
:108C5000B9760F5F1F4FF8018491F7CF8AE00F9428
:108C6000B976109266191092651989ED96E10E9405
:108C700077E68BE1E9EDF6E1DE01119601900D92C8
:108C80008A95E1F740E050E0BE016F5F7F4F86E0DC
:108C900094E00F946681CE0101960F941467EFE281
:108CA000F6E084918F01882339F00F94B9760F5F35
:108CB0001F4FF8018491F7CF8AE00F94B9760C9496
:108CC000F4680F94642B0C94F4681092851610923B
:108CD00086160C94F4688091100D9091110D6AE243
:108CE00070E004960F9473BB009711F0DC011C92A6
:108CF0008091100D9091110D41E061E004960F9468
:108D00008E260C94F4688091871681111EC060E055
:108D100086E69FE00F94B4B560E088E69FE00F948C
:108D2000B4B560E085E69FE00F94B4B560E084E6FA
:108D30009FE00F94B4B560E082ED9EE00F94B4B56F
:108D400060E08FEC9EE00F94B4B580918616882386
:108D500029F081E080938516109287160F94FB45C9
:108D600060932E0E70932F0E8093300E9093310EE1
:108D70000C94F46880918516882311F40C94F4689F
:108D80001092851681E0809387160C94F468809188
:108D90008616882311F40C94F46883E50F9448A791
:108DA00081110C94496C0C94F46880918516882389
:108DB00009F4B8C001EA16E1F80181918F01882316
:108DC00019F00F94B976F8CFE6E6FDE084918F01B3
:108DD000882339F00F94B9760F5F1F4FF801849103
:108DE000F7CFE1E1F5E084918F01882339F00F940A
:108DF000B9760F5F1F4FF8018491F7CF609160192A
:108E00007091611980916219909163194AE00F94F1
:108E1000CD76E4E6FDE084918F01882339F00F944C
:108E2000B9760F5F1F4FF8018491F7CF6091581901
:108E30007091591980915A1990915B194AE00F94D9
:108E4000CD768AE00F94B9760F94FB4540E6C42EA8
:108E50004AEED42EE12CF12CA70196010F94F2B525
:108E600049015A0160912E0E70912F0E8091300EA3
:108E70009091310EA70196010F94F2B58401021B67
:108E8000130BC8016CE370E00F94CDBACB019927A6
:108E9000EAE0F0E0BF010F94E1BA282FCB01BF0157
:108EA0000F94E1BA805D8093B419205D2093B519C9
:108EB0001092B61954EBE52E59E1F52E6701D60153
:108EC0008D916D01882319F00F94B976F8CF8AE35C
:108ED0000F94B976C8016CE370E00F94CDBA6AE0E4
:108EE00070E00F94E1BA605D6093B419805D809387
:108EF000B5191092B619F70181917F01882319F0F5
:108F00000F94B976F8CFE2E6FDE084918F018823D3
:108F100011F40C94F4680F94B9760F5F1F4FF801A9
:108F20008491F5CF80918716882371F0E2E5FDE00A
:108F300084918F01882309F4BFCE0F94B9760F5F17
:108F40001F4FF8018491F6CF8091390E882371F07C
:108F5000E6E4FDE084918F01882309F4ADCE0F94FF
:108F6000B9760F5F1F4FF8018491F6CFE6E3FDE07D
:108F700084918F01882309F49FCE0F94B9760F5FF7
:108F80001F4FF8018491F6CF8091100D9091110D33
:108F90006AE270E004960F9473BB8C01892BA9F0F0
:108FA00080918C1590918D156EE470E08E559C4EDD
:108FB0000F9473BB60E270E00F9473BB01969093C3
:108FC000110D8093100DD8011C928091100D90917D
:108FD000110D41E060E004960F948E260C94F46825
:108FE00080918616882311F40C94F4680F94CA5665
:108FF0008091100D9091110D6AE270E004960F942B
:1090000073BB8C01892BA9F080918C1590918D15E3
:109010006EE470E08E559C4E0F9473BB60E270E07E
:109020000F9473BB01969093110D8093100DF8016E
:109030001082C090100DD090110D86010C5F1F4F53
:1090400080918616882311F40C94F4688BEA98E1D9
:109050000E949DE9109285161F8E1AA289ED96E155
:109060009093F5168093F4160115110591F0D60131
:1090700014968C918F3239F4BE01615E7F4FC80126
:109080000F94BE5806C086EF96E19093F516809334
:10909000F4166091F4167091F51619821C8222E084
:1090A000A801CE0101960E9464EB8823A1F0CE01B5
:1090B00001960F94D480882371F061E0CE0101966F
:1090C0000E941EE9009739F025EEFC0120831C82E6
:1090D0000E94A2E3F82ECE0101960F941467FF20A0
:1090E00021F1E8E2FDE084917F01882341F00F94B3
:1090F000B976FFEFEF1AFF0AF7018491F6CFD80196
:109100008D918D01882319F00F94B976F8CF8AE0FC
:109110000F94B97610926019109261191092621929
:10912000109263190F94512926C0E0E1FDE084916B
:109130007F01882341F00F94B976BFEFEB1AFB0A49
:10914000F7018491F6CFD8018D918D01882319F014
:109150000F94B976F8CFEEE0FDE084918F0188237B
:1091600039F00F94B9760F5F1F4FF8018491F7CF54
:109170008AE00F94B976CE014F960F9414670C9441
:10918000F4688091851681110F94F9880091100D73
:109190001091110D0C5F1F4F6AE270E0C8010F942F
:1091A00073BB7C0161E270E0C8010F9473BB009750
:1091B00019F08C010F5F1F4FE114F10411F0D7017A
:1091C0001C9280E50F9448A7F82E8091100D909185
:1091D000110D0817190708F4F12C809186168823C1
:1091E00011F40C94F46841E04F2561E0C8010F943C
:1091F0008E2683E50F9448A78823B9F08091100D3F
:109200009091110D8017910780F40F9436A7AB0150
:10921000BC01409360195093611960936219709377
:1092200063198BEA98E10E94E1E580918616882314
:1092300029F081E08093851610928716F1100C9426
:10924000F4680F94FB4560932E0E70932F0E80935D
:10925000300E9093310E0C94F4688091100D909123
:10926000110D6AE270E005960F9473BB8C01892B97
:10927000A9F080918C1590918D156EE470E08E555B
:109280009C4E0F9473BB60E270E00F9473BB019629
:109290009093110D8093100DF80110828091100DA4
:1092A0009091110D21E02093841641E060E0059635
:1092B0000F948E260C94F4680F94FB4500912E0EAB
:1092C00010912F0E2091300E3091310E6B017C01E8
:1092D000C01AD10AE20AF30AC701B60128EE33E048
:1092E00040E050E00F94F2B5CA01B9012CE330E040
:1092F00040E050E00F94F2B57F936F93C701B60141
:1093000020E63AEE40E050E00F94F2B53F932F9301
:109310008CE79FE09F938F938E010F5F1F4F1F93EA
:109320000F930F9406ADE7E8FEE584910FB6F8942D
:10933000DEBF0FBECDBF7F01882341F00F94B97609
:109340003FEFE31AF30AF7018491F6CF7801D701D2
:109350008D917D01882319F00F94B976F8CF8AE0BA
:109360000F94B976C8010F94844B0C94F46883E58C
:109370000F9448A7882311F40C94F4680F9440A725
:109380000F948DB7F62EE72E862F9E2D8C0180E54B
:109390000F9448A7882331F00F3F110509F010F40E
:1093A0000C945A6C0DE010E0EDE8F2E0819191919F
:1093B0008017910711F40C94F468B2E0E53CFB07C8
:1093C000A9F70630110539F48F2D9E2D9093BD1904
:1093D0008093BC1904C017FF02C00C94F46861E0CC
:1093E000802F0F94C0446F2D802F0F94F0436F2D6A
:1093F0007E2D802F0F94FC440C94F4688FEF0F9413
:10940000F16860E070E088EF9FE00F94CEB50F94B4
:109410009D0F0F947F0F0C94F46884E090E090937C
:109420002602809325020F94A1190E94D1870F94E0
:10943000AA8381E00F94730860E080E00F94F21437
:109440008FEF9CE00F94191461E080E00F94F21408
:109450001E9903C089EF9CE002C08CEF9CE00F9442
:10946000191462E080E00F94F2141D9903C083EF99
:109470009CE002C086EF9CE00F94191463E080E04A
:109480000F94F2141C9903C08DEE9CE002C080EF93
:109490009CE00F9419140F94EF12882341F20F945B
:1094A000A1190F94238E0C94F46880E50F9448A7BB
:1094B000882331F00F9440A70F9493B76093530221
:1094C00082E50F9448A7882341F00F9440A70F949A
:1094D00093B7709359026093580281E50F9448A79F
:1094E000882331F00F9440A70F9493B760935202F2
:1094F00083E50F9448A7882341F00F9440A70F9469
:1095000093B77093570260935602809159028F93DC
:10951000809158028F93809153021F928F938BEE0C
:1095200095E09F938F9302EF15E01F930F930F9495
:10953000AEAC809157028F93809156028F938091A9
:1095400052021F928F9384EE95E09F938F931F9307
:109550000F930F94AEAC0FB6F894DEBF0FBECDBF25
:109560000C94F468BE016F5F7F4F88E690E00F9423
:109570009CA381110C94F46883E50F9448A7882379
:1095800011F40C94F46819810F9440A711110C94F4
:10959000F4680F948DB770938F1560938E150C94AB
:1095A000F46863E083EE95E00F94140883E50F946C
:1095B00048A7882311F40C94F4680F9440A70F94E3
:1095C0008DB770930B0D60930A0D0C94F468BE0177
:1095D0006F5F7F4F89E690E00F949CA381110C94FC
:1095E000F468E6E7FFE084918F01882339F00F9457
:1095F000B9760F5F1F4FF8018491F7CFE98124E01E
:10960000E29FF0011124EF5DFF4E60817181828144
:10961000938141E00F943E77E3E7FFE084918F016F
:10962000882339F00F94B9760F5F1F4FF8018491AA
:10963000F7CFE981F0E0EE0FFF1FE257FA4E6081AD
:109640007181072E000C880B990B0F9448AD41E0F7
:109650000F943E77EFE6FFE084918F01882339F085
:109660000F94B9760F5F1F4FF8018491F7CF609187
:10967000100770911107809112079091130741E034
:109680000F943E77ECE6FFE084918F01882339F058
:109690000F94B9760F5F1F4FF8018491F7CF609157
:1096A0000A0D70910B0D072E000C880B990B0F946F
:1096B00048AD41E00F943E77E9E6FFE084918F01E9
:1096C000882339F00F94B9760F5F1F4FF80184910A
:1096D000F7CF60E070E0CB010F94546CE7E6FFE059
:1096E00084918F01882339F00F94B9760F5F1F4F53
:1096F000F8018491F7CF6091211070912210809130
:1097000023109091241041E00F943E77E4E6FFE0AF
:1097100084918F01882339F00F94B9760F5F1F4F22
:10972000F8018491F7CF60918E1570918F15072EF7
:10973000000C880B990B0F9448AD41E00F943E77D5
:10974000E0E6FFE084918F01882339F00F94B97629
:109750000F5F1F4FF8018491F7CFE981F0E0E35CE0
:10976000F04F608170E080E090E00F94546CEBE586
:10977000FFE084918F01882339F00F94B9760F5F51
:109780001F4FF8018491F7CF60913C0F70E080E0AB
:1097900090E00F94546CE7E5FFE084918F018823FB
:1097A00039F00F94B9760F5F1F4FF8018491F7CF0E
:1097B00060915D0E70915E0E80915F0E9091600ED3
:1097C00041E00F943E77E3E5FFE084918F01882329
:1097D00039F00F94B9760F5F1F4FF8018491F7CFDE
:1097E0006091590E70915A0E80915B0E90915C0EB3
:1097F00041E00F943E778AE00F94B97681E090E0E3
:1098000090932602809325020C948770BE016F5FAF
:109810007F4F8DE690E00F949CA381110C94F46827
:109820008FE399E40F94184A81E090E09093DB0E67
:109830008093DA0E8091A90F882329F060E081E0FF
:1098400090E00E94ADDA83E50F9448A7882379F071
:1098500019810F9440A7111106C00F948DB7709312
:109860008F1560938E1581E08093060212C082E509
:109870000F9448A7882369F019810F9440A711110C
:1098800006C00F948DB770938F1560938E1510924C
:1098900006020F94FB454B015C01F9800F2D10E08F
:1098A000F801EE0FFF1FE257FA4E60817181072E1B
:1098B000000C880B990B0F9448ADF801EE0FFF1FB9
:1098C000EE0FFF1FEF5DFF4E11E0208131814281DD
:1098D00053810F9479B818160CF010E010930B0F09
:1098E00081E090E090932602809325021092380E3A
:1098F0004F2DC501B4010F94660B81E399E40F94D9
:10990000184A82E090E0909326028093250290937B
:10991000DB0E8093DA0E8091A90F882329F060E096
:1099200082E090E00E94ADDA0F94FB456093030F54
:109930007093040F8093050F9093060F0C94F468B6
:1099400085E299E40F94184A83E090E09093DB0E4F
:109950008093DA0E8091A90F882329F060E081E0DE
:1099600090E00E94ADDA83E50F9448A7882361F068
:109970000F9440A70F948DB770930B0D60930A0D51
:1099800081E0809306020FC082E50F9448A78823E8
:1099900051F00F9440A70F948DB770930B0D609307
:1099A0000A0D109206020F94FB454B015C011092C8
:1099B000380E60910A0D70910B0D072E000C880B6C
:1099C000990B0F9448AD11E02091100730911107C9
:1099D00040911207509113070F9479B818160CF0A4
:1099E00010E010930B0F81E090E09093260280939B
:1099F000250200E51FE0BCE4EB2EBFE0FB2E88E46F
:109A0000C82E8FE0D82E80910B0F60910A0D7091B7
:109A10000B0D8823B9F08091380E811113C0072EE9
:109A2000000C880B990B0F9448AD209110073091D2
:109A3000110740911207509113070F9479B8181627
:109A4000BCF08BC0072E000C880B990B0F9448AD0F
:109A50002091100730911107409112075091130780
:109A60000F9442AD87FF79C080910602811175C0C5
:109A70000F94FB45DC01CB0188199909AA09BB09A0
:109A8000893E9340A105B10508F45EC08091A90FFD
:109A9000811156C0E091060D24E0E29FF0011124EF
:109AA000EF5DFF4E4080518062807380F8018491A9
:109AB000A0E5AA2EAFE0BA2E882341F00F94B97624
:109AC000FFEFAF1ABF0AF5018491F6CF42E0C30160
:109AD000B2010F943E77F7018491FCE4AF2EFFE0D2
:109AE000BF2E882341F00F94B976FFEFAF1ABF0A5B
:109AF000F5018491F6CF6091060D70E080E090E072
:109B00000F94546CF6018491E8E4AE2EEFE0BE2E83
:109B1000882341F00F94B976FFEFAF1ABF0AF50121
:109B20008491F6CF60911007709111078091120710
:109B30009091130741E00F943E778AE00F94B97635
:109B40000F94FB454B015C010F94AA8380E00F94B6
:109B5000730880E00F94171256CF8CE199E40F94AC
:109B6000184A82E090E0909326028093250284E0D8
:109B700090E09093DB0E8093DA0E0F94FB45609398
:109B8000030F7093040F8093050F9093060F0C94AE
:109B9000F46883E50F9448A7882319F10F9440A730
:109BA00020E030E0A9010F9442AD87FD0FC00F9473
:109BB00040A720E030E04FE753E40F9479B818163F
:109BC00044F00F9440A70F948DB705C060E070E09B
:109BD00002C06FEF70E07093BD196093BC190C94D4
:109BE000F4688FEF90E09093BD198093BC190C94AA
:109BF000F4681092BD191092BC190C94F4680F947B
:109C00002A1D0F94F988149A0F9452891092BD1945
:109C10001092BC1968EE73E080E090E00F94C345A9
:109C200087E094E00F94184A80E00F9417120C9488
:109C3000F46810923F0D0C94F46883E50F9448A7E4
:109C4000882399F00F9440A720E030E04AE754E4DD
:109C50000F943AA80F9493B76093770270937802A9
:109C60008093790290937A021DC088E50F9448A7EB
:109C700081110C94616C89E50F9448A781110C94B3
:109C8000616C8AE50F9448A781110C94616C85E49E
:109C90000F9448A781110C94616C0F94F988149A61
:109CA0000F9452898FEF9FEF90935902809358023F
:109CB00090935702809356028093530280935202EE
:109CC0001092400D0C94F46883E50F9448A7882304
:109CD00011F40C94F4680F9440A720E030E04AE7B8
:109CE00054E40F943AA80F9493B76093FF0E7093C7
:109CF000000F8093010F9093020F0C94F46883E59A
:109D00000F9448A7882311F40C94F4680F9440A78B
:109D100020E030E04AE754E40F943AA80F9493B758
:109D2000609373027093740280937502909376022D
:109D30008EE696E10E9411E30C94F46827EF32E07E
:109D40003BAF2AAF00E810E172E5C72E7DE0D72EC9
:109D5000F12CAAADBBAD8D91BBAFAAAF0F9448A7B4
:109D6000882309F463C0B3E0FB1259C00F9440A7E5
:109D70002B013C0120E030E040EA51E40F9442AD79
:109D800087FF45C0A3019201F80164817581868136
:109D900097810F941CB74B015C019B01AC01609152
:109DA000D4107091D5108091D6109091D7100F9447
:109DB0003AA86093D4107093D5108093D6109093E6
:109DC000D71020902B0230902C02A5019401D101D4
:109DD0001C966D917D918D919C911F970F943AA83F
:109DE000F1016487758786879787D6016D917D918C
:109DF0008D919C910F9446ADA50194010F943AA8C2
:109E00000F9493B7F6016083718382839383D801A3
:109E100014964D925D926D927C92179707C00F94A5
:109E200040A7F8016483758386839783F3940C5F5E
:109E30001F4FF4E0CF0ED11C64E0862EF81089CFBE
:109E40000C94F4688EE40F9448A7882311F40C94C2
:109E5000F4680F9436A76093120D7093130D8093DE
:109E6000140D9093150D0C94F46883E50F9448A796
:109E7000882379F08091100D9091110D4AE050E007
:109E800060E070E001960F9462AA609346020C9421
:109E9000F468E7E8FEE584918F01882339F00F9498
:109EA000B9760F5F1F4FF8018491F7CFC09046023B
:109EB000D12CE12CF12CE1E4FFE084918F01882387
:109EC00039F00F94B9760F5F1F4FF8018491F7CFE7
:109ED0004AE0C701B6010F94CD768AE00F94B976B7
:109EE0000C94F46886E50F9448A7882379F0E3EB97
:109EF000FAE584918F01882311F40C945C460F9449
:109F0000B9760F5F1F4FF8018491F5CF85E50F9467
:109F100048A7382E8823D9F1E090100DF090110D4C
:109F2000FFEFEF1AFF0AF092110DE092100D2701DA
:109F300067014601D6018D916D0190ED980F9A3021
:109F4000C0F38E3211F00C94F4685D013501F50117
:109F500081915F0190ED980F9A30C0F38E3211F02D
:109F60000C94F468CF018C01DC012C90019620ED5B
:109F7000220D2A30C0F3822D0F94EE4981110C94EA
:109F8000806CBDE22B120C94F4680C94806CE3E2BC
:109F9000FFE084918F01882339F00F94B9760F5F29
:109FA0001F4FF8018491F7CFE3EBFAE584918F011D
:109FB000882339F00F94B9760F5F1F4FF801849111
:109FC000F7CFE9ECFEE084918F01882339F00F94FC
:109FD000B9760F5F1F4FF8018491F7CFE5ECFEE0F3
:109FE00084918F01882339F00F94B9760F5F1F4F4A
:109FF000F8018491F7CFE6EBFEE084918F0188238E
:10A0000039F00F94B9760F5F1F4FF8018491F7CFA5
:10A01000E9EAFEE084918F01882339F00F94B97644
:10A020000F5F1F4FF8018491F7CFE8E9FEE08491BC
:10A030008F01882339F00F94B9760F5F1F4FF80115
:10A040008491F7CFE6E9FEE084918F01882339F00F
:10A050000F94B9760F5F1F4FF8018491F7CFEFE8A7
:10A06000FEE084918F01882339F00F94B9760F5F59
:10A070001F4FF8018491F7CFEAE6FEE084918F014B
:10A08000882311F40C945C460F94B9760F5F1F4F30
:10A09000F8018491F5CF882339F00F94B9760F5FDA
:10A0A0001F4FF8018491F7CF60913C1070913D10E3
:10A0B00080913E1090913F1042E00F943E77E5EE84
:10A0C000FCE084918F01882339F00F94B9760F5FFB
:10A0D0001F4FF8018491F7CF6091401070914110AB
:10A0E000809142109091431042E00F943E77E1EE50
:10A0F000FCE084918F01882339F00F94B9760F5FCB
:10A100001F4FF8018491F7CF609144107091451072
:10A11000809146109091471042E00F943E77EDED0C
:10A12000FCE084918F01882339F00F94B9760F5F9A
:10A130001F4FF8018491F7CF60914810709149103A
:10A1400080914A1090914B1042E00F943E77E6E0E8
:10A15000F5E084918F01882339F00F94B9760F5F71
:10A160001F4FF8018491F7CF80E00F94D8880F94A7
:10A1700048AD209184103091851040918610509107
:10A1800087100F941CB742E00F943E77E9EDFCE096
:10A1900084918F01882339F00F94B9760F5F1F4F98
:10A1A000F8018491F7CF81E00F94D8880F9448ADDF
:10A1B000209188103091891040918A1050918B1015
:10A1C0000F941CB742E00F943E77E5EDFCE08491DC
:10A1D0008F01882339F00F94B9760F5F1F4FF80174
:10A1E0008491F7CF82E00F94D8880F9448AD2091E6
:10A1F0008C1030918D1040918E1050918F100F94D3
:10A200001CB742E00F943E77E1EDFCE084918F01B2
:10A21000882339F00F94B9760F5F1F4FF8018491AE
:10A22000F7CF83E00F94D8880F9448AD2091901019
:10A230003091911040919210509193100F941CB74F
:10A2400042E00F943E778AE00F94B9760C94F4685C
:10A2500081E0809324020C94F468EAECF5E08491A8
:10A260008F01882339F00F94B9760F5F1F4FF801E3
:10A270008491F7CF8AE00F94B976E2ECF5E084910F
:10A280008F01882339F00F94B9760F5F1F4FF801C3
:10A290008491F7CF1E9B0DC0E8EBF5E084918F0110
:10A2A0008823A1F00F94B9760F5F1F4FF8018491B6
:10A2B000F7CFE3EBF5E084918F01882339F00F9419
:10A2C000B9760F5F1F4FF8018491F7CF8AE00F94A2
:10A2D000B976EBEAF5E084918F01882339F00F9489
:10A2E000B9760F5F1F4FF8018491F7CF8091060177
:10A2F00082FF0DC0E8EBF5E084918F018823A1F087
:10A300000F94B9760F5F1F4FF8018491F7CFE3EBFD
:10A31000F5E084918F01882339F00F94B9760F5FAF
:10A320001F4FF8018491F7CF8AE00F94B976E3EAE2
:10A33000F5E084918F01882339F00F94B9760F5F8F
:10A340001F4FF8018491F7CF1D9B0DC0E8EBF5E09E
:10A3500084918F018823A1F00F94B9760F5F1F4F6E
:10A36000F8018491F7CFE3EBF5E084918F01882326
:10A3700039F00F94B9760F5F1F4FF8018491F7CF32
:10A380008AE00F94B976EBE9F5E084918F01882398
:10A3900039F00F94B9760F5F1F4FF8018491F7CF12
:10A3A0008091060187FF0DC0E8EBF5E084918F01F5
:10A3B0008823A1F00F94B9760F5F1F4FF8018491A5
:10A3C000F7CFE3EBF5E084918F01882339F00F9408
:10A3D000B9760F5F1F4FF8018491F7CF8AE00F9491
:10A3E000B976E3E9F5E084918F01882339F00F9481
:10A3F000B9760F5F1F4FF8018491F7CF1C9B0DC0FA
:10A40000E8EBF5E084918F018823A1F00F94B976F1
:10A410000F5F1F4FF8018491F7CFE3EBF5E08491D4
:10A420008F01882339F00F94B9760F5F1F4FF80121
:10A430008491F7CF8AE00F94B976EBE8F5E0849148
:10A440008F01882339F00F94B9760F5F1F4FF80101
:10A450008491F7CF01990FC0E8EBF5E084918F016B
:10A46000882311F40C945C460F94B9760F5F1F4F4C
:10A47000F8018491F5CFE3EBF5E084918F01882317
:10A4800011F40C945C460F94B9760F5F1F4FF801DE
:10A490008491F5CF1091060D84E50F9448A7882389
:10A4A00001F10F9440A70F9493B7162F6623C9F0BC
:10A4B000E7E8FEE584918F01882339F00F94B9769F
:10A4C0000F5F1F4FF8018491F7CF04E715E0D80123
:10A4D0008D918D01882311F40C94F4680F94B97652
:10A4E000F6CF84E40F9448A7882311F40C94F46801
:10A4F0000F9440A720E030E0A9010F9442AD8111F4
:10A5000003C0109217112EC00F9440A7B4E01B9FF8
:10A51000F0011124E85EFE4E608371838283938391
:10A52000C0901811D0901911E0901A11F0901B11E1
:10A5300020E030E0A901C701B6010F9442AD8111BE
:10A5400006C0C12CD12C50EEE52E5FE3F52EC09253
:10A550001811D0921911E0921A11F0921B1181E09A
:10A56000809317110F94E4060C94F468F70181911D
:10A570007F010F9448A78823A1F10F9440A70F945F
:10A5800093B7F1E0FD15ACF0653C29E07207810559
:10A590009105A0F4562F472F382F292F613CA3E0B7
:10A5A0007A078105910590F050EC43E030E020E01F
:10A5B0000DC0562F472F382F292F08C050EC43E0ED
:10A5C00030E020E064EC79E080E090E0F80164A302
:10A5D00075A386A397A3E455FF4F5083418332832D
:10A5E0002383D3940C5F1F4FF4E0DF12BFCF0E9490
:10A5F00001B50C94F46827EFA22E22E0B22E30E8C9
:10A60000C32E30E1D32E912CD5018D915D010F9495
:10A6100048A7882309F43EC00F9440A77B018C0112
:10A62000B1E0B91514F120E030E048E453E40F94B0
:10A6300079B818163CF4512C612C88E4782E93E4F8
:10A64000892E04C05E2C6F2C702E812E20E030E00D
:10A6500048EC52E4B701C8010F9479B818164CF4CD
:10A66000E12CF12C08EC12E404C0562E6F2C782E4D
:10A67000812E852D962DA72DB82DF601848B958BD7
:10A68000A68BB78BC701D801E456FF4F8083918317
:10A69000A283B3839394F4E0CF0ED11C14E0812EF7
:10A6A0009810B2CF0C94F46883E50F9448A78823E0
:10A6B000E9F00F9440A76093B4107093B5108093A5
:10A6C000B6109093B71084E50F9448A7882311F42F
:10A6D0000C94F4680F9440A76093B8107093B9106D
:10A6E0008093BA109093BB100C94F46880E50F949B
:10A6F00048A7882351F00F9440A76093B41070933B
:10A70000B5108093B6109093B71082E50F9448A7C8
:10A71000882351F00F9440A76093B8107093B9103C
:10A720008093BA109093BB1084E50F9448A70C94C3
:10A73000F46883E50F9448A7882351F00F9440A74D
:10A740006093BC107093BD108093BE109093BF10A7
:10A7500084E50F9448A7882351F00F9440A7609395
:10A76000C0107093C1108093C2109093C31082E404
:10A770000F9448A7882361F00F9440A70F9493B7D4
:10A780006093C4107093C5108093C6109093C71047
:10A7900088E50F9448A7882391F00F9440A7609311
:10A7A000CC107093CD108093CE109093CF10609307
:10A7B000C8107093C9108093CA109093CB1089E58C
:10A7C0000F9448A7882351F00F9440A76093CC10B2
:10A7D0007093CD108093CE109093CF108AE50F9494
:10A7E00048A7882351F00F9440A76093D01070932E
:10A7F000D1108093D2109093D31085E40F9448A782
:10A80000882351F00F9440A76093D4107093D51013
:10A810008093D6109093D71020E030E040E251E4CE
:10A820006091C8107091C9108091CA109091CB109E
:10A830000F9479B8181664F480E090E0A0E2B1E4D7
:10A840008093C8109093C910A093CA10B093CB10F6
:10A8500020E030E040E251E46091CC107091CD10E6
:10A860008091CE109091CF100F9479B8181614F0F3
:10A870000C94F46880E090E0A0E2B1E48093CC1006
:10A880009093CD10A093CE10B093CF100C94F46899
:10A89000A7EFEA2EA2E0FA2E08ED10E1B4EECB2EDF
:10A8A000B0E1DB2ED7018D917D010F9448A788235D
:10A8B00039F00F9440A7F8016083718382839383FA
:10A8C0000C5F1F4FC016D10669F70C94F46883E53E
:10A8D0000F9448A7882351F00F9440A76093031169
:10A8E00070930411809305119093061186E40F94E0
:10A8F00048A7882381F00F9440A720E030E040E78C
:10A9000052E40F941CB76093071170930811809361
:10A91000091190930A118AE50F9448A7882311F42E
:10A920000C94F4680F9440A760930B1170930C1172
:10A9300080930D1190930E110C94F46883E50F949D
:10A9400048A7882351F00F9440A760930F1170938C
:10A950001011809311119093121186E40F9448A75F
:10A96000882311F40C94F4680F9440A720E030E0A1
:10A9700040E752E40F941CB76093131170931411C5
:10A9800080931511909316110C94F46883E50F943D
:10A9900048A7882311F40C94F4680F9440A70F94EF
:10A9A0008DB76115710551F06130710569F481E071
:10A9B000809302111092BA0F0C94F4681092021155
:10A9C0001092BA0F0C94F468E7E8FEE584918F01C9
:10A9D000882339F00F94B9760F5F1F4FF8018491E7
:10A9E000F7CFE1E6F5E084918F01882339F00F94E9
:10A9F000B9760F5F1F4FF8018491F7CF00918C1546
:10AA000010918D150E551C4ED8018D918D01882306
:10AA100019F00F94B976F8CFE5E6FEE084918F0146
:10AA2000882311F40C945C460F94B9760F5F1F4F86
:10AA3000F8018491F5CF82E40F9448A7882341F070
:10AA40008091330290913402909305028093040226
:10AA500083E50F9448A7882341F00F9440A70F94F3
:10AA60008DB7709334026093330282E50F9448A748
:10AA7000882311F40C94F4688091040290910502EB
:10AA800090933402809333020C94F46883E50F941E
:10AA900048A7882309F466CD0F9440A70F948DB77B
:10AAA0006B017C0184E50F9448A7882359F0BE010F
:10AAB0006F5F7F4F8DED90E00F949CA381110C94FC
:10AAC000F46850CDD0928102C09280024BCD80E5D7
:10AAD0000F9448A7882311F40C94F4680F9440A7AE
:10AAE0000F948DB7D62E862F972F7C0183E50F9478
:10AAF00048A7882331F00F9440A70F948DB78B019E
:10AB000002C00FEF1FEFC8010196039710F00C94DD
:10AB1000F468EDE8F2E085EC92E021913191E216E3
:10AB2000F30611F40C94F4688E179F07B1F7F7FE43
:10AB300002C00C94F4680F94F988FD2C60E08D2D10
:10AB40000F94C0440F3FFFEF1F0731F00130110594
:10AB500071F401E010E00DC08D2D0F94A9A631E035
:10AB600020E0892B09F030E0032F122F02C000E013
:10AB700010E08F2D0F94A9A68017910711F40C9463
:10AB8000F4680F94AA8380E00F94730880E00F9418
:10AB90001712EFCF83E50F9448A7882331F00F9465
:10ABA00040A70F948DB78B0102C00EE610E080E540
:10ABB0000F9448A7882329F00F9440A70F948DB7CE
:10ABC00002C068EE73E06B01770FEE08FF08101605
:10ABD000110694F48091090790910A07029718F4DE
:10ABE000C8010F94AB5DC701B6010F94C34584E55E
:10ABF0000F941E440C94F468C701B6010F94C3452A
:10AC00000C94F46880E50F9448A7882351F00F94C2
:10AC100040A76093E8107093E9108093EA10909336
:10AC2000EB1089E40F9448A7882381F00F9440A784
:10AC30002CEA35EC47E25EE30F943AA86093EC10FF
:10AC40007093ED108093EE109093EF1084E40F94C6
:10AC500048A7882381F00F9440A72CEA35EC47E2FF
:10AC60005EE30F941CB76093F0107093F110809323
:10AC7000F2109093F31083E40F9448A7882351F0C7
:10AC80000F9440A760930002709301028093020228
:10AC9000909303020F940788EDE6F7E184918F010A
:10ACA000882339F00F94B9760F5F1F4FF801849114
:10ACB000F7CF04E114E0D8018D918D01882319F0BC
:10ACC0000F94B976F8CF6091E8107091E9108091F7
:10ACD000EA109091EB1042E00F943E7708E114E007
:10ACE000F80181918F01882319F00F94B976F8CF7C
:10ACF0002CEA35EC47E25EE36091EC107091ED10C8
:10AD00008091EE109091EF100F941CB742E00F94D9
:10AD10003E770CE114E0D8018D918D01882319F064
:10AD20000F94B976F8CF2CEA35EC47E25EE36091F8
:10AD3000F0107091F1108091F2109091F3100F9437
:10AD40003AA842E00F943E7700E214E0F8018191C6
:10AD50008F01882319F00F94B976F8CF6091000223
:10AD600070910102809102029091030242E00F94DF
:10AD70003E778AE00F94B9760C94F46880E50F94DE
:10AD800048A7882351F00F9440A76093F410709364
:10AD9000F5108093F6109093F71089E40F9448A76C
:10ADA000882381F00F9440A72CEA35EC47E25EE35C
:10ADB0000F943AA86093F8107093F9108093FA10EA
:10ADC0009093FB1084E40F9448A7882381F00F949C
:10ADD00040A72CEA35EC47E25EE30F941CB7609382
:10ADE000FC107093FD108093FE109093FF100F9451
:10ADF0000788EDE6F7E184918F01882339F00F94FD
:10AE0000B9760F5F1F4FF8018491F7CF04E114E08A
:10AE1000D8018D918D01882319F00F94B976F8CF60
:10AE20006091F4107091F5108091F6109091F710E8
:10AE300042E00F943E7708E114E0F80181918F0120
:10AE4000882319F00F94B976F8CF2CEA35EC47E255
:10AE50005EE36091F8107091F9108091FA10909172
:10AE6000FB100F941CB742E00F943E770CE114E006
:10AE7000D8018D918D01882319F00F94B976F8CF00
:10AE80002CEA35EC47E25EE36091FC107091FD1016
:10AE90008091FE109091FF100F943AA842E00F9419
:10AEA0003E778AE00F94B9760C94F46883E50F94AA
:10AEB00048A7882319F00F9440A703C060E070E012
:10AEC000CB016093820270938302809384029093FB
:10AED00085020C94F46885E40F9448A7882359F000
:10AEE0000F9440A70F948DB724967FAF6EAF249731
:10AEF00077FF05C013C024961FAE1EAE249763963D
:10AF00001FAE639765961FAE659726E167962FAFD4
:10AF1000679733E468963FAF68970EC063961FAE9D
:10AF2000639765961FAE65974CE867964FAF679736
:10AF300052E468965FAF689783E50F9448A788232B
:10AF400071F00F9440A763966FAF639765967FAFDC
:10AF5000659767968FAF679768969FAF689783E40A
:10AF60000F9448A7882349F00F9440A70F948DB7FA
:10AF7000A6967FAF6EAFA69706C085E090E0A69636
:10AF80009FAF8EAFA697A6968EAC9FACA6979092D9
:10AF9000D70E8092D60E1092F20E1092D90E109209
:10AFA000D80E0F94FB4562966CAF7DAF8EAF9FAF0E
:10AFB00062972496AEACBFAC2497B7FC05C02AE0DC
:10AFC000A7962FAFA79704C03DE2A7963FAFA797DC
:10AFD0000F94FB45E3966CAF7DAF8EAF9FAFE397C9
:10AFE00024968EAC9FAC249718141904B4F404E290
:10AFF00014E0D8018D918D01882319F00F94B97652
:10B00000F8CF8AE00F94B97681E08093F20E109227
:10B01000D90E1092D80E0C94F4680EE414E0F801E6
:10B0200081918F01882319F00F94B976F8CF8AE0C7
:10B030000F94B9760F942A1D24968EAC9FAC24975A
:10B040008FE7892809F451C080933C0F62968CAC3D
:10B050009DACAEACBFAC62976C968CAE9DAEAEAE06
:10B06000BFAE6C97AF968CAE9DAEAEAEBFAEAF9797
:10B070002B961FAE2B976D961FAE6D9720E46E96A4
:10B080002FAF6E973CE16F963FAF6F9746E4A09667
:10B090004FAFA097A1961FAEA197A2961FAEA29701
:10B0A000A3961FAEA397A4961FAEA497EFE78E2E8C
:10B0B000912CA12CB12C2A968CAE9DAEAEAEBFAE1B
:10B0C0002A97FFE74F2E512C612C712CAB961CAEAA
:10B0D0001DAE1EAE1FAEAB9721E0E8962FAFE897EE
:10B0E0001AAE1EAE212C312C06C080933D0FAECF80
:10B0F00080E00F941712A89580913E0F882309F4E1
:10B1000074C10F94732424968EAC9FAC2497892825
:10B1100059F4909021109AAEA0902210AEAE2090DB
:10B120002310309024100AC0B0901007BAAE80905F
:10B1300011078EAE20901207309013072AAD3EAD56
:10B14000A101A1966FADA197A2967FADA297A396FC
:10B150008FADA397A4969FADA4970F9479B81816B6
:10B1600074F09AACA1969FAEA197AEACA296AFAE8A
:10B17000A297A3962FAEA397A4963FAEA4976D96E1
:10B180002FAD6D976E963FAD6E976F964FAD6F97E3
:10B19000A0965FADA0976AAD7EADC1010F9479B85E
:10B1A000181674F0BAAC6D96BFAE6D978EAC6E96F5
:10B1B0008FAE6E976F962FAE6F97A0963FAEA0970B
:10B1C0000F94FB45DC01CB01E3968CAC9DACAEAC9F
:10B1D000BFACE39788199909AA09BB09853C994036
:10B1E000A105B10550F00F9488830F94FB45E396B9
:10B1F0006CAF7DAF8EAF9FAFE397E8968FACE897CB
:10B20000882009F474C02AAD3EADA10163966FADEC
:10B21000639765967FAD659767968FAD67976896DC
:10B220009FAD68970F9442AD87FFDFC00F94FB4539
:10B23000DC01CB0162968CAC9DACAEACBFAC62972E
:10B2400088199909AA09BB0989389341A105B10553
:10B2500008F4CBC0D301C2012A968CAC9DACAEAC35
:10B26000BFAC2A9788199909AA09BB092496AEACE4
:10B27000BFAC2497B595A79597958795AB2819F0FE
:10B2800080933C0F02C080933D0F0F94FB456C965A
:10B290006CAF7DAF8EAF9FAF6C974B015C01629638
:10B2A0002CAD3DAD4EAD5FAD6297821A930AA40AF4
:10B2B000B50AAB968CAE9DAEAEAEBFAEAB97639605
:10B2C0008FAC6397A1968FAEA19765969FAC65975B
:10B2D000A2969FAEA2976796AFAC6797A396AFAEC4
:10B2E000A3976896BFAC6897A496BFAEA4972AAD03
:10B2F0003EADA10163966FAD639765967FAD65978F
:10B3000067968FAD679768969FAD68970F9479B8E9
:10B31000181614F00C946D6F0F94FB45DC01CB01F3
:10B320006C968CAC9DACAEACBFAC6C97881999098F
:10B33000AA09BB0989389341A105B10510F40C9401
:10B340006D6F0F94FB4562966CAF7DAF8EAF9FAF74
:10B350006297DC01CB0188199909AA09BB092091E0
:10B36000D80E3091D90E1216130614F40C94986D61
:10B370002A968CAD9DADAEADBFAD2A97840D951DBF
:10B38000A61DB71D24968EAC9FAC2497B595A795A6
:10B3900097958795892811F40C94696F80933C0FD9
:10B3A0008091D80E9091D90E01969093D90E8093EA
:10B3B000D80E63969FAC63976D969FAE6D9765961A
:10B3C000AFAC65976E96AFAE6E976796BFAC67975A
:10B3D0006F96BFAE6F9768968FAC6897A0968FAE4A
:10B3E000A09721E0E8962FAFE89720E030E040EA10
:10B3F00051E463966FAD639765967FAD65976796E9
:10B400008FAD679768969FAD68970F942EB62AAD5B
:10B410003EADA1010F9442AD87FF0EC0E0E6FCE017
:10B4200084918F01882309F4ECCD0F94B9760F5FD6
:10B430001F4FF8018491F6CF0F94FB45DC01CB013F
:10B44000AF968CAC9DACAEACBFACAF9788199909E8
:10B45000AA09BB09813D9740A105B10508F4B4C014
:10B4600024968EAC9FAC2497892881F0E0903C0F05
:10B47000F12CEDE5FCE084918F018823B9F00F9465
:10B48000B9760F5F1F4FF8018491F7CFE0903D0F21
:10B49000F12CEAE5FCE084918F01882339F00F94C8
:10B4A000B9760F5F1F4FF8018491F7CF42E06AAD84
:10B4B0007EADC1010F943E77E6E5FCE084918F01FB
:10B4C000882339F00F94B9760F5F1F4FF8018491EC
:10B4D000F7CFB701FF0C880B990B0F94546C8AE0DF
:10B4E0000F94B9762B968FAC2B97882009F452C015
:10B4F000A7969FACA797891418F4282D2F5F59C0E1
:10B500002B968FAC2B97A7969FACA797891054C00A
:10B51000282D2F5F2B962FAF2B97E4962FADE49716
:10B52000E5963FADE597E6964FADE697E7965FADBA
:10B53000E7976AAD7EADC1010F942DB66B017C011A
:10B5400020E030E0A9010F9479B818165CF420E0EF
:10B5500030E040EA50E4C701B6010F9442AD87FFE6
:10B560002BC00AC020E030E040EA50ECC701B60131
:10B570000F9479B8181604F524966FAD2497661FBA
:10B580006627661F80E00F945D2081E08093F20EB5
:10B590000C94F4688AACE4968FAEE4979EACE59682
:10B5A0009FAEE597E6962FAEE697E7963FAEE79714
:10B5B00021E02B962FAF2B970F94FB45AF966CAFE6
:10B5C0007DAF8EAF9FAFAF970F94FB456B017C01B2
:10B5D0000F94FB456C960CAD1DAD2EAD3FAD6C9739
:10B5E00062968CAC9DACAEACBFAC6297080D191DD9
:10B5F0002A1D3B1DC01AD10AE20AF30ADC01CB0165
:10B600008C0D9D1DAE1DBF1D81389F44A241B1050B
:10B6100070F0E9E3FCE084918F01882309F4F1CC18
:10B620000F94B9760F5F1F4FF8018491F6CF809188
:10B63000D80E9091D90EA6968EAC9FACA697881680
:10B6400099060CF055CDEDEDFBE084918F01882338
:10B6500009F4D7CC0F94B9760F5F1F4FF80184918E
:10B66000F6CF0F94F9880C94F46880911810882311
:10B6700011F40C94F46885E40F9448A7882331F002
:10B680000F9440A70F9493B7162F01C01FEF86E4C5
:10B690000F9448A7882331F00F9440A70F9493B7D5
:10B6A000062F01C00FEF1F920F931F921F938CEC78
:10B6B0009BE09F938F930F94AEAC1F920F931F92BA
:10B6C0001F9384EC9BE09F938F930E94899A0FB6FF
:10B6D000F894DEBF0FBECDBF1AE00E94749A181610
:10B6E00014F40C94F468115011F00C94726F0C94D3
:10B6F000F4680F9434780C94F4680F94FE770C94EB
:10B70000F4688091E3108F938091E2108F93809181
:10B71000E1108F938091E0108F938091DF108F93D1
:10B720008091DE108F938091DD108F938091DC10DB
:10B730008F938091DB108F938091DA108F9380919B
:10B74000D9108F938091D8108F9307E81EE51F932F
:10B750000F931F930F938091D7108F938091D610E2
:10B760008F938091D5108F938091D4108F93809177
:10B77000D3108F938091D2108F938091D1108F939B
:10B780008091D0108F938091CF108F938091CE10A5
:10B790008F938091CD108F938091CC108F93809157
:10B7A000CB108F938091CA108F938091C9108F9383
:10B7B0008091C8108F938091C7108F938091C6108D
:10B7C0008F938091C5108F938091C4108F93809137
:10B7D000C3108F938091C2108F938091C1108F936B
:10B7E0008091C0108F938091BF108F938091BE1075
:10B7F0008F938091BD108F938091BC108F931F9376
:10B800000F931F930F938091BB108F938091BA1069
:10B810008F938091B9108F938091B8108F938091FE
:10B82000B7108F938091B6108F938091B5108F933E
:10B830008091B4108F931F930F931F930F93809158
:10B840003B118F9380913A118F93809139118F938F
:10B85000809138118F93809137118F938091361199
:10B860008F93809135118F93809134118F938091B4
:10B8700033118F93809132118F93809131118F9377
:10B88000809130118F9380912F118F9380912E1181
:10B890008F9380912D118F9380912C118F931F93F3
:10B8A0000F931F930F938091B3108F938091B210D9
:10B8B0008F938091B1108F938091B0108F9380916E
:10B8C000AF108F938091AE108F938091AD108F93B6
:10B8D0008091AC108F938091AB108F938091AA10C0
:10B8E0008F938091A9108F938091A8108F9380914E
:10B8F000A7108F938091A6108F938091A5108F939E
:10B900008091A4108F931F930F931F930F93809197
:10B910002B118F9380912A118F93809129118F93EE
:10B92000809128118F93809127118F9380912611F8
:10B930008F93809125118F93809124118F93809103
:10B9400023118F93809122118F93809121118F93D6
:10B95000809120118F9380911F118F9380911E11E0
:10B960008F9380911D118F9380911C118F931F9342
:10B970000F931F930F938091A3108F938091A21028
:10B980008F938091A1108F938091A0108F938091BD
:10B990009F108F9380919E108F9380919D108F9315
:10B9A00080919C108F9380919B108F9380919A101F
:10B9B0008F93809199108F93809198108F9380919D
:10B9C00097108F93809196108F93809195108F93FD
:10B9D000809194108F931F930F931F930F938091D7
:10B9E00093108F93809192108F93809191108F93E9
:10B9F000809190108F9380918F108F9380918E10F3
:10BA00008F9380918D108F9380918C108F93809164
:10BA10008B108F9380918A108F93809189108F93D0
:10BA2000809188108F93809187108F9380918610DA
:10BA30008F93809185108F93809184108F931F93A3
:10BA40000F931F930F9384E199E09F938F930F942B
:10BA5000AEAC0FB6F894DEBF0FBECDBF2CEA35EC0E
:10BA600047E25EE36091F0107091F1108091F21066
:10BA70009091F3100F943AA89F938F937F936F93B5
:10BA80002CEA35EC47E25EE36091EC107091ED102A
:10BA90008091EE109091EF100F941CB79F938F93AD
:10BAA0007F936F938091EB108F938091EA108F9327
:10BAB0008091E9108F938091E8108F931F930F93DB
:10BAC0001F930F9387EE98E09F938F930F94AEACE4
:10BAD0002CEA35EC47E25EE36091FC107091FD10BA
:10BAE0008091FE109091FF100F943AA89F938F932E
:10BAF0007F936F932CEA35EC47E25EE36091F81098
:10BB00007091F9108091FA109091FB100F941CB76E
:10BB10009F938F937F936F938091F7108F93809172
:10BB2000F6108F938091F5108F938091F4108F937E
:10BB30001F930F931F930F9382EB98E09F938F9324
:10BB40000F94AEAC0FB6F894DEBF0FBECDBF8091A0
:10BB500002111F928F931F930F931F930F9320E057
:10BB600030E040E752E4609113117091141180911C
:10BB70001511909116110F943AA89F938F937F936C
:10BB80006F93809112118F93809111118F938091F7
:10BB900010118F9380910F118F931F930F931F9309
:10BBA0000F9380910E118F9380910D118F9380913F
:10BBB0000C118F9380910B118F9320E030E040E7C0
:10BBC00052E46091071170910811809109119091D0
:10BBD0000A110F943AA89F938F937F936F9380914C
:10BBE00006118F93809105118F93809104118F938B
:10BBF000809103118F931F930F931F930F9381EBEA
:10BC000097E09F938F930F94AEAC0FB6F894DEBF7E
:10BC10000FBECDBF809117118823E9F080911B11D1
:10BC20008F9380911A118F93809119118F93809126
:10BC300018118F931F930F931F930F938BE897E027
:10BC40009F938F930F94AEAC0FB6F894DEBF0FBEE8
:10BC5000CDBF0C94F4681F930F938CE697E09F93ED
:10BC60008F930F94AEAC0F900F900F900F900C9499
:10BC7000F468E7E8FEE584918F01882339F00F949A
:10BC8000B9760F5F1F4FF8018491F7CFE5E5FEE02D
:10BC900084918F01882311F40C94F4680F94B97681
:10BCA0000F5F1F4FF8018491F5CF8AE50F9448A7E5
:10BCB000882309F489C00F9440A76B017C0120E020
:10BCC00030E040E751EC0F9479B887FD38C020E0B0
:10BCD00030E040EA50ECC701B6010F9442AD1816AF
:10BCE00074F1F7FAF094F7F8F094C092E410D0925F
:10BCF000E510E092E610F092E710E7E8FEE58491A7
:10BD00008F01882339F00F94B9760F5F1F4FF80128
:10BD10008491F7CFE8E5F5E084918F01882339F02D
:10BD20000F94B9760F5F1F4FF8018491F7CF8AE027
:10BD30000F94B9768AE00F94B9760C94F468E7E82A
:10BD4000FEE584918F01882339F00F94B9760F5F57
:10BD50001F4FF8018491F7CFE8E5F5E084918F015A
:10BD6000882339F00F94B9760F5F1F4FF801849143
:10BD7000F7CFE3E9F5E084918F01882339F00F9440
:10BD8000B9760F5F1F4FF8018491F7CF61EF7FEF16
:10BD90008FEF9FEF0F94546CEBE8F5E084918F01E7
:10BDA000882339F00F94B9760F5F1F4FF801849103
:10BDB000F7CF6BEF7FEF8FEF9FEF0F94546C8AE01C
:10BDC0000F94B9760C94F468E7E8FEE584918F014E
:10BDD000882339F00F94B9760F5F1F4FF8018491D3
:10BDE000F7CFE8E5F5E084918F01882339F00F94CF
:10BDF000B9760F5F1F4FF8018491F7CF8AE00F9457
:10BE0000B9768091E4109091E510A091E610B09180
:10BE1000E710BC01CD01905842E00F943E778AE0D4
:10BE20000F94B9760C94F4680F94F98885E40F9414
:10BE300048A7882329F00F9440A76B017C0105C017
:10BE4000C12CD12CE12C00ECF02E8CE40F9448A7EF
:10BE500081110F9440A78AE50F9448A7882329F001
:10BE60000F9440A72B013C011CC020E030E048ECBF
:10BE700051E460914410709145108091461090916A
:10BE800047100F9442AD87FF07C0412C512C18ED8D
:10BE9000612E11E4712E05C0412C512C612CB0E4AF
:10BEA0007B2E88E50F9448A7882339F00F9440A78C
:10BEB0006AAF7BAF8CAF9DAF0AC0812C912CA3E5FC
:10BEC000AA2EA3E4BA2E8AAE9BAEACAEBDAE89E577
:10BED0000F9448A7882349F00F9440A722966CAF8F
:10BEE0007DAF8EAF9FAF229706C022961CAE1DAECF
:10BEF0001EAE1FAE229780911810882311F40C9467
:10BF0000786F81E694E00F940067882311F40C9415
:10BF1000786F332433940F94F9888091A90F882384
:10BF200029F060E086E190E00E94ADDA9090330263
:10BF30002F969FAE2F9720903402E091060DF0E0EF
:10BF4000EE0FFF1FE257FA4EA080B1806496BFAE9D
:10BF5000AEAE64972091BC193091BD1966963FAF83
:10BF60002EAF669780913C1090913D10A0913E10AD
:10BF7000B0913F1026968CAF9DAFAEAFBFAF269766
:10BF800089839A83AB83BC8380904010909041104A
:10BF9000A0904210B09043102A968CAE9DAEAEAEEB
:10BFA000BFAE2A978D829E82AF82B88620914410C0
:10BFB0003091451040914610509147102E962CAF6D
:10BFC0003DAF4EAF5FAF2E9729873A874B875C878F
:10BFD000209148103091491040914A1050914B10D7
:10BFE0002D873E874F87588BC701B6010F942EB619
:10BFF000609348107093491080934A1090934B10AF
:10C0000046E05DE05F934F93812C912C68EEA62E65
:10C0100062E4B62E78E4C72E70E1D72E2E96ECACF3
:10C02000FDAC0EAD1FAD2E972A962CAD3DAD4EAD9D
:10C030005FAD2A9726966CAD7DAD8EAD9FAD2697F0
:10C040000F94C8300F94F988209144103091451016
:10C050004091461050914710C301B2010F942EB683
:10C060007B018C01609344107093451080934610BF
:10C070009093471020914010309141104091421010
:10C080005091431060913C1070913D1080913E1092
:10C0900090913F10A6E0BDE0BF93AF93812C912C0F
:10C0A000E0E7AE2EE1E4BE2E0F94C8300F94F9887D
:10C0B0008AAC9BACACACBDAC80923C1090923D1075
:10C0C000A0923E10B0923F1022962CAD3DAD4EADE9
:10C0D0005FAD22972093401030934110409342105F
:10C0E00050934310E0904410F0904510009146109A
:10C0F0001091471046E05DE05F934F93812C912CA7
:10C10000F8E4AF2EF2E4BF2E22962CAD3DAD4EAD3D
:10C110005FAD22976AAD7BAD8CAD9DAD0F94C830FD
:10C120000F94F9880F900F900F900F900F900F9031
:10C1300080911810811124C084E090E09093260231
:10C14000809325020F94FB454B015C018BEB90E142
:10C150000E9482DFCC24C394D12CE12CF12CD1108D
:10C160000C94BC6F0F94EF12882311F40C94BC6FE5
:10C170009FB7F894809102018B7F809302019FBF4B
:10C180001092B00680911810882319F00E94AD9982
:10C1900002C00E948CA20F94F9888091181081111E
:10C1A0005DC084E090E0909326028093250241E0F8
:10C1B00060E084ED91E10E948FDF8093B0068111F1
:10C1C00048C00F94A11962E080E00F94F21487E850
:10C1D00099E40F94191420E030E048EC52E46091A7
:10C1E0003C1070913D1080913E1090913F100F9443
:10C1F0002DB660933C1070933D1080933E10909349
:10C200003F10E0904410F0904510009146101091BE
:10C2100047102091401030914110409142105091B0
:10C220004310E6E0FDE0FF93EF93812C912CE8E4CE
:10C23000AE2EE2E4BE2EF8E4CF2EF0E1DF2E0F9416
:10C24000C8300F94F98884EA91E10E9433E00F909E
:10C250000F9080911810882309F478C0311072C0B3
:10C260008091390E882329F060E0809155020E9468
:10C27000769884E090E0909326028093250284EEE5
:10C2800090E10E9482DFFF24F39400E010E00F941D
:10C29000EF12811139C00F94AA8381E00F947308C3
:10C2A000043F41E0140711F400E010E08091010127
:10C2B00084608093010101151105A1F480910907A3
:10C2C00090910A07009721F00197B9F4FF20A9F097
:10C2D0009FB7F894809102018460809302019FBF10
:10C2E000F12C0BC00431110541F49FB7F8948091F3
:10C2F00002018B7F809302019FBF0F5F1F4F84E07D
:10C3000090E00F94B70CC3CF9FB7F89480910201CF
:10C310008B7F809302019FBF8091390E882391F01B
:10C320000F94A11962E080E00F94F21487E899E479
:10C330000F94191480E60E94579740E060E080E077
:10C340000E943493832D0F94C59B56C00F94A1195E
:10C3500061E080E00F94F2148DE391E10F941914E1
:10C3600062E080E00F94F2148AE291E10F941914D4
:10C3700084E090E090932602809325020E946089D9
:10C380000F94EF1281111AC00F94AA8381E00F94C9
:10C3900073080E94A789882399F3809109079091D7
:10C3A0000A07029720F488EE93E00F94AB5D82E3D6
:10C3B00090E00F94B70C84E50F941E440E94098806
:10C3C00082E090E090932602809325020F94569C81
:10C3D0008091090790910A07029720F484EF91E079
:10C3E0000F94AB5D82E390E00F94B70C84E50F945B
:10C3F0001E4480E00F94AB193110F3C01092B006C8
:10C40000A4E0CA2ED12CB2E0AB2EB12C8091B006A4
:10C41000813009F4E6C01092B006D0922602C09294
:10C4200025020F94A11960E080E00F94F21483E7D5
:10C4300091E10F94191461E081E00F94F2148DE101
:10C440009BE30F94191462E081E00F94F2148FE5DE
:10C4500091E10F94191463E081E00F94F2148DE4DC
:10C4600091E10F94191461E080E00F94F21486E6D4
:10C4700094E00F949413E090BE190E2C000CFF086A
:10C480000E94D18701E010E08091B006811168C060
:10C490000F94AA8381E00F9473088091BE19082E2F
:10C4A000000C990B9701281B390B37FF03C03195FE
:10C4B00021953109253031050CF444C08E159F05B6
:10C4C00014F401501109E816F90634F40F5F1F4FF8
:10C4D0000430110564F009C00430110534F401156D
:10C4E000110529F401E010E002C003E010E061E072
:10C4F00080E00F94F2148FE396E00F94941362E0BF
:10C5000080E00F94F2148FE396E00F94941363E0AD
:10C5100080E00F94F2148FE396E00F949413602F51
:10C5200080E00F94F21486E694E00F949413E09068
:10C53000BE190E2C000CFF0864E670E080E090E06D
:10C540000F94C3450F94EF12882309F49DCF0093F5
:10C55000B00664EF71E080E090E00F94C34594CFA3
:10C560000F94A1190F94238EB0922602A092250257
:10C570008091B0068230F9F0833041F50F94F9884C
:10C580000E9424CE0F94A11960E080E00F94F21471
:10C5900086E891E10F94191462E080E00F94F214A0
:10C5A00087E899E40F94191487E99DE10F94139C8F
:10C5B0000F94F9882BCF80911810882321F080E008
:10C5C0000F94C59B23CF0F94569C20CF0F94A11995
:10C5D00062E080E00F94F21484E991E10F94191461
:10C5E00015CF81E00F94AB1966968EAD9FAD66971F
:10C5F0009093BD198093BC1931103FC020E030E00A
:10C6000040EA50E4609148107091491080914A10BE
:10C6100090914B100F942EB6609348107093491070
:10C6200080934A1090934B10E0904410F090451086
:10C630000091461010914710209140103091411008
:10C64000409142105091431060913C1070913D1008
:10C6500080913E1090913F10E6E0FDE0FF93EF9354
:10C66000812C912CA12CE0E4BE2EF8E4CF2EF0E139
:10C67000DF2E0F94C8300F900F90E0904410F09090
:10C68000451000914610109147102D813E814F8139
:10C69000588569817A818B819C81E6E06E2EEDE080
:10C6A0007E2E7F926F92812C912CF8E4AF2EF2E4D3
:10C6B000BF2EA8E4CA2EA0E1DA2E0F94C8300F9442
:10C6C000F988E984FA840B851C852D813E814F8190
:10C6D000588569817A818B819C817F926F92812CB0
:10C6E000912CB0E7AB2EB1E4BB2E0F94C8300F9461
:10C6F000F988CE010D960E945FB580E1FE0131966A
:10C70000ACE3B0E101900D928A95E1F780E1ECE3B2
:10C71000F0E1AAEABFE001900D928A95E1F72F9629
:10C720009FAD2F9790933302209234022F929F93C4
:10C7300083E697E09F938F938E01015E1F4F1F93B7
:10C740000F930F9406AD60E0C8010E9459E186E4A2
:10C7500094E10F94184A10921F0E10921E0E0FB6FD
:10C76000F894DEBF0FBECDBF3FC50E94F5BB3CC5F0
:10C7700083E50F9448A7882309F436C50F9440A792
:10C780000F948DB76B017C012B0187E899E40F941E
:10C79000184AE2E3FEE084918F01882339F00F9478
:10C7A000B9760F5F1F4FF8018491F7CF0D2C000C65
:10C7B000EE08FF08C701B6010F94546C8AE00F948D
:10C7C000B9760F94FB454B015C011092380E6091D5
:10C7D0000A0D70910B0D072E000C880B990B0F940E
:10C7E00048AD20E030E0A9010F9442AD811111C0A5
:10C7F00060918E1570918F15072E000C880B990B88
:10C800000F9448AD11E020E030E0A9010F9442AD53
:10C81000811110E0052C000C660877088DE2282EA7
:10C820008EE0382E111115C08091380E81116CC028
:10C83000C301B2010F9448AD20915D0E30915E0EA0
:10C8400040915F0E5091600E0F9479B818168CF0DD
:10C850005BC0C301B2010F9448AD20915D0E3091D1
:10C860005E0E40915F0E5091600E0F9442AD87FFB7
:10C870004BC00F94FB45DC01CB0188199909AA092B
:10C88000BB09893E9340A105B10508F434C0EFE22D
:10C89000FEE084915F01882341F00F94B976FFEFA9
:10C8A000AF1ABF0AF5018491F6CF60915D0E7091C9
:10C8B0005E0E80915F0E9091600E41E00F943E7786
:10C8C000F10184910DE2A02E0EE0B02E882341F0FC
:10C8D0000F94B976FFEFAF1ABF0AF5018491F6CF36
:10C8E000C701B6010F94546C8AE00F94B9760F9487
:10C8F000FB454B015C010F94AA8380E00F94730801
:10C9000080E00F9417128ECF8DE697E10F94184AAE
:10C910006BC48FE30F9448A7882309F4BCC00F941D
:10C92000E7681A821982882381F008E614E0D801AA
:10C930008D918D01882319F00F94B976F8CF8AE094
:10C940000F94B9760CE714E00AC003E914E0F8018B
:10C9500081918F01882399F30F94B976F8CFD8018C
:10C960008D918D01882319F00F94B976F8CF8AE064
:10C970000F94B97688248A94982C5401A3E24A2E05
:10C98000512C612C712CB0EB2B2EBFE03B2E1AAE3C
:10C9900069817A81072E000C880B990B0F9448ADA2
:10C9A00020918C1030918D1040918E1050918F10ED
:10C9B0000F941CB76B017C012AAD21110DC0E9E277
:10C9C000FEE084918F01882359F00F94B9760F5FB0
:10C9D0001F4FF8018491F7CFC501B4010F94546C37
:10C9E000E6E2FEE084918F01882339F00F94B97656
:10C9F0000F5F1F4FF8018491F7CFC301B2010F946D
:10CA0000546CE3E2FEE084918F01882339F00F94A7
:10CA1000B9760F5F1F4FF8018491F7CF69817A8152
:10CA2000072E000C880B990B0F94546CE0E2FEE08B
:10CA300084918F01882339F00F94B9760F5F1F4FCF
:10CA4000F8018491F7CF20E030E04AE754E4C701D1
:10CA5000B6010F943AA842E00F943E778AE00F9413
:10CA6000B976FAADFF5FFAAFF63009F4BDC3BE0187
:10CA70006F5F7F4FC1010E94BFC8B2E02B0E311C17
:10CA8000E5E04E0E511C611C711CFFEF8F1A9F0ACE
:10CA9000AF0ABF0A7DCF81E20F9448A7882309F42B
:10CAA0004AC061E086EA9FE00F94D2B588E090E04A
:10CAB0009A838983BE016F5F7F4F80EB9FE00E9466
:10CAC000D9C888E190E09A838983BE016F5F7F4F68
:10CAD00082EB9FE00E94D9C880E390E09A8389832B
:10CAE000BE016F5F7F4F84EB9FE00E94D9C880E555
:10CAF00090E09A838983BE016F5F7F4F86EB9FE052
:10CB00000E94D9C888E790E09A838983BE016F5F4D
:10CB10007F4F88EB9FE00E94D9C807EA14E0D80154
:10CB20008D918D01882319F00F94B976F8CF8AE0A2
:10CB30000F94B97659C38AE50F9448A7882319F151
:10CB400061E086EA9FE00F94D2B51A82198200EB69
:10CB50001FE0BE016F5F7F4FC8010E94D9C80E5F02
:10CB60001F4F0A3BBFE01B07A1F708EB14E0F801D9
:10CB700081918F01882319F00F94B976F8CF8AE05C
:10CB80000F94B97631C383E50F9448A7882309F43D
:10CB9000CEC00F9440A70F948DB77A83698389E440
:10CBA0000F9448A7882309F41FC30F9440A70F943C
:10CBB00093B7653008F018C3862F90E08852984FDD
:10CBC000BE016F5F7F4F880F991F0E94D9C802EC8A
:10CBD00014E0D8018D918D01882319F00F94B97656
:10CBE000F8CF8AE00F94B9760CE714E0F801819150
:10CBF0008F01882319F00F94B976F8CF8AE00F944B
:10CC0000B9763EEA232E3FE0332E44244A94542C36
:10CC1000320153E2852E912CA12CB12C1AAE1A822E
:10CC20001982FAADFF2331F0BE016F5F7F4FC10162
:10CC30000E94BFC869817A81072E000C880B990B6E
:10CC40000F9448AD20918C1030918D1040918E1032
:10CC500050918F100F941CB76B017C012AAD2111EC
:10CC60000DC0ECE1FEE084918F01882359F00F9410
:10CC7000B9760F5F1F4FF8018491F7CFC301B2015E
:10CC80000F94546CE9E1FEE084918F01882339F020
:10CC90000F94B9760F5F1F4FF8018491F7CFC5014C
:10CCA000B4010F94546CE6E1FEE084918F01882377
:10CCB00039F00F94B9760F5F1F4FF8018491F7CFC9
:10CCC00069817A81072E000C880B990B0F94546CA4
:10CCD000E3E1FEE084918F01882339F00F94B97667
:10CCE0000F5F1F4FF8018491F7CF20E030E04AE753
:10CCF00054E4C701B6010F943AA842E00F943E777E
:10CD00008AE00F94B976FAADFF5FFAAF25E0820EA4
:10CD1000911CA11CB11C3FEF431A530A630A730A0A
:10CD200042E0240E311CF63009F079CF5DC2E2E01A
:10CD3000FEE084918F01882309F456C20F94B976DE
:10CD40000F5F1F4FF8018491F6CF0F94F9888BE4A1
:10CD50000F9448A7882399F00F940DA76B017C01CD
:10CD600020E030E0A9010F9479B887FD08C0C09297
:10CD7000D10FD092D20FE092D30FF092D40F82E570
:10CD80000F9448A7882361F00F940DA76B017C01D5
:10CD900020E030E0A9010F9442AD87FF89C006C0B2
:10CDA000C12CD12C20E8E22E2FEBF22E84E40F943C
:10CDB00048A7882329F00F940DA74B015C0106C0FA
:10CDC000812C912C90E8A92E9FEBB92E87E50F942A
:10CDD00048A7882329F00F940DA72B013C0106C01A
:10CDE000412C512C80E8682E8FEB782E88E40F942C
:10CDF00048A7882339F00F940DA76AAF7BAF8CAF9B
:10CE00009DAF08C020E030E040E85FEB2AAF3BAFC9
:10CE10004CAF5DAF20E030E0A901C501B4010F9433
:10CE200079B887FD45C020E030E0A901C301B20117
:10CE30000F9479B887FD3CC020E030E0A9016AADCD
:10CE40007BAD8CAD9DAD0F9479B887FD31C020E0EE
:10CE500030E0A901C501B4010F9442AD882391F1DE
:10CE600020E030E040E05FE3C501B4010F943AA850
:10CE70006B017C012AAD3BAD4CAD5DADC301B20190
:10CE80000F943AA84B015C01A7019601C701B601B6
:10CE90000F943AA82BED3FE049E450E40F943AA8F0
:10CEA0009B01AC01C501B4010F941CB76B017C015F
:10CEB00020E030E0A901C701B6010F9479B887FFDF
:10CEC00004C00BC0C12CD12C7601C092CD0FD092E2
:10CED000CE0FE092CF0FF092D00FE7E8FEE58491FD
:10CEE0008F01882339F00F94B9760F5F1F4FF80137
:10CEF0008491F7CFE8E5F7E084918F01882339F03A
:10CF00000F94B9760F5F1F4FF8018491F7CF6091AE
:10CF1000D10F7091D20F8091D30F9091D40F42E036
:10CF20000F943E778AE00F94B976E2E5F7E08491BA
:10CF30008F01882339F00F94B9760F5F1F4FF801E6
:10CF40008491F7CFC090CD0FD090CE0FE090CF0F4F
:10CF5000F090D00F20E030E0A901C701B6010F9496
:10CF600042AD882349F042E0C701B6010F943E77F5
:10CF70008AE00F94B97638C1EDE4F7E084918F012F
:10CF8000882311F40C945C460F94B9760F5F1F4F01
:10CF9000F8018491F5CF0F9436A70F9448AD6B013B
:10CFA0007C0120E030E0A9010F9442AD87FD40C034
:10CFB00020E030EA40E854E4C701B6010F9479B8A4
:10CFC000181674F120E030E047E054E4C701B601E0
:10CFD0000F9479B887FD2FC020E030E04CE752E491
:10CFE000C701B6010F943AA820E030EA40E854E4C3
:10CFF0000F941CB70F9493B7162F802F0F94829D18
:10D00000612F802F0F94719D0F5F043009F4ECC0E5
:10D01000D5018D915D010F9448A78823A9F3BBCF5B
:10D02000C12C10EAD12E10E8E12E14E4F12ED4CF59
:10D03000C12CD12C760120E030E04CE752E4C7014E
:10D04000B6010F943AA820E034EB40E954E4D0CF85
:10D0500085E40F9448A7882309F4C6C00F9440A71D
:10D060000F9493B76B017C018B016830710569F0F7
:10D070006031710551F06032710539F0603471052D
:10D0800021F06038710509F0AFC00F94F98880E095
:10D0900091E05C0100901B0702C0B694A7940A942B
:10D0A000E2F7C6010E94ACF480931B0720911F0297
:10D0B00040912302682F83E00E94CFF440907C10BF
:10D0C00050907D1060907E1070907F10A016B10679
:10D0D00070F5C801B5010F94CDBA6B01E12CF12CAC
:10D0E000C701B6010F9446AD9B01AC016091901051
:10D0F0007091911080919210909193100F943AA892
:10D10000609390107093911080939210909393106D
:10D11000A3019201C701B6010F94E3B560937C109F
:10D1200070937D1080937E1090937F105DC0C50139
:10D13000B8010F94CDBA6B01E12CF12CC701B601F7
:10D140000F9446AD9B01AC016091901070919110CD
:10D1500080919210909193100F941CB7609390104F
:10D16000709391108093921090939310C301B20129
:10D17000A70196010F94F4BA20937C1030937D1090
:10D1800040937E1050937F102FC0809118108823F9
:10D1900029F085E40F9448A7811197C70F94706C0C
:10D1A00023C083E40F9448A790911810882329F096
:10D1B0009923D1F00E94AD9917C09111FBCF0E9425
:10D1C0008CA212C080918C1590918D158E559C4E1D
:10D1D0009F938F938DEE9DE09F938F930F94AEACB2
:10D1E0000F900F900F900F9010923B0D10923A0DF0
:10D1F000ACC284E50F9448A7882309F437C1209175
:10D20000100D3091110DF90131968F01021B130B96
:10D210007F0181918032C9F38930B9F3082E000C67
:10D22000990B0F9430BBF7018083E091100DF091C2
:10D23000110DE00FF11F808190ED980F953008F4EB
:10D2400063C08F3309F447C0883781F08336A9F172
:10D25000EDEDFDE084918F01882309F403C10F9463
:10D26000B9760F5F1F4FF8018491F6CF80911810A7
:10D27000882309F46AC240E050E061EC76E28CE871
:10D2800092E10E94ADA380935402909155028913BC
:10D2900007C08091410D882319F083EC9DE059C0AF
:10D2A0000F94F98880915402805F0E94579743E061
:10D2B00061E081E00E94349348C280911810882375
:10D2C00009F443C20F94F9880E9462978091540236
:10D2D0008093550256C08091181040E050E088239A
:10D2E00051F061EC76E28CE892E10E94ADA380936C
:10D2F000540211E010C062E772E18BE792E10E94F4
:10D30000ADA38093540206C00F9440A70F9493B727
:10D310006093540210E00F94F9888091540221E048
:10D3200030E0082E01C0220F0A94EAF79091400DD8
:10D33000292B2093400D90911810992329F1909159
:10D34000550289130DC09091410D992349F089EA46
:10D350009DE09F938F930F94AEAC0F900F90D7C624
:10D36000805F0E94579743E061E081E00E94349320
:10D370000E9462978091540280935502112309F410
:10D38000E4C10E940792E1C1882309F432C0E7E8B2
:10D39000FEE584918F01882339F00F94B9760F5FF1
:10D3A0001F4FF8018491F7CFE7EAFDE084918F01E8
:10D3B000882339F00F94B9760F5F1F4FF8018491DD
:10D3C000F7CF6091540270E080E090E00F94546CCD
:10D3D0008AE00F94B976E7E4F5E084918F01882321
:10D3E00009F440C00F94B9760F5F1F4FF801849184
:10D3F000F6CF86E40F9448A7882399F00F9440A7AE
:10D400006B017C0120E030E0A9010F9479B8181677
:10D4100044F4C0927C02D0927D02E0927E02F092AF
:10D420007F02E7E8FEE584918F01882339F00F94AD
:10D43000B9760F5F1F4FF8018491F7CFE5E3F5E070
:10D4400084918F01882339F00F94B9760F5F1F4FB5
:10D45000F8018491F7CF6091060D70E080E090E0D4
:10D460000F94546C8AE00F94B9766FC184E40F94E2
:10D4700048A7882309F408C10F9440A70F948DB7DB
:10D480006330710509F061C18EEE94E09F938F9334
:10D490000F94AEAC81E40F9448A70F900F908823AF
:10D4A000B9F08091100D9091110DDC0111962C9125
:10D4B000283741F440E150E060E070E002960F94BC
:10D4C00062AA04C00F9440A70F948DB78B0102C0CD
:10D4D00000E010E083E40F9448A7882339F00F940C
:10D4E00040A70F948DB7262F872F02C020E080E140
:10D4F0001F71A22EB82EB1E0AB16B0E1BB0618F03A
:10D50000A12CB0E1BB2EC501800F911F813090414D
:10D5100028F080E090E15C01A01AB10A88E50F9440
:10D5200048A7882309F475C02091100D3091110D82
:10D53000A9014F5F5F4F9E012F5F3F4F6901F901C6
:10D54000E12CF12C9A01D9018C912F5F3F4F882358
:10D55000A1F140E1E416F10469F18032A1F38A30CF
:10D5600061F190ED980F9A3018F48295807F07C092
:10D570009FE9980F9630A8F48295807F8057AD017F
:10D580004E5F5F4F11969C9120ED290F2A3010F4C9
:10D59000822B0BC02FE9290F263018F49755892BC1
:10D5A00004C0F194E194F10808C081936FEFE61A8A
:10D5B000F60AC8CFA0E1EA2EF12C5701E114F104DC
:10D5C00041F1812C912CD6016D916D01C401800F28
:10D5D000911F0F94D2B5BFEF8B1A9B0AE814F90480
:10D5E00091F71F930F93FF92EF9281EC94E09F933A
:10D5F0008F930F94AEAC6091CF197091D0198AE0DF
:10D6000090E00F94DFB40F900F900F900F900F9059
:10D610000F906801E12CF12CA114B10409F495C01C
:10D620008D2D0F946AA78C2D0F946AA76091CF1946
:10D630007091D01980E290E00F94DFB410E1EFEF29
:10D64000CE1ADE0AEE0AFE0AC60101970F94A2B5B1
:10D65000082F6091CF197091D01980E290E00F945B
:10D66000DFB4802F0F946AA71150F1E0AF1AB10810
:10D6700011F01111E4CF6091CF197091D0198AE0A7
:10D6800090E00F94DFB4C8CFE7E8FEE584918F0106
:10D69000882339F00F94B9760F5F1F4FF8018491FA
:10D6A000F7CFE1E6F5E084918F01882339F00F94FC
:10D6B000B9760F5F1F4FF8018491F7CF00918C1559
:10D6C00010918D150E551C4ED8018D918D0188231A
:10D6D00019F00F94B976F8CFE2EAFDE084918F015A
:10D6E000882309F4BFCE0F94B9760F5F1F4FF8015E
:10D6F0008491F6CFC090B60FD090B70FE090B80FDE
:10D70000F090B90F209148103091491040914A1083
:10D7100050914B10C701B6010F942DB64B015C011F
:10D720002DEC3CEC4CEC5DEB0F9442AD87FD3AC028
:10D730002DEC3CEC4CEC5DE3C501B4010F9479B8E1
:10D7400018160CF438C00F9440A181E090E090933B
:10D750002602809325020F94FB456093030F70937C
:10D76000040F8093050F9093060FE0918C15F091B4
:10D770008D15E156FC4E8081813019F0863009F01C
:10D78000C6C4EDE6F7E184918F01882339F00F9448
:10D79000B9760F5F1F4FF8018491F7CF8AE00F949D
:10D7A000B976B5C4E091060DF0E0E654F04F808103
:10D7B000811192C409C0E091060DF0E0E654F04FEB
:10D7C0008081882309F4BFCFC0924810D0924910BD
:10D7D000E0924A10F0924B1088E490E10E945FB50D
:10D7E000E091060DF0E0E654F04F908181E089274A
:10D7F0000F9401A58CC420E030E040E85FE3609125
:10D8000048107091491080914A1090914B100F94DC
:10D810002EB6609348107093491080934A109093ED
:10D820004B10E0904410F09045100091461010917C
:10D83000471020914010309141104091421050917A
:10D84000431060913C1070913D1080913E1090917A
:10D850003F10E6E0FDE0FF93EF93812C912CE8EC84
:10D86000AE2EE3E4BE2EF8E4CF2EF0E1DF2E0F94CF
:10D87000C8300F900F900C94BE4182E090E09093DE
:10D880002602809325021092250E1092240E0C94ED
:10D8900007460F9436A7AB01BC0140936019509323
:10D8A000611960936219709363198BEA98E10E9481
:10D8B000E1E59ACC0F9440A70F948DB78B010C949F
:10D8C000D4490F94F98888E50F9448A7882319F064
:10D8D000179A1092070D89E50F9448A7882319F02D
:10D8E000169A1092080D8AE50F9448A785E40F94C4
:10D8F00048A7882311F40C94524E149A0C94524E5B
:10D900001A8219824AE050E0BE016F5F7F4FC70163
:10D910000F9462AA78A36F8F89819A8188169906DD
:10D9200009F062CC4AE050E0BE016F5F7F4FC60154
:10D930000F9462AA7AA369A389819A8168167906ED
:10D9400009F052CC4AE050E0BE016F5F7F4FC50145
:10D950000F9462AA7CA36BA389819A810817190787
:10D9600009F042CC8FE790E09EA38DA35801EFEF22
:10D97000AE1ABE0AD8018C918D3211F5750167017E
:10D98000BFEFCB1ADB0AF70180810F94EE49382EE6
:10D99000811102C07601F3CFEA18FB08DE2CC70123
:10D9A00099278330910569F543E050E067EC7AE50B
:10D9B000C5010F94D4AB892B09F042C01EA21DA251
:10D9C000332009F411CCCE0101960F94A46388236F
:10D9D00009F40ACCFE017F96DE011196AE01495D85
:10D9E0005F4F219131918D919D918217930708F49A
:10D9F0004CC02817390708F4F7CB4E175F0789F793
:10DA0000F3CB8530910571F445E050E061EC7AE5A7
:10DA1000C5010F94D4AB892B99F481E090E09EA3CB
:10DA20008DA3CECF049761F444E050E06CEB7AE52F
:10DA3000C5010F94D4AB892B19F482E090E0EFCFAD
:10DA40008EEF8E0D823008F0CFCBD80111968C91DD
:10DA500011978F7D823509F0C7CB12968C918F7DFF
:10DA6000833409F0C1CBB2E0DB1203C083E090E065
:10DA7000D6CFF801838190ED980F9A3008F0B4CB9F
:10DA8000082E000C990B8E97CACF84E092E10E9479
:10DA900082DF4CEE5CE062E080E00F949619D201E8
:10DAA0001D912D01812F0F94EE49811108C06FEC5B
:10DAB00076E0812F110F990B0F94DFB4F0CF44EF74
:10DAC00051E163E080E00F949619809109079091ED
:10DAD0000A07029720F488EE93E00F94AB5D82E38F
:10DAE00090E00F94B70C84E50F941E4484EF91E00E
:10DAF0000F94B70C8091090790910A07029720F4C0
:10DB000088EE93E00F94AB5D82E390E00F94B70C46
:10DB100084E50F941E4480E090E00F94B59C81E072
:10DB20000F94AB190F94A11980E00F9417125CCBDE
:10DB3000AB96CCACDDACEEACFFACAB97C80ED91E4F
:10DB4000EA1EFB1EAB962CAD3DAD4EAD5FADAB9767
:10DB5000281B390B4A0B5B0B2A966CAD7DAD8EAD45
:10DB60009FAD2A970F94E3B5A70196010F94F4BADD
:10DB7000DA01C901840D951DA61DB71D84319105DB
:10DB8000A105B105E4F02C013D018C3E9105A105F4
:10DB9000B1052CF06BEE462E512C612C712C40E817
:10DBA0004416510461047104DCF05EEF852E912C63
:10DBB000A12CB12C84189508A608B7080AC034E136
:10DBC000432E512C612C712C44E1842E912CA12CDC
:10DBD000B12C2A968CAE9DAEAEAEBFAE2A9706C0D3
:10DBE0002A964CAE5DAE6EAE7FAE2A97E9ECFCE0B5
:10DBF00084918F01882339F00F94B9760F5F1F4FFE
:10DC0000F8018491F7CFC301B2010F94546CE4EC96
:10DC1000FCE084918F01882339F00F94B9760F5F6F
:10DC20001F4FF8018491F7CF2A966CAD7DAD8EAD74
:10DC30009FAD2A970F94546CEDEBFCE084918F011B
:10DC4000882339F00F94B9760F5F1F4FF801849144
:10DC5000F7CF42E06D966FAD6D976E967FAD6E9784
:10DC60006F968FAD6F97A0969FADA0970F943E775C
:10DC7000E6EBFCE084918F01882339F00F94B976AC
:10DC80000F5F1F4FF8018491F7CF42E0A1966FAD6F
:10DC9000A197A2967FADA297A3968FADA397A496C6
:10DCA0009FADA4970F943E778AE00F94B976809148
:10DCB000D80E9091D90E039714F40C94B8592A9663
:10DCC0006CAD7DAD8EAD9FAD2A970F9448AD20E031
:10DCD00030E040E850E40F943AA84B015C016D96A7
:10DCE0002FAD6D976E963FAD6E976F964FAD6F9758
:10DCF000A0965FADA097A1966FADA197A2967FADBC
:10DD0000A297A3968FADA397A4969FADA4970F94C7
:10DD10002DB620ED3FE049E450E40F943AA820E00E
:10DD200030E040E05FE30F943AA89B01AC01C501ED
:10DD3000B4010F941CB74B015C01C701B6010F94ED
:10DD400048AD20E030E04AE754E40F941CB76B0183
:10DD50007C01E0EBFCE084918F01882339F00F9483
:10DD6000B9760F5F1F4FF8018491F7CF42E0C501EC
:10DD7000B4010F943E77EAEAFCE084918F01882396
:10DD800039F00F94B9760F5F1F4FF8018491F7CFE8
:10DD900042E0C701B6010F943E778AE00F94B9764E
:10DDA0002AE939E949E15FE3C501B4010F943AA8D2
:10DDB0004B015C016093EE0E7093EF0E8093F00EBA
:10DDC0009093F10E9B01AC010F942EB6A701960122
:10DDD0000F941CB76093EA0E7093EB0E8093EC0ED9
:10DDE0009093ED0EA5019401C701B6010F943AA8D6
:10DDF00020E030E040E05EE30F943AA86093E60E46
:10DE00007093E70E8093E80E9093E90EECE9FCE046
:10DE100084918F01882339F00F94B9760F5F1F4FDB
:10DE2000F8018491F7CF8AE00F94B976E6E9FCE037
:10DE300084918F01882339F00F94B9760F5F1F4FBB
:10DE4000F8018491F7CF6091EE0E7091EF0E809102
:10DE5000F00E9091F10E42E00F943E778AE00F941D
:10DE6000B976E0E9FCE084918F01882339F00F94C2
:10DE7000B9760F5F1F4FF8018491F7CF6091EA0EDA
:10DE80007091EB0E8091EC0E9091ED0E42E00F94AC
:10DE90003E778AE00F94B976EAE8FCE084918F013E
:10DEA000882339F00F94B9760F5F1F4FF8018491E2
:10DEB000F7CF6091E60E7091E70E8091E80E909199
:10DEC000E90E42E00F943E778AE00F94B9760C9405
:10DED000B85980933D0F0C94D059E8961FAEE8973F
:10DEE0000C94F55984E690E00F94B70C0C946D5B9C
:10DEF000312C0C948B5FE12CF12C8091010184601A
:10DF000080930101E114F10409F04EC080910907EA
:10DF100090910A070097F1F10197D1F19FEFE91A6B
:10DF2000F90AA1E0DA1609F452C0DA1608F04AC07C
:10DF300084E090E00F94B70C0F94FB4595018401A9
:10DF40000054184D264F3F4F06171707280739076B
:10DF500010F00C94AF6080E990E10E9482DF1F8E88
:10DF600018A219A21AA2CE014F960F94A37C0F9467
:10DF7000F988149ADD24D3940F94AA8381E00F9436
:10DF80007308F4EFEF16F1E0FF0609F0B6CFB3CF58
:10DF9000CC2021F29FB7F894809102018460809395
:10DFA00002019FBFC12CBACF84E1E816F10409F049
:10DFB000B5CF9FB7F894809102018B7F80930201C7
:10DFC0009FBFACCFB2E0DB16E1F00C94AF6084E011
:10DFD00090E00F94B70C0F94EF12882369F2E09150
:10DFE000060DF0E0EE0FFF1FE257FA4E64962EADDD
:10DFF0003FAD6497318320830E946EC842E0D42EE7
:10E00000BBCF0091060D10E0F801EE0FFF1FE257A5
:10E01000FA4E60817181072E000C880B990B0F94CA
:10E0200048AD000F111F000F111FF801EF5DFF4EEB
:10E0300020813181428153810F942DB62B013C0107
:10E0400020E030E0A9010F9479B818165CF420E0C4
:10E0500030E040E85FE3C301B2010F9442AD87FFB7
:10E0600016C00AC020E030E040E85FEBC301B20117
:10E070000F9479B818165CF48BEB90E10E9482DF64
:10E080000F94FB454B015C01D12C0C94B26064E011
:10E0900081E00F94F214E091060D34E0E39FF0016B
:10E0A0001124EF5DFF4E80819181A281B3818F8F1A
:10E0B00098A3A9A3BAA3CE014F960E94068C0F94F1
:10E0C0009413A4E1EA2EF12C57CF0F9440A70F949C
:10E0D00093B76093540262C82DEC3CEC4CEC5DE3CA
:10E0E000C501B4010F9479B818160CF46DCB2BCB85
:10E0F000A5019401F101662D772D8F2F922D0F949C
:10E1000042AD181614F40C94D93A0C94E93AC95853
:10E11000DF4F0FB6F894DEBF0FBECDBFDF91CF91BA
:10E120001F910F91FF90EF90DF90CF90BF90AF9035
:10E130009F908F907F906F905F904F903F902F9027
:10E1400008952F923F924F925F926F927F928F929B
:10E150009F92AF92BF92CF92DF92EF92FF920F9376
:10E160001F93CF93DF93CDB7DEB7C95CD1090FB64C
:10E17000F894DEBF0FBECDBF782E81E00F94B06D56
:10E18000711025C010920B0D10920A0D19821A827F
:10E190001B821C82CE0101960F94A37C61E080EC6F
:10E1A0009FE00F94B4B560E08FEB9FE00F94B4B59F
:10E1B00060E08EEB9FE00F94B4B560E08DEB9FE0E4
:10E1C0000F94B4B560E08CEB9FE00F94B4B580E0A1
:10E1D0000F94AB190F9488600F947F0F1092050D68
:10E1E0001092040D83E0E7E0FDE0DF011D928A95C7
:10E1F000E9F781E00F941665C855DF4F998388834E
:10E20000C85AD0408AEE9BE10E9482DF0F94456598
:10E2100040E050E061E080E090E00F94F16D40E07C
:10E2200050E061E081E090E00F94F16DE0904410E7
:10E23000F090451000914610109147102091401029
:10E2400030914110409142105091431060913C1028
:10E2500070913D1080913E1090913F100F944D5958
:10E260000E9465B41092240220E030E040EA50E4BD
:10E2700060913C1070913D1080913E1090913F1044
:10E280000F942EB61B012C0160933C1070933D102F
:10E2900080933E1090933F1020E030E040EA50E43D
:10E2A0006091401070914110809142109091431004
:10E2B0000F942EB69B01AC016093401070934110F7
:10E2C0008093421090934310E0904410F0904510DA
:10E2D000009146101091471086E09DE09F938F9328
:10E2E000812C912CB0EAAB2EB1E4BB2E88E4C82E71
:10E2F00080E1D82EC201B1010F94C8300F94F98883
:10E300000F944F650F900F90882311F40C94B584EF
:10E3100080EB9BE10E9433E0772089F080E89BE16D
:10E320000E9482DF63E080E00F94F21461E070E00D
:10E3300080E090E00F9479138AE79BE110C08AE5B2
:10E340009BE10E9482DF62E080E00F94F21461E0C2
:10E3500070E080E090E00F94791384E59BE10F94E6
:10E3600019140F94E66D71102EC084E090E0909324
:10E3700026028093250240E060E089E39BE10E9451
:10E380008FDF882321F081E19BE10E9433E08BE75E
:10E390009AE10E9433E082E090E09093260280931D
:10E3A00025028AE59BE10E9482DF62E080E00F9413
:10E3B000F21461E070E080E090E00F94791384E55E
:10E3C0009BE10F941914609024021092240220E023
:10E3D00030E040E85FE36091441070914510809117
:10E3E0004610909147100F942DB67B018C016093DD
:10E3F00044107093451080934610909347102091DD
:10E400004010309141104091421050914310609162
:10E410003C1070913D1080913E1090913F10E6E0CD
:10E420004E2EEDE05E2E5F924F92812C912CF0EA01
:10E43000AF2EF1E4BF2EA8E4CA2EA0E1DA2E0F948D
:10E44000C8300F94F98880E090E0A0EAB0E48093AF
:10E45000441090934510A0934610B093471081E06C
:10E460008093240284E00F94831AE0904410F0908B
:10E4700045100091461010914710209140103091A6
:10E480004110409142105091431060913C107091A6
:10E490003D1080913E1090913F105F924F920F94EB
:10E4A000C8300F94F9880F94E8196092240282E032
:10E4B0000F94E6880F900F900F900F9020E030E0BF
:10E4C00040EA50E40F9442AD81110C94B18477205E
:10E4D000E9F0C855DF4F88819981C85AD0400F9420
:10E4E000F5640F946E110F94810D0F9420158823FD
:10E4F00011F40C9461840F94506C803F11F00C94D3
:10E50000AD8481E00F94F1680C94AD848AEF0F9490
:10E51000F16860E070E088EF9FE00F94CEB50F9453
:10E52000E66D84ECE2E9F5E1DF011D928A95E9F7F9
:10E53000E1E9FEE184918F01882339F00F94B976E7
:10E540000F5F1F4FF8018491F7CF61E070E080E02A
:10E5500090E00F94546C0F94B777BE016F5A7F4FC1
:10E560008AE59BE10E9470DF62968FAD62978430EE
:10E5700020F083E062968FAF629780E090E0A0EA9F
:10E58000B0E48093441090934510A0934610B0934C
:10E59000471021E73EE1C657DF4F39832883CA5829
:10E5A000D04081E995E1CE57DF4F99838883C258E7
:10E5B000D040A0969FAF8EAFA097A8963FAF2EAF4A
:10E5C000A89781E090E0A0E0B0E0AE968CAF9DAF60
:10E5D000AEAFBFAFAE970F94E66D62966FAD629728
:10E5E00080E00F94F214AE966CAD7DAD8EAD9FAD14
:10E5F000AE970F94791384E59BE10F94191465E5A8
:10E6000075E585E591E40F94130DA896EEADFFAD89
:10E61000A89785919591A591B49180933C10909382
:10E620003D10A0933E10B0933F10A896EEADFFAD05
:10E63000A897349685919591A591B49180934010B7
:10E6400090934110A0934210B093431060E070E0AB
:10E6500088E492E40F94130D00913410109135105A
:10E660002091361030913710409130105091311078
:10E67000609132107091331080912C1090912D1078
:10E68000A0912E10B0912F103F932F931F930F93B3
:10E690007F936F935F934F93BF93AF939F938F93AA
:10E6A0008DEF9DE19F938F930F94AEAC0F94F988FB
:10E6B00040912C1050912D1060912E1070912F10C0
:10E6C0008091301090913110A0913210B0913310A0
:10E6D000C0903410D0903510E0903610F090371084
:10E6E00021E00FB6F894DEBF0FBECDBF41315742D7
:10E6F0000CF420E08131974214F00C94B784822FFF
:10E7000090E0880F991FFC01EB50F24EA590B49059
:10E71000FC01E351F24E85909490DF92CF929F924C
:10E720008F92BF92AF921F922F9384ED9DE19F93A2
:10E730008F930F94AEAC84EF9BE19F938F930F94D4
:10E74000AEAC0F942A1D80916E008B7F80936E007B
:10E75000EF9880916F008D7F80936F000FB6F894D3
:10E76000A89580916000886180936000109260009D
:10E770000FBE1092030D1092020D88E991E0909364
:10E78000010D8093000D84E491E09093FF0C809341
:10E79000FE0C00E028EC30E0A601B401C5010F94A6
:10E7A000514600913410109135102091361030915F
:10E7B00037104091301050913110609132107091AB
:10E7C000331080912C1090912D10A0912E10B091AB
:10E7D0002F103F932F931F930F937F936F935F930C
:10E7E0004F93BF93AF939F938F9384E99CE19F9343
:10E7F0008F930F94AEAC80912C1090912D10A0911E
:10E800002E10B0912F10782E692E8091301090919B
:10E810003110A0913210B0913310582E492EC09073
:10E820003410D0903510E0903610F09037100FB6BD
:10E83000F894DEBF0FBECDBF4BE0242E4CE1342E4A
:10E8400095E0C91697EFD9060CF46EC01A821982AA
:10E850001F921F92A3E0AF93B4E8BF931F92E4E628
:10E86000EF93DF92CF924F925F926F927F923F929F
:10E870002F920F94AEAC0FB6F894DEBF0FBECDBF93
:10E8800089819A81803D924030F089819A81803AD5
:10E89000954050F512C0CE0101967C0100E010E0D9
:10E8A00024E833E0A601652D742D872D962D0F9455
:10E8B000546281110C94BC84E8CFDE0111967D0175
:10E8C00000E010E02CE73CEFA60144565109652D0D
:10E8D000742D872D962D0F945462882329F08981F9
:10E8E0009A8180539D4F1CC089819A8180379840BE
:10E8F00008F04AC0FE0131967F0104EB10E024E8E5
:10E9000033E0A601485C5109652D742D872D962DA5
:10E910000F9454628823C1F189819A8180569A4F5D
:10E920009A8389830C94BC84009134101091351023
:10E9300020913610309137104091301050913110A5
:10E94000609132107091331080912C1090912D10A5
:10E95000A0912E10B0912F103F932F931F930F93E0
:10E960007F936F935F934F93BF93AF939F938F93D7
:10E9700083E49CE19F938F930F94AEAC0FB6F89411
:10E98000DEBF0FBECDBFD8C389819A8180349B4042
:10E99000A0F49E012F5F3F4F790104EB10E02CE7BC
:10E9A0003CEFA6014C525140652D742D872D962DBC
:10E9B0000F94546281110C94A38580E0E981FA815F
:10E9C000882311F40C94BF8480912C1090912D1009
:10E9D000A0912E10B0912F10409130105091311015
:10E9E00060913210709133100091341010913510F5
:10E9F0002091361030913710FF93EF931F930F93B0
:10EA00005F934F939F938F9380E79CE19F938F93A6
:10EA10000F94AEAC40913410509135106091361087
:10EA20007091371000E028EC30E0B401C5010F947C
:10EA3000514685E08F9380E78F9384EA9DE19F9311
:10EA40008F930F94AEAC84E08F9388E38F9382E929
:10EA50009DE19F938F930F94AEAC80912C10909179
:10EA60002D10A0912E10B0912F106A968CAF9DAFF3
:10EA7000AEAFBFAF6A976896CEACDFAC68978091B7
:10EA8000301090913110A0913210B0913310E29675
:10EA90008CAF9DAFAEAFBFAFE29780913410909135
:10EAA0003510A0913610B09137106E968CAF9DAF97
:10EAB000AEAFBFAF6E971C0198E4291A310889E008
:10EAC0008F9380E68F933F922F92E096AFADE097C1
:10EAD000AF93AF96BFADAF97BF936896EFAD689712
:10EAE000EF936796FFAD6797FF938DEB9CE19F9344
:10EAF0008F930F94AEAC40913410509135106091CB
:10EB00003610709137107A0120E931E0E0966EAD51
:10EB10007FADE09768968EAD9FAD68970F94514694
:10EB2000E0962EAD3FADE0973450EC963FAF2EAF60
:10EB3000EC970FB6F894DEBF0FBECDBF812C912CA1
:10EB4000D601B450E896BFAFAEAFE897F601FC5FD0
:10EB5000C258DF4FF983E883CE57D040382D31704B
:10EB6000A3963FAFA39780FC02C00C94C584EF9698
:10EB70008FADEF97C158DF4F9881CF57D04000E05D
:10EB800020E931E0A701EC966EAD7FADEC970F94D4
:10EB90005146C0903010D0903110E0903210F0907B
:10EBA000331080912C1090912D10A0912E10B091C7
:10EBB0002F1001E028EC30E0A101B6010F9451467E
:10EBC000C0903010D0903110E0903210F09033109F
:10EBD00080912C1090912D10A0912E10B0912F109B
:10EBE0000FEF28EC30E040E659E0B6010F945146B3
:10EBF0008091341090913510A0913610B09137105B
:10EC00007C01A3966FADA39780910B01662311F44D
:10EC10000C94CD84816080930B010000840125E079
:10EC2000000F111F2A95E1F7A3968FADA3978823B4
:10EC300011F40C94D08490EC492E55245A94652CF0
:10EC4000752CC12CD12C90E4E3969FAFE397A12CB7
:10EC5000B12C93B1A70142195309292F207194FFB8
:10EC600002C00C94D78488EE9FEF840F951F97FD08
:10EC700002C00C94DB8480E090E0A80EB91E809165
:10EC80000B0121110C94E584846080930B0100003A
:10EC900021110C94E8842E143F0434F484E00F9482
:10ECA0002A7BA1E0EA1AF10881E00F942A7B8BE528
:10ECB00099E00197F1F7E396FFADE397F150E39602
:10ECC000FFAFE397F111C5CFB6E0B694A794BA951C
:10ECD000E1F7A3962FADA397222311F40C94F784A8
:10ECE0008FE190E08C199D09800F911FFC01E25784
:10ECF000F84FA08280912C1090912D10A0912E1091
:10ED0000B0912F10840D951DA61DB71D80932C105A
:10ED100090932D10A0932E10B0932F10C7010F2C9D
:10ED2000000CAA0BBB0B8093341090933510A0936A
:10ED30003610B09337103FEFC31AD30A60E2C616FD
:10ED4000D10409F080CF0257184FF0E2BF2EA8EB94
:10ED5000CA2EACE1DA2ED8018D918D011F928F93CE
:10ED6000DF92CF920F94AEACBA940F900F900F90A9
:10ED70000F90B110F0CF86EB9CE19F938F930F948F
:10ED8000AEACBFEF8B1A9B0AEC96EEADFFADEC97E5
:10ED9000E05CFF4FEC96FFAFEEAFEC970F900F905B
:10EDA000F0E28F16910409F0D9CEEEE8AE2EEBE03A
:10EDB000BE2E8EEA9BE0F501119211928E179F07ED
:10EDC000D9F780E090E0DC0175E0AA0FBB1F7A95CF
:10EDD000E1F7A257B84F40E2ED91F0E054E0F5952D
:10EDE000E7955A95E1F7EE0FFF1FE257F44F2081A8
:10EDF00031812F5F3F4F31832083415069F7019666
:10EE00008032910501F72EE8C22E2BE0D22E00E0D1
:10EE100010E035EFE32E3CE1F32ED6018C911196F4
:10EE20009C91B2E0CB0ED11C9F938F931F930F93B5
:10EE3000FF92EF920F94AEAC0F5F1F4F0F900F90A9
:10EE40000F900F900F900F900031110531F78091C6
:10EE5000900B9091910BE0E9FBE031E021E04191D2
:10EE600051918417950710F4322FCA012F5F20317A
:10EE7000B1F7032F1F923F939F938F938CE19DE1F6
:10EE80009F938F930F94AEACECEAFBE00F900F9042
:10EE90000F900F900F900F908EE0329122912A30B8
:10EEA000310510F40C94FA848295807F20918E0BAA
:10EEB00030918F0B2037334010F00C940185000FF8
:10EEC000000F000F182F101B1F921F931F928F937C
:10EED0001F920F9385E09DE19F938F930F94AEACAB
:10EEE0009EE8492E97E0592E0FB6F894DEBF0FBE6C
:10EEF000CDBFF201202F30E0012F10E0808190E0A3
:10EF00002817390710F00C940485821B930B982F57
:10EF100080E0B8010F94CDBA6F3F710519F010F081
:10EF20006FEF70E06193AE16BF0641F700E010E0AE
:10EF3000B0E0AB2EBDE1BB2E8EEFC82E8CE1D82EFB
:10EF4000C801A5E0880F991FAA95E1F7DC01A25737
:10EF5000B84F7D01912CF70181917F011F928F9312
:10EF6000BF92AF920F94AEAC93940F900F900F900E
:10EF70000F90F0E29F12EFCFDF92CF920F94AEACE2
:10EF80000F5F1F4F0F900F9000321105C9F68AE7EF
:10EF90009DE126EE3BE0AEECBBE0FC0145915491D7
:10EFA0004D935D9302962A173B07B9F7612C712C9C
:10EFB000E12CF12C10E000E0A12C40E050E0EB96B9
:10EFC0004FAFEB972EEC3BE0E8963FAF2EAFE897C4
:10EFD000A0E0B0E080E090E0B12C4A01860C971CE4
:10EFE00020E030E014012A0E3B1E6EEF6B0DE3961D
:10EFF0006FAFE397B1100C9408856EEF620F683025
:10F0000010F40C940F852F5F3F4F2C30310591F792
:10F01000B3949096E896EEADFFADE8973296E896F9
:10F02000FFAFEEAFE897FCE0BF12DACFE816F906C3
:10F030002CF47C010A2DEB961FADEB974F5F5F4FD1
:10F040004431510509F0BBCFA39420E2620E711C3C
:10F0500034E1A312B2CFFF92EF921F920F931F924F
:10F060001F9380E39DE19F938F930F94AEAC0FB6F7
:10F07000F894DEBF0FBECDBF93E4E916F10414F49B
:10F080000C9445851F920F931F921F9381E69DE17B
:10F090009F938F930F94AEAC1A5FE12EF12CA0E1F9
:10F0A000EA1AF108E6E0EE0CFF1CEA95E1F7689633
:10F0B000EEADFFAD6897EE0EFF1E0A5FC02ED12C9D
:10F0C000F0E1CF1AD108F6E0CC0CDD1CFA95E1F79F
:10F0D000E0962EAD3FADE097C20ED31E6C963FADCD
:10F0E0006C973F936B966FAD6B976F93DF92CF9258
:10F0F000FF92EF9280E59DE19F938F930F94AEACCA
:10F1000000E028EC30E06C964EAD5FAD6C97B60138
:10F11000C7010F9451460FB6F894DEBF0FBECDBFA6
:10F1200081E0D2011D922D01BEEF4B16BCE05B06C3
:10F13000C1F781110C94488510E08DEB9DE19F9300
:10F140008F930F94AEAC0F94063F80916E00846055
:10F1500080936E00EF9A80916F00826080936F00C1
:10F1600098E288E10FB6F894A895809360000FBEEE
:10F17000909360001092030D1092020D1092010DF9
:10F180001092000D1092FF0C1092FE0C0F900F9039
:10F19000112311F40C94E88320E030E0A901A0963B
:10F1A000EEADFFADA09761817281838194810F9450
:10F1B0003AA820913C1030913D1040913E10509162
:10F1C0003F100F942EB6A096AEADBFADA09711968E
:10F1D0006D937D938D939C931497C0904010D09025
:10F1E0004110E0904210F090431020E030E0A9017F
:10F1F00015966D917D918D919C9118970F943AA8D9
:10F20000A70196010F942EB6A096EEADFFADA09784
:10F21000658376838783908720E030E040E850EC78
:10F22000C701B6010F9442AD87FF0CC080E090E0AB
:10F23000A0E8B0EC8093401090934110A09342104E
:10F24000B093431020E030E040E450E4609144107B
:10F250007091451080914610909147100F942EB6F2
:10F26000609344107093451080934610909347101C
:10F27000AE968CAD9DADAEADBFADAE970196A11D66
:10F28000B11DAE968CAF9DAFAEAFBFAFAE97A89697
:10F29000AEADBFADA8971896A896BFAFAEAFA89772
:10F2A000A096EEADFFADA0973896A096FFAFEEAF5B
:10F2B000A097AE968CAD9DADAEADBFADAE970597A8
:10F2C000A105B10509F087C980E090E00F94B70C63
:10F2D00020E030E040E950EC609196157091971570
:10F2E00080919815909199150F9442AD87FF43C076
:10F2F000E0E7FEE184918F01882339F00F94B9761D
:10F300000F5F1F4FF8018491F7CF8AE00F94B97611
:10F31000EEE3FEE184918F01882339F00F94B976F2
:10F320000F5F1F4FF8018491F7CF60919615709190
:10F330009715809198159091991542E00F943E771A
:10F34000EAE3FEE184918F01882339F00F94B976C6
:10F350000F5F1F4FF8018491F7CF42E060E070E04B
:10F3600080E990EC0F943E770F94B777F2E0AF9678
:10F37000FFAFAF9703C0AF961FAEAF971092C21505
:10F380001092C3151092C4151092C5151092C6158F
:10F390001092C7151092C8151092C91524E6EB9665
:10F3A0002FAFEB97A2961CAE1DAE1EAE1FAEA2975E
:10F3B0006A961CAE1DAE1EAE1FAE6A97CE010196B8
:10F3C00064969FAF8EAF6497DE01AF5BBF4F6696CA
:10F3D000BFAFAEAF66976A966CAD7DAD8EAD9FAD9B
:10F3E0006A970F9419B7AA966CAF7DAF8EAF9FAF97
:10F3F000AA976A966CAD7DAD8EAD9FAD6A970F945E
:10F40000A8B9C457DF4F688379838A839B83CC581C
:10F41000D040A2966CAD7DAD8EAD9FADA2970F94FE
:10F4200019B7C057DF4F688379838A839B83C0599C
:10F43000D040A2966CAD7DAD8EAD9FADA2970F94DE
:10F44000A8B9CC56DF4F688379838A839B83C459DC
:10F45000D0406496EEADFFAD649720E411922A95FA
:10F46000E9F76696AEADBFAD6697E0E11D92EA950D
:10F47000E9F780E090E00F94B70C8091C21590916D
:10F48000C315A091C415B091C515C655DF4F88832B
:10F490009983AA83BB83CA5AD0408091C6159091A4
:10F4A000C715A091C815B091C915C255DF4F888303
:10F4B0009983AA83BB83CE5AD040DE01AF5BBF4F96
:10F4C000C856DF4FB983A883C859D040FE01319692
:10F4D000AC96FFAFEEAFAC9700E0CC56DF4F888123
:10F4E0009981AA81BB81C459D040B058E6968CAFAF
:10F4F0009DAFAEAFBFAFE697C057DF4F8881998110
:10F50000AA81BB81C059D040B058EA968CAF9DAF5C
:10F51000AEAFBFAFEA97C457DF4F88819981AA8108
:10F52000BB81CC58D040B058C258DF4F88839983F4
:10F53000AA83BB83CE57D040AC962EAC3FACAC97E1
:10F5400010E061E9462E65E1562E74E0772EC12C5D
:10F55000D12C7601013011F40C94CB85113011F4CB
:10F560000C94D785002311F1023081F4D201119659
:10F570002D913D914D915C911497C258DF4F688158
:10F5800079818A819B81CE57D0400BC0F2012581C1
:10F59000368147815085EA966CAD7DAD8EAD9FADCD
:10F5A000EA970F943AA84B015C0106C0812C912C7C
:10F5B00050E8A52E5FE3B52E112301F1123081F43E
:10F5C000D20111962D913D914D915C911497C258A5
:10F5D000DF4F688179818A819B81CE57D0400BC0F3
:10F5E000F2012581368147815085EA966CAD7DAD6B
:10F5F0008EAD9FADEA970F943AA804C060E070E02A
:10F6000080E89FE39B01AC01C501B4010F943AA8C7
:10F610009B01AC01C701B6010F942EB66B017C01B2
:10F620000023E1F11123D1F1023011F00C94AB85EC
:10F63000D20111962D913D914D915C911497AA960E
:10F640006CAD7DAD8EAD9FADAA970F943AA84B01DE
:10F650005C01113011F40C94C585123011F00C943A
:10F66000B885D20111962D913D914D915C911497E1
:10F67000AA966CAD7DAD8EAD9FADAA970F943AA8BA
:10F680009B01AC01C501B4010F943AA89B01AC01E8
:10F69000C701B6010F942EB66B017C017A94F8E095
:10F6A0004F0E511C711056CFD101CD92DD92ED92CB
:10F6B000FD921D011F5F143009F043CF31E9232E65
:10F6C00035E1332EE1E7FEE16C96FFAFEEAF6C97CC
:10F6D000CA57DF4F1882C658D040C456DF4F188231
:10F6E000CC59D040C056DF4F1882C05AD04010E0ED
:10F6F000002321F1013049F1023081F4D10111964A
:10F700002D913D914D915C911497C258DF4F6881C6
:10F7100079818A819B81CE57D0400BC0F101258130
:10F72000368147815085EA966CAD7DAD8EAD9FAD3B
:10F73000EA970F943AA84B015C010AC0812C912CE6
:10F7400020E8A22E2FE3B22E03C0812C912C54016D
:10F75000D10111964D905D906D907C901497A3010E
:10F760009201AA966CAD7DAD8EAD9FADAA970F9418
:10F770003AA86B017C01D10115968D919D910D9058
:10F78000BC91A02DA6968CAF9DAFAEAFBFAFA69794
:10F790006C96EEADFFAD6C9785919591A591B49166
:10F7A000CC55DF4F88839983AA83BB83C45AD0404A
:10F7B000A6962CAD3DAD4EAD5FADA697CC56DF4FB6
:10F7C000688179818A819B81C459D0400F943AA87D
:10F7D0009B01AC01C701B6010F942DB6C655DF4F92
:10F7E000288139814A815B81CA5AD0400F942EB654
:10F7F000CC55DF4F288139814A815B81C45AD04082
:10F800000F942DB6A50194010F943AA8CA57DF4F63
:10F810002881C658D040C456DF4F3881CC59D040DB
:10F82000C056DF4F4881C05AD040512F0F942EB69A
:10F83000CA57DF4F688379838A839B83C658D04039
:10F840000023A9F00130B9F00230D9F0A6962CAD12
:10F850003DAD4EAD5FADA697E6966CAD7DAD8EAD80
:10F860009FADE6970F943AA86B017C010AC0C12CAA
:10F87000D12C760106C0C12CD12C90E8E92E9FE353
:10F88000F92E6C96EEADFFAD6C9734968590959001
:10F89000A590B490A3019201C457DF4F688179818C
:10F8A0008A819B81CC58D0400F943AA82B013C010F
:10F8B000A6962CAD3DAD4EAD5FADA697C057DF4FC0
:10F8C000688179818A819B81C059D0400F943AA880
:10F8D0009B01AC01C301B2010F942EB6C255DF4F9C
:10F8E000288139814A815B81CE5AD0400F942EB64F
:10F8F000A50194010F942DB6A70196010F943AA883
:10F90000CA57DF4F288139814A815B81C658D04070
:10F910000F942EB6CA57DF4F6883C658D040C456DE
:10F92000DF4F7883CC59D040C056DF4F8883C05A10
:10F93000D040192F6C96AEADBFAD6C9718966C96F3
:10F94000BFAFAEAF6C97B8E02B0E311CE1EB2E16BB
:10F95000E5E13E0609F0CCCEDC01CB01B058C8563B
:10F96000DF4FE881F981C859D04081939193A193E9
:10F97000B193C856DF4FF983E883C859D0400F5F71
:10F98000AC962EAD3FADAC97205F3F4FAC963FAFEE
:10F990002EAFAC97043009F0CFCD25968CAD9DAD40
:10F9A000AEADBFAD2597AA968CAF9DAFAEAFBFAF42
:10F9B000AA978D819E81AF81B885AE968CAF9DAFA1
:10F9C000AEAFBFAFAE9789859A85AB85BC85A6964D
:10F9D0008CAF9DAFAEAFBFAFA6978D859E85AF852F
:10F9E000B889E6968CAF9DAFAEAFBFAFE697898181
:10F9F0009A81AB81BC81EA968CAF9DAFAEAFBFAFB1
:10FA0000EA9729968CAD9DADAEADBFAD2997C25892
:10FA1000DF4F88839983AA83BB83CE57D0408989DF
:10FA20009A89AB89BC89C457DF4F88839983AA839D
:10FA3000BB83CC58D040898D9A8DAB8DBC8DC0577F
:10FA4000DF4F88839983AA83BB83C059D0408D8DB3
:10FA50009E8DAF8DB8A1CC56DF4F88839983AA8342
:10FA6000BB83C459D0408D899E89AF89B88DC85653
:10FA7000DF4F88839983AA83BB83C859D0402D96D2
:10FA80008CAD9DADAEADBFAD2D97CA57DF4F88830E
:10FA90009983AA83BB83C658D04089A19AA1ABA100
:10FAA000BCA1C456DF4F88839983AA83BB83CC59FA
:10FAB000D0408DA19EA1AFA1B8A5C056DF4F8883CD
:10FAC0009983AA83BB83C05AD0408DA59EA5AFA5BC
:10FAD000B8A9CC55DF4F88839983AA83BB83C45AC6
:10FAE000D04089A59AA5ABA5BCA5CE54DF4F88838D
:10FAF0009983AA83BB83C25BD04061968CAD9DADD8
:10FB0000AEADBFAD6197CA54DF4F88839983AA8396
:10FB1000BB83C65BD04089A99AA9ABA9BCA9C6542E
:10FB2000DF4F88839983AA83BB83CA5BD0408DA9AA
:10FB30009EA9AFA9B8ADC254DF4F88839983AA8329
:10FB4000BB83CE5BD04089AD9AADABADBCADCE53DF
:10FB5000DF4F88839983AA83BB83C25CD040219600
:10FB60008CAD9DADAEADBFAD2197CA53DF4F88833D
:10FB70009983AA83BB83C65CD04014E6C12CD12CE8
:10FB800076014601570126013701A3019201AE9685
:10FB90006CAD7DAD8EAD9FADAE970F943AA89B0135
:10FBA000AC01AA966CAD7DAD8EAD9FADAA970F94BA
:10FBB0002DB62B013C01A5019401A6966CAD7DAD3F
:10FBC0008EAD9FADA6970F943AA89B01AC01C301DF
:10FBD000B2010F942DB62B013C01A7019601E696C8
:10FBE0006CAD7DAD8EAD9FADE6970F943AA89B01AD
:10FBF000AC01C301B2010F942DB6EA962CAD3DAD18
:10FC00004EAD5FADEA970F941CB76E966CAF7DAFAB
:10FC10008EAF9FAF6E97C457DF4F288139814A81DD
:10FC20005B81CC58D0400F943AA89B01AC01C258DC
:10FC3000DF4F688179818A819B81CE57D0400F94B4
:10FC40002DB62B013C01A5019401C057DF4F6881FF
:10FC500079818A819B81C059D0400F943AA89B0139
:10FC6000AC01C301B2010F942DB64B015C01A70199
:10FC70009601CC56DF4F688179818A819B81C45976
:10FC8000D0400F943AA89B01AC01C501B4010F9478
:10FC90002DB6C856DF4F288139814A815B81C8590A
:10FCA000D0400F941CB72B013C01C456DF4F288174
:10FCB00039814A815B81CC59D0406E966CAD7DAD67
:10FCC0008EAD9FAD6E970F943AA89B01AC01CA57B9
:10FCD000DF4F688179818A819B81C658D0400F941B
:10FCE0002DB64B015C01C056DF4F288139814A8116
:10FCF0005B81C05AD040C301B2010F943AA89B0166
:10FD0000AC01C501B4010F942DB64B015C01A701F4
:10FD10009601CC55DF4F688179818A819B81C45AD5
:10FD2000D0400F943AA89B01AC01C501B4010F94D7
:10FD30002DB6CE54DF4F288139814A815B81C25B69
:10FD4000D0400F941CB74B015C01C654DF4F288193
:10FD500039814A815B81CA5BD0406E966CAD7DADC6
:10FD60008EAD9FAD6E970F943AA89B01AC01CA541B
:10FD7000DF4F688179818A819B81C65BD0400F9477
:10FD80002DB66B017C01C254DF4F288139814A8135
:10FD90005B81CE5BD040C301B2010F943AA89B01B6
:10FDA000AC01C701B6010F942DB66B017C01CE5397
:10FDB000DF4F288139814A815B81C25CD040C50117
:10FDC000B4010F943AA89B01AC01C701B6010F948E
:10FDD0002DB6CA53DF4F288139814A815B81C65CC9
:10FDE000D0400F941CB76B017C01115009F0CDCEAF
:10FDF0006E962CAD3DAD4EAD5FAD6E97C655DF4FE7
:10FE0000688179818A819B81CA5AD0400F942EB62D
:10FE10006093C2157093C3158093C4159093C51554
:10FE2000A3019201C255DF4F688179818A819B814C
:10FE3000CE5AD0400F942EB66093C6157093C71556
:10FE40008093C8159093C915A50194016A966CAD6D
:10FE50007DAD8EAD9FAD6A970F942EB66A966CAF4E
:10FE60007DAF8EAF9FAF6A97A7019601A2966CAD4A
:10FE70007DAD8EAD9FADA2970F942EB6A2966CAFBE
:10FE80007DAF8EAF9FAFA297EB969FADEB97915052
:10FE9000EB969FAFEB9791119ECA6A966CAD7DADC4
:10FEA0008EAD9FAD6A970F9419B76093B21570939A
:10FEB000B3158093B4159093B5156A966CAD7DAD6E
:10FEC0008EAD9FAD6A970F94A8B96093B6157093E5
:10FED000B7158093B8159093B915A2966CAD7DAD0A
:10FEE0008EAD9FADA2970F94A8B9DC01CB01B0589D
:10FEF0008093BA159093BB15A093BC15B093BD1514
:10FF0000A2966CAD7DAD8EAD9FADA2970F9419B743
:10FF10006093BE157093BF158093C0159093C11563
:10FF20006A962CAD3DAD4EAD5FAD6A97A2966CADB5
:10FF30007DAD8EAD9FADA2970F942DB66B017C0168
:10FF4000E894F7F8B701A60180E69FE00F94C6B5E4
:10FF50002FE132E449E05BE3C701B6010F9479B8C1
:10FF600018166CF425E33AEF4EE85BE3C701B601DF
:10FF70000F9479B8181634F001E010E005C000E0E5
:10FF800010E002C002E010E025E33AEF4EE85BE348
:10FF90006A966CAD7DAD8EAD9FAD6A979F770F94DD
:10FFA00079B818167CF025E33AEF4EE85BE3A296A9
:10FFB0006CAD7DAD8EAD9FADA2979F770F9479B854
:10FFC000181614F402E010E08091B2159091B31568
:10FFD000A091B415B091B515AE968CAF9DAFAEAFF4
:10FFE000BFAFAE978091BA159091BB15A091BC158B
:10FFF000B091BD15A6968CAF9DAFAEAFBFAFA69723
:020000021000EC
:100000008091C2159091C315A091C415B091C515EA
:10001000EE968CAF9DAFAEAFBFAFEE978091B615A9
:100020009091B715A091B815B091B915E6968CAF1F
:100030009DAFAEAFBFAFE6978091BE159091BF1553
:10004000A091C015B091C115EA968CAF9DAFAEAF2F
:10005000BFAFEA978091C6159091C715A091C815BA
:10006000B091C915C258DF4F88839983AA83BB8397
:10007000CE57D040A1E7BEE16C96BFAFAEAF6C9754
:1000800081E9282E85E1382EF10181809280A380BC
:10009000B48085819681A781B085AA968CAF9DAFEB
:1000A000AEAFBFAFAA976C96EEADFFAD6C97C590A3
:1000B000D590E590F490A5019401AE966CAD7DAD20
:1000C0008EAD9FADAE970F943AA82B013C01AA9636
:1000D0002CAD3DAD4EAD5FADAA97A6966CAD7DAD96
:1000E0008EAD9FADA6970F943AA89B01AC01C301BA
:1000F000B2010F942EB6EE962CAD3DAD4EAD5FAD78
:10010000EE970F942EB69B01AC01C701B6010F9478
:100110002DB66B017C016C96EEADFFAD6C973496FD
:100120004590559065907490E6962CAD3DAD4EADE2
:100130005FADE697C501B4010F943AA84B015C018D
:10014000EA962CAD3DAD4EAD5FADEA97AA966CAD8B
:100150007DAD8EAD9FADAA970F943AA89B01AC01DF
:10016000C501B4010F942EB6C258DF4F28813981E2
:100170004A815B81CE57D0400F942EB69B01AC01D3
:10018000C301B2010F942DB64B015C01A70196018A
:10019000C701B6010F943AA86B017C01A501940137
:1001A000C501B4010F943AA89B01AC01C701B60187
:1001B0000F942EB60F94B3B92DEC3CEC4CE45FE3F6
:1001C0000F9479B8181614F40EEF1FEFB8E02B0E49
:1001D000311C6C96EEADFFAD6C9738966C96FFAF08
:1001E000EEAF6C9721EB35E12215330509F04CCFCA
:1001F0000115110509F07AC1A2962CAD3DAD4EADA9
:100200005FADA2976A966CAD7DAD8EAD9FAD6A97DE
:100210000F942EB620E030E040E05FE30F943AA860
:100220006B017C010F9419B72B013C016093B2154F
:100230007093B3158093B4159093B515C701B601AB
:100240000F94A8B9A2966CAF7DAF8EAF9FAFA29767
:100250006093B6157093B7158093B8159093B91540
:10026000DC01CB01B058AA968CAF9DAFAEAFBFAF4B
:10027000AA978093BA159093BB15A093BC15B09321
:10028000BD154092BE155092BF156092C015709278
:10029000C1151092C2151092C3151092C415109278
:1002A000C5151092C6151092C7151092C815109258
:1002B000C9156E961CAE1DAE1EAE1FAE6E976A9629
:1002C0001CAE1DAE1EAE1FAE6A97CE57DF4FA88183
:1002D000B981C258D04011968D909D90AD90BC9040
:1002E000149715968D919D910D90BC91A02DAE9671
:1002F0008CAF9DAFAEAFBFAFAE97C657DF4FE881B3
:10030000F981CA58D040C590D590E590F490A501E8
:100310009401C301B2010F943AA8A6966CAF7DAFC9
:100320008EAF9FAFA697AE962CAD3DAD4EAD5FADF7
:10033000AE97AA966CAD7DAD8EAD9FADAA970F948A
:100340003AA89B01AC01A6966CAD7DAD8EAD9FAD7C
:10035000A6970F942EB69B01AC01C701B6010F946E
:100360002DB62091C2153091C3154091C4155091FE
:10037000C5150F942EB66B017C016093C215709366
:10038000C3158093C4159093C51520E030E040E874
:100390005FE36A966CAD7DAD8EAD9FAD6A970F94AD
:1003A0002EB66A966CAF7DAF8EAF9FAF6A97C65779
:1003B000DF4FE881F981CA58D040349685919591F4
:1003C000A591B491A6968CAF9DAFAEAFBFAFA697E7
:1003D000A5019401A2966CAD7DAD8EAD9FADA297A7
:1003E0000F943AA84B015C01AE962CAD3DAD4EADDD
:1003F0005FADAE97C301B2010F943AA89B01AC0167
:10040000C501B4010F942EB69B01AC01A6966CAD4C
:100410007DAD8EAD9FADA6970F942DB62091C615DC
:100420003091C7154091C8155091C9150F942EB63B
:100430004B015C016093C6157093C7158093C81576
:100440009093C91520E030E040E85FE36E966CAD14
:100450007DAD8EAD9FAD6E970F942EB66E966CAF40
:100460007DAF8EAF9FAF6E97CE57DF4FA881B9811A
:10047000C258D0401896CE57DF4FB983A883C258D0
:10048000D040C657DF4FE881F981CA58D04038962E
:10049000C657DF4FF983E883CA58D0402A163B0677
:1004A00009F013CF6A962CAD3DAD4EAD5FAD6A97A6
:1004B000C701B6010F941CB76093C2157093C315A2
:1004C0008093C4159093C5156E962CAD3DAD4EAD81
:1004D0005FAD6E97C501B4010F941CB76093C6154C
:1004E0007093C7158093C8159093C9154090B215A5
:1004F0005090B3156090B4157090B515C090BE15AE
:10050000D090BF15E090C015F090C1158091B61540
:100510009091B715A091B815B091B915A2968CAF6E
:100520009DAFAEAFBFAFA2978091BA159091BB15AA
:10053000A091BC15B091BD156A968CAF9DAFAEAFC2
:10054000BFAF6A97A7019601C301B2010F943AA801
:100550004B015C016A962CAD3DAD4EAD5FAD6A9727
:10056000A2966CAD7DAD8EAD9FADA2970F943AA8CB
:100570009B01AC01C501B4010F942DB64B015C0188
:100580009B01AC01C701B6010F941CB76B017C0144
:100590006A966CAD7DAD8EAD9FAD6A979058A50102
:1005A00094010F941CB76A966CAF7DAF8EAF9FAF6E
:1005B0006A97A2966CAD7DAD8EAD9FADA297905817
:1005C000A50194010F941CB7CE57DF4F6883798340
:1005D0008A839B83C258D040A5019401C301B20114
:1005E0000F941CB74B015C014090C2155090C3158D
:1005F0006090C4157090C5158091C6159091C7156F
:10060000A091C815B091C915A2968CAF9DAFAEAFA1
:10061000BFAFA297C092B215D092B315E092B415B5
:10062000F092B515CE57DF4F88819981AA81BB81A1
:10063000C258D0408093B6159093B715A093B815C3
:10064000B093B9156A968CAD9DADAEADBFAD6A974E
:100650008093BA159093BB15A093BC15B093BD15AC
:100660008092BE159092BF15A092C015B092C11590
:10067000C701B6019058A30192010F943AA86B01EB
:100680007C01A2962CAD3DAD4EAD5FADA2976A96B2
:100690006CAD7DAD8EAD9FAD6A970F943AA89B016E
:1006A000AC01C701B6010F942DB66093C2157093CB
:1006B000C3158093C4159093C515CE57DF4F68813D
:1006C00079818A819B81C258D0409058A3019201C0
:1006D0000F943AA86B017C01A2962CAD3DAD4EADB6
:1006E0005FADA297C501B4010F943AA89B01AC017C
:1006F000C701B6010F942DB66093C6157093C71548
:100700008093C8159093C91580E090E00F94B70CC2
:1007100017FD53C042EC55E16AEB75E182EB95E1C0
:100720000F94FC0D4091C2155091C3156091C415F2
:100730007091C51585EE9FE00F94C6B54091C61522
:100740005091C7156091C8157091C91589EE9FE049
:100750000F94C6B54091B2155091B3156091B41580
:100760007091B5158DED9FE00F94C6B54091B6150B
:100770005091B7156091B8157091B91581EE9FE051
:100780000F94C6B54091BA155091BB156091BC1538
:100790007091BD1585ED9FE00F94C6B54091BE15D3
:1007A0005091BF156091C0157091C11589ED9FE002
:1007B0000F94C6B50F94810D09C00E3F9FEF190726
:1007C00029F4AF96AFADAF97A23049F038010BC016
:1007D000AF961FAEAF9766246A94762C04C0BEEF26
:1007E0006B2E77247A94C855DF4F88819981C85A37
:1007F000D0400F94F56480E090E0A0EAB0E48093EC
:10080000441090934510A0934610B0934710209148
:10081000401030914110409142105091431060912E
:100820003C1070913D1080913E1090913F10E6E099
:10083000FDE0FF93EF93812C912CE0EAAE2EE1E4F2
:10084000BE2EF8E4CF2EF0E1DF2EE12CF12C00EAF1
:1008500010E40F94C8300F94F9880F900F9077FC34
:1008600022C020E030E046E153E4609144107091F2
:10087000451080914610909147100F942EB66093CA
:10088000441070934510809346109093471065E58F
:1008900075E585E591E40F94130D89EB99E10E94CC
:1008A00033E00F94201581E00F94AB1982E00F9490
:1008B0001712BFEF6B167B0631F48CE799E10E94AB
:1008C00033E010E04BC0EEEF6E16EFEF7E0681F4E2
:1008D000AF96FFADAF97FF2329F0F23031F085E3FB
:1008E00098E1EDCF8AEB98E1EACF8AE798E1E7CF8C
:1008F000AF962FADAF97211107C033E06316710497
:1009000098F08AEB98E117C0AF966FADAF97623061
:1009100019F487E399E102C08DEE98E10E9433E07B
:100920001614170454F309C0F301EE0FFF1FE3532D
:10093000FD4F808191810E9433E06720609409F22D
:1009400086EE0F94F1688FE59FE00F94A2B5813099
:1009500021F08EED99E10E9433E011E00F94E81947
:100960002BC18DE99EE10E9433E010E025C183E0B8
:10097000821B282F0C947F7381E00C94DE74F0E9C5
:10098000CF1AF1E0DF0A0C942074E7968FADE79759
:10099000E8969FADE8970C94BF758E7F0C940B760C
:1009A00080E4482E512C612C712C0C94217687E127
:1009B00090E00C9435768F3F910509F014F40C9477
:1009C0003D768FEF90E00C943D768B7F0C944576CE
:1009D000B0E6EB16B9E0FB0614F00C94547684E014
:1009E0000F942A7BEFEFEE1AFE0A0C945476C601A0
:1009F0000C9474768150883011F00C944D770C94DF
:100A0000547700E00C94627780E090E00C94877754
:100A1000EBE0BE1611F40C94FD77222311F02B307D
:100A200039F4E396FFADE397F83010F00C940378B7
:100A3000B101620F731F6257784FFB01F081A396DB
:100A4000FFAFA397E896EEADFFADE897C080D180E9
:100A500061E070E0022E02C0660F771F0A94E2F791
:100A60006C217D21672B31F0A396FFADA397F13167
:100A700048F005C0A3966FADA397613118F40196B5
:100A80000C94037801970C94037880E00C9491788F
:100A900084EF91E00F949747882311F40C949C788D
:100AA00014E0812C912C5401C12CD12C760188EEBC
:100AB00093E00F949747882311F40C949C788091CD
:100AC0002C1090912D10A0912E10B0912F10092E66
:100AD000000CAA0BBB0BC80ED91EEA1EFB1E809190
:100AE000301090913110A0913210B0913310092E36
:100AF000000CAA0BBB0B880E991EAA1EBB1E115020
:100B0000B1F64090341050903510609036107090CF
:100B10003710C501B40122E09695879577956795C2
:100B20002A95D1F732E0F694E794D794C7943A9592
:100B3000D1F700E028EC30E0A201C6010F94514645
:100B400011E00C949D7829813A812059374F3A83DE
:100B500029830C94DE74F20125813681478150850A
:100B6000E6966CAD7DAD8EAD9FADE6970C94257B82
:100B7000F2012581368147815085E6966CAD7DADC9
:100B80008EAD9FADE6970C943E7B60E070E080E810
:100B90009FE30C94407B112311F40C944E7B812C29
:100BA000912C40E8A42E4FE3B42E0C94297B011124
:100BB0000C94147B0C944E7B81E00F94AB1980E075
:100BC0000F94B06D812FC753DF4F0FB6F894DEBF7F
:100BD0000FBECDBFDF91CF911F910F91FF90EF908E
:100BE000DF90CF90BF90AF909F908F907F906F904D
:100BF0005F904F903F902F90089560E08091931305
:100C00000F94F04361E0809193130F94F04360E000
:100C1000809193130F94F0438BE891E00197F1F7E3
:100C2000089581E00F946D7F0D94D214CF92DF92DE
:100C3000EF92FF920F931F93CF93DF939DEDE92ED9
:100C400096E0F92EC0E0D0E0082F10E0670161E0E7
:100C5000F70181917F010F94C044B8010C2E02C0AE
:100C6000759567950A94E2F76170F60180810F949B
:100C7000F0432196C430D10549F7DF91CF911F9100
:100C80000F91FF90EF90DF90CF90B7CFCF92DF9290
:100C9000EF92FF920F931F93CF93DF93182F8091C2
:100CA00094130F94F043809192138F3F19F060E0FA
:100CB0000F94F04380919713C12FD0E084FF27C099
:100CC0003DEDE32E36E0F32E00E010E0670161E039
:100CD000F70181917F010F94C044BE01002E02C034
:100CE000759567950A94E2F76170F60180810F941B
:100CF000F0430F5F1F4F0830110541F7DF91CF918F
:100D00001F910F91FF90EF90DF90CF9076CFCE01A3
:100D100024E0959587952A95E1F788DF812FDF916B
:100D2000CF911F910F91FF90EF90DF90CF907ECFEA
:100D300060E0ACCF982F8A3071F4809195138430A5
:100D400018F08FEF80939513609195136F5F80E09B
:100D50000F94F21420C1E0918913E11104C08B318A
:100D600009F017C11BC0E230C8F0F0E0E757FC4EB5
:100D7000808380918A1320ED290F2A3060F421E0CE
:100D800030E00090891302C0220F331F0A94E2F76B
:100D90008160822B01C08E7F80938A1340918913DA
:100DA00081E0840F8093891350E04830510508F0AA
:100DB000EDC0FA018827EE58FF4F8F4F0D9410BBFE
:100DC0009B3109F0E3C0E7C010928A139B3509F00C
:100DD000DDC0E1C0923309F4DEC09F3309F4DBC00B
:100DE00080918A1370C080918B13823331F08F33DE
:100DF00059F4923309F0CAC0CEC09A3429F40F9442
:100E0000A11910929513C2C080918A1382FFBEC0AF
:100E10009B3309F058C0BFC080918B138F3349F4C6
:100E200080918C13823309F0B1C0953309F0AEC0C4
:100E3000B2C080918A1382FFA9C020918C132B33FA
:100E400011F480FDA8C083FFA1C09B3309F09EC0B0
:100E5000A2C060918B136F33F9F480918C138233AD
:100E600009F094C080918D13853309F08FC09836B6
:100E700051F09C3609F08AC0809191138D7F809348
:100E80009113886007C080919113982F926090937E
:100E900091138A604DDF7AC080918A1382FF76C0F9
:100EA00020918C132B3341F484FF06C0983459F4FD
:100EB000605380918D133CC083FF68C090918D1367
:100EC0009B3309F063C080FF61C065C020918A1325
:100ED00022FF5CC080918C138B33A1F4322F3073CE
:100EE000303381F4983471F460918B1360538091A6
:100EF0008D13880F8056982F990F990F890F909115
:100F00008E1340C023FF42C030918D133B33F1F567
:100F100025FF3CC0983471F460918B13660F6056C6
:100F2000962F990F990F690F8053680F80918E1338
:100F300080532AC020FF2AC02EC080918A13282FF8
:100F40002C702C3019F520918D132B33F9F4807609
:100F50008036E1F49834D1F460918B13660F6056BB
:100F6000862F880F880F680F80918C138053680F2D
:100F700080918E13880F8056982F990F990F890FA3
:100F800090918F139053890F0F94F214109289133C
:100F900002C061E07BDE81E00895CCDE80E090E07D
:100FA00008951092BF19809102108B7F80930210D8
:100FB000089520913102222359F1FC01808D83FF95
:100FC00003C07195619571098091E60D9091E70DCF
:100FD000680F791F7093E70D6093E60D8091E80D1F
:100FE0009091E90D6817790734F4919581959109ED
:100FF000861797076CF08091030184FF04C08091ED
:1010000005018F7E03C080910501806180930501F9
:101010000895809131028823A9F0809107028823E6
:1010200089F08091360D882369F083E091E20F9476
:10103000D5AC10922F0D1092360D81E080932702CF
:101040001092270D08951092310260E087E69FE02C
:101050000F94B4B51092320208951F920F920FB6FA
:101060000F9211240BB60F921F932F933F934F9320
:101070005F936F937F938F939F93AF93BF93CF9320
:10108000DF93EF93FF9380911810811103C190912A
:10109000030180910F07892784FFFCC08091030121
:1010A00080930F078091390D8111F4C081E0809306
:1010B000390DC091E60DD091E70D1092E70D109219
:1010C000E60D78941091270D8091260D882319F054
:1010D0000F94657B02C00F94337B811110C0B3DF86
:1010E00081E0809317101F928F9385E89FE19F9373
:1010F0008F930F94AEAC0F900F900F900F90809144
:10110000C3199091C4191C161D060CF0AEC097FFB0
:1011100008C02091270D222311F02E5F21C021E06D
:101120001FC0009731F02091270D2223D9F02150C4
:1011300017C02091370D3091380D1216130624F484
:101140002091270D222371F02091E80D3091E90DB7
:10115000359527952C173D072CF42091270D2F5FEF
:101160002093270D2091260D222309F47EC0209183
:10117000250D222331F021502093250D1092270DAB
:1011800074C02091E80D3091E90D4091200D6091DF
:101190001E0D70911F0DC217D30769F51816190699
:1011A000A4F42091230D3091240D8217930784F429
:1011B000280F391F37FF02C02F5F3F4F3595279506
:1011C0003093240D2093230D03C0009709F058C0DD
:1011D0002091210D3091220D2817390764F4280F32
:1011E000391F37FF02C02F5F3F4F3595279530934A
:1011F000220D2093210D4F5F4093200DC60FD71F66
:10120000D0931F0DC0931E0D1816190654F420918B
:101210001C0D30911D0D280F391F30931D0D20938B
:101220001C0D4091270D141770F4242F30E0211B62
:10123000310960911A0D70911B0D260F371F3093E5
:101240001B0D20931A0D2091190D241710F44093B3
:10125000190D4091C6192091170D3091180D240FCA
:10126000311D3093180D2093170D9093380D8093F6
:10127000370D1092C4191092C3191092390D0AC07B
:101280004F5F4093200DC60FD71FD0931F0DC09303
:101290001E0DC7CFFF91EF91DF91CF91BF91AF911D
:1012A0009F918F917F916F915F914F913F912F917E
:1012B0001F910F900BBE0F900FBE0F901F901895AF
:1012C00080913102882309F441C08091070288236C
:1012D000E9F18091360D811139C00F94337B811172
:1012E00014C0B1DE81E0809317101092360D1F926A
:1012F00083E08F9385E89FE19F938F930F94AEAC2B
:101300000F900F900F900F90089582ED90E20F9440
:10131000D5AC8091C3199091C4199093310D8093ED
:10132000300D10922E0D10922F0D0F94FB456093EF
:10133000320D7093330D8093340D9093350D1092D0
:10134000270281E08093360D1092270D08950F93A8
:101350001F93CF9380913102882309F474C0809148
:101360000702882309F46FC0C091360DC11102C075
:10137000A7DF6AC00F94FB450091320D1091330D29
:101380002091340D3091350DDC01CB01801B910B88
:10139000A20BB30B4997A105B10508F454C00F94F3
:1013A000FB456093320D7093330D8093340D909311
:1013B000350D0F94337B811112C045DE81E080939F
:1013C00017101F9282E08F9385E89FE19F938F9380
:1013D0000F94AEAC0F900F900F900F9034C04091CF
:1013E000C3195091C4198091300D9091310D9A011B
:1013F000281B390B80912E0D2115310591F03CF001
:1014000090912F0D290F20932F0D8D5F03C08230F7
:1014100018F0825080932E0D5093310D4093300D73
:1014200005C0882319F0815080932E0D80912E0DD8
:10143000811103C010922F0D06C08C3020F08091D6
:101440002F0D853108F4C0E08C2FCF911F910F91A3
:101450000895CF9380911810811131C00F94BA7BF9
:10146000C82F1F928F9382E79FE19F938F930F94D2
:10147000AEAC0F900F900F900F90CC2319F01092FC
:10148000171003C081E08093171061E0C11101C003
:1014900060E06093310281E0809327021092260D74
:1014A0001092270D1092380D1092370D87E69FE0AD
:1014B0000F94B4B580913102809332020AC0C1E02A
:1014C000C093310261E087E69FE00F94B4B5C0930A
:1014D000320280913102CF910895CF93DF930F9420
:1014E000BA7BC82F1F928F938FE59FE19F938F93B5
:1014F0000F94AEAC87E69FE00F94A2B5D82F87E09B
:101500009FE00F94A2B591E00F900F900F900F9075
:10151000811101C090E09093070285ED9EE00F9449
:10152000A2B591E0813009F090E09093160D2AE089
:1015300037ED43E25FE360919010709191108091DC
:101540009210909193100F943AA80F948DB77093C6
:10155000E90D6093E80DC11104C081E0809317107C
:1015600006C010921710DD2311F073DF01C06BDD90
:1015700080913102811103C081E49FE102C08BE4BC
:101580009FE19F938F9383E59FE19F938F930F94A8
:10159000AEAC0F900F900F900F90DF91CF91089508
:1015A0008DE19FE19F938F930F94AEAC81E0809388
:1015B00027021092270D0F900F908091390E8823EB
:1015C00029F060E070E0CB010C9402CC089580E03B
:1015D0009FE19F938F930F94AEAC0F900F9020E0FC
:1015E00030E0A901CA01B9010C946CCEFC018081E4
:1015F00091818436910524F164E670E00F94E1BA9C
:10160000CB012AE030E0B9010F94E1BA805D80930C
:10161000B41980819181B9010F94E1BACB01B9016C
:101620000F94E1BA805D8093B51980819181B901F1
:101630000F94E1BA805D8093B6191092B7191FC05C
:101640008A3091059CF02AE030E0B9010F94E1BAAC
:10165000605D6093B41980819181B9010F94E1BA02
:10166000805D8093B5191092B61909C06AE070E0E8
:101670000F94E1BA805D8093B4191092B51984EB90
:1016800099E10895FC012081318137FF07C08DE287
:101690008093B41931952195310914C02436310550
:1016A00074F0C90164E670E00F94E1BACB016AE01E
:1016B00070E00F94E1BA805D8093B41906C080E2B7
:1016C0008093B4192A30310564F0EAE0F0E0C901F2
:1016D000BF010F94E1BACB01BF010F94E1BA805D65
:1016E00001C080E28093B519C9016AE070E00F94EF
:1016F000E1BA805D8093B6191092B71984EB99E135
:1017000008958F929F92AF92BF92CF92DF92EF9205
:10171000FF92CF9320E030E048EC52E4FC0160817E
:101720007181828193810F943AA80F948DB74B01F8
:101730005C0197FD12C020E137E240E050E00F94D9
:10174000F4BACA01B9012AE030E040E050E00F9459
:10175000F4BA605D6093B41903C08DE28093B4194C
:10176000640197FE04C0CC24DD24C818D9080D2CD0
:10177000000CEE08FF08C701B60128EE33E040E098
:1017800050E00F94F4BA8AE0882E912CA12CB12C51
:10179000CA01B901A50194010F94F4BA605D609388
:1017A000B519C701B60124E630E040E050E00F94DF
:1017B000F4BACA01B901A50194010F94F4BA605DAD
:1017C0006093B6198EE28093B719C701B601A501DF
:1017D00094010F94F4BAC62FCA01B901A50194016E
:1017E0000F94F4BA605D6093B819C05DC093B919E5
:1017F0001092BA1984EB99E1CF91FF90EF90DF90AE
:10180000CF90BF90AF909F908F900895CF93DF932C
:101810001F921F92CDB7DEB7FC016081718182817A
:1018200093810F948DB77A836983CE0101962ADF65
:101830000F900F90DF91CF9108950E941C318091FD
:101840009C13811102C00E9430E210929C130895F3
:10185000CF939C0140918C1550918D1580919A13D6
:1018600090919B134817590739F4E0919D13F0911B
:101870009E131E161F06A4F1C62FFC01E20FF31FD4
:10188000BF0163597F4F8417950728F481E04617FD
:10189000570738F525C06E3E714000F13496EE3E94
:1018A000F14018F449365105C8F423593F4F421707
:1018B0005307B0F04DEE51E0481B590B60E070E06B
:1018C00081569C4E0F944EBBCC2309F0F894109295
:1018D0009B1310929A13CC2309F0789481E001C0F5
:1018E00080E0CF91089520919D1330919E13211592
:1018F0003105A9F180918C1590918D1540E050E053
:10190000FC01E156FC4EA081A23021F4618172817C
:10191000460F571F2150310929F1FC01EE55FC4EAD
:10192000CF018F599341A191A111FACF01968D3E1C
:10193000E1E09E0738F4FC01E156FC4EE081EE2325
:10194000A9F3DECF8D3EE1E09E07D1F6EFE9F3E1AA
:10195000CF018F599341A191AA23D1F3D1CF80E038
:1019600090E00895CA0108952F923F924F925F929E
:101970006F927F928F929F92AF92BF92CF92DF929F
:10198000EF92FF920F931F93CF93DF93CDB7DEB704
:101990006E970FB6F894DEBF0FBECDBF61E08FE546
:1019A00090E056DF882309F491C42091E40D309132
:1019B000E50D8091E20D9091E30D821B930B8F77E3
:1019C00099278F379105A1F43093E30D2093E20D11
:1019D000E1EFFEE184918F01882339F00F94B9760D
:1019E0000F5F1F4FF8018491F7CF8AE00F94B9760B
:1019F00006EB1FE144E2F42E8091E20D9091E30D9D
:101A00002091E40D3091E50D821B930B8F77992780
:101A1000892B09F4C2C18091390E882329F0809165
:101A20004207882309F4B9C10F941576E82E0F9464
:101A3000FB456093651670936616809367169093C6
:101A400068160F94FB45E7FCD7CF2091981330918F
:101A50009913FAE0EF1639F04DE0E41621F02F3536
:101A600031050CF47FC12115310519F410922D0DAB
:101A70002DC4C0909A13D0909B13C6010396215693
:101A80003C4EF901E80FF91F108220912D0D211114
:101A90004FC11092290D10922A0D10922B0D109209
:101AA0002C0DFC01E156FC4E5F0169E773E0CF01AC
:101AB0000F94ABBB892B09F07DC0F50180818E347A
:101AC00009F078C04AE050E060E070E0C6018D5552
:101AD0009C4E0F9462AA6093290D70932A0D8093F7
:101AE0002B0D90932C0D8090120D9090130DA090C3
:101AF000140DB090150D24013501FFEF4F1A5F0A48
:101B00006F0A7F0AC0909A13D0909B1364157505D5
:101B10008605970509F4E6C16CEE7EE1C6018E5597
:101B20009C4E0F94F1AB892B09F0DCC1E5E6FEE594
:101B300084918F01882339F00F94B9760F5F1F4F7E
:101B4000F8018491F7CFEFE9F0E284918F018823C7
:101B500039F00F94B9760F5F1F4FF8018491F7CFDA
:101B6000C501B4010F94546C8AE00F94B9760F94B8
:101B7000D80C1092991310929813A8C3E091100DED
:101B8000F091110D1082E0919A13F0919B13E156A0
:101B9000FC4EF3828091290D90912A0DA0912B0D7E
:101BA000B0912C0D8093120D9093130DA093140DF2
:101BB000B093150D80919A1390919B139C012E5513
:101BC0003C4E6901F90180818E3461F1843251F11A
:101BD0006AE270E0C9010F9473BB892B19F1E5E645
:101BE000FEE584918F01882339F00F94B9760F5F59
:101BF0001F4FF8018491F7CFECE2F0E284918F015E
:101C0000811109C06091120D7091130D8091140D16
